:020000040800F2
:100000000050002029360108C936010811200108D6
:10001000C9360108C9360108C936010800000000C8
:10002000000000000000000000000000C9360108C8
:10003000C936010800000000C936010877B200087F
:10004000C9360108C9360108C9360108C936010890
:10005000C9360108C936010801650008FF640008B7
:10006000C9360108C9360108C9360108C936010870
:10007000C9360108C936010875E00008C93601080B
:1000800003650008C9360108C9360108C9360108E8
:10009000C9360108C9360108C9360108FD640008DF
:1000A000C936010841DE0008C936010851DE0008E2
:1000B00035DE000825DE000815DE00089153000833
:1000C00095530008895300088D530008C93601086C
:1000D000C936010869E000085DE0000851E0000849
:1000E00085B20008C9360108C936010800000000C1
:1000F0000000000000000000000000000000000000
:0C01000000000000000000005FF808F1A3
:100110002DE9F04F754B764EA3B03360002373602A
:1001200010F00DFA18B910F02DFA0AF0A9F80AF03B
:1001300071F9704A704C1378704D43F001031370DD
:1001400000230A930B930C934FF4E0130D93236851
:10015000287B43F480332360A36943F01003A36139
:10016000236803F400330B930A9B01330A930B9B20
:100170001BB90A9BB3F5A06FF2D123685E4913F453
:10018000003301D0022315E00A6842F001020A6040
:100190000A93236803F002030B930A9B01330A932B
:1001A0000B9B1BB90A9BB3F5A06FF2D123689B0789
:1001B00039D501230C93524B52491A6842F0100270
:1001C0001A601A6822F003021A601A6842F00202EA
:1001D0001A606368636063686360636843F48063A4
:1001E0006360494B1A68043B22F070425A60474AE8
:1001F0001160616821F47C116160596841F000412F
:100200005960D96821F40041D9609B681F0449BF37
:100210003F4B4FF4E01313604FF480130D930C9B8E
:10022000012B01D117E0FEE7022B18D168B10D9B1D
:10023000B3F5801F02D14FF4A01305E00D9BB3F579
:10024000E01F02D14FF400130D930D9963680B4327
:1002500043F4803302E0636843F46013636023680F
:1002600043F0807323602168234B8901FBD55968D3
:1002700021F003015960596841F002015960636837
:100280001D4903F00C03082BF9D14B68DFF88C8073
:1002900003F00C03042B03D0082B03D0194B12E0FE
:1002A000136810E04B684868C3F38343C70303F146
:1002B000020301D4174905E0496811F4003F1168B1
:1002C00018BF49084B43C8F8003063681249C3F3AC
:1002D00003130B44197ED8F80030CB40C8F8003027
:1002E0001368084A93421BD101221DE0F79A0008C7
:1002F000C0000020FC2F002000100240FC2700203E
:100300000020024000127A0004100140300000205A
:10031000001BB70000093D00107101084C000020CF
:100320008A4A934202D10222894B1A70DFF878A2DE
:10033000884BDFF878C2CAF80C30A3690DF1880B3E
:1003400043F00103A361636A834FB360636A60464D
:1003500043F080736362A3694FF0000943F01C030C
:10036000A3614FF6FF732BF82C3D5946CDF80CC016
:100370008DF85E9006F0CFF93846594606F0CBF975
:100380005946764806F0C7F9754A5846536843F00F
:10039000007353600CF0A0FA724A179B4946B3FBF6
:1003A000F2F3714A71481360182215F028FAD8F850
:1003B00000304FF47A72B3FBF2F36D4A013B5360A5
:1003C000F0238AF823300723C2F808901360AB6843
:1003D000DFF8DC91DFF8DC81C9F8003098E80F0025
:1003E0008BE80F00A3694FF0100A43F00803A361E4
:1003F000A369179843F00803A36108233B6118A978
:10040000C7F810A006F087F919981AA906F083F921
:10041000D9F80020100713D5564B93F89021012AE4
:100420000ED8554993F89121896811F0805300F056
:10043000E68505E04F4B002283F891210AF0B0F9E0
:1004400064200AF00EFFA0224C48002115F0D7F9D5
:10045000E369002243F00703E361A36943F4006307
:1004600043F00C03A361444B4FF0000803F10C016F
:1004700002F8018001320E2AF5D1FF229A76DA764F
:100480001A775A773E4B3F4A41461A603E483C2213
:10049000D9F8004015F0B3F94146C4F3801705239D
:1004A0003A4ADFF8E4E0885C0C224A4302F80E0086
:1004B00047B91E3801289FBFFF2003F1FF3302F820
:1004C0000E00DBB201310529EAD1314A95F805A0C9
:1004D0001370304B304983F800A0304B264A33620A
:1004E000C0330B602E4BA10603EBCA035B7848BFF9
:1004F00001235362002340F2DC512A4A22F81310F0
:100500000133082BF7D110A800211C2215F077F930
:1005100014F4007CDFF8A09004F400684ED0A3042B
:100520000AD4B8F1000F0AD095F8842109F10C0320
:10053000012A08BF4B4604E0CDF8109002E009F113
:100540000C030493CDF858B03AE000BF001BB7008D
:10055000253000200005FA05000C01400010014084
:100560000000014040420F0068160020D015002016
:1005700010E000E0FC270020C00000202818002028
:1005800028160020EA2900202C16002062AD010860
:10059000100F002060170020C81800200C28002031
:1005A000A49E0108C20E002000ED00E000080140FA
:1005B000901B00203871010810710108CDF810C09F
:1005C000BAF10E0F04D00AF0EF0ABAF1080F02D107
:1005D00001238DF852300120CDF814C009F068F8DD
:1005E000DDF814C018B14088003018BF0120C4F3F2
:1005F00040038DF84630C4F3403300F001008DF81D
:100600004030C4F3C0338DF845008DF849708DF843
:100610004330B8F1000F07D095F8848108F1FF3717
:10062000D7F1000848EB0708C4F300438DF84A30BF
:100630001CF1000318BF01238DF84B30736A04F0DE
:100640000101003318BF01238DF84C30C4F300536F
:100650008DF84D30B5F84631C4F3C002ADF85030D6
:10066000B5F85231B5F84471ADF84E30C4F380435B
:100670008DF8473095F85431ADF85670181C18BFF6
:100680000120E40448BFAF4C8DF8480048BFB4F8DF
:100690004C41B5F8500148BFADF85640B0F5FA7F6F
:1006A0008DF844808DF841108DF84220ADF854004B
:1006B00002D90BB9ADF8563095F8D431A24886F876
:1006C0002830002386F8293043709DF85230002BE3
:1006D0000CBF0023022301B902B1013309EB8309E6
:1006E000D9F838309A1E1A330793002306920593DF
:1006F000069B33F8024F06934FF6FF739C4200F0BF
:100700009F819DF84520E3B2240AE5B21AB19A1EF2
:10071000012A40F290819DF8492032B18B491A019B
:1007200089588B4A914200F086819DF84A0030B189
:1007300086491A018958864A914200F07C819DF8C9
:10074000462052B18149039E01EB03114A68B2422F
:1007500003D10A89102A00F06E819DF8432052B11E
:100760007A49039E01EB03114A68B24203D10A8918
:10077000022A00F060819DF8442052B17349754E01
:1007800001EB03114A68B24203D10A89022A00F040
:100790005281169E7EB16D4F326807EB0317796860
:1007A000914208D13A89B188914200F04481F188A0
:1007B000914200F04081022C02D19DF8402003E0DC
:1007C000012C04D19DF84120002A00F034819DF8CD
:1007D0004C205E4C1E015AB19DF8522042B9A3F143
:1007E0000802012A04D8A2595B498A4208BF04259D
:1007F0009DF84D20344452B19DF852203AB910B1C1
:100800000C3B012B01E0043B032B40F2FC80012D4B
:1008100048D1524FDFF834A1FF2387F8703087F8B2
:1008200071300AEB06035A7B586803F108091B89EB
:100830004FF00008ADF85C3017A9022387F87480E8
:10084000C7F880408DF85F308DF85E2087F82C80E7
:10085000C7F83080C7F83480C7F83880C7F86C8094
:1008600087F8728087F8738005F055FF5AF8060004
:1008700099F80210424605F0ECFD204641462A4612
:100880000DF042FB364BC7F88C80C7F88430354BEF
:100890002046C7F8883007F1840107F188020DF07F
:1008A0007BFBC8E0022D63D19DF814204FF01C0C97
:1008B0000CFB02FC294B002703EB0C0808939DF866
:1008C00014304FF0010988F87530204B88F87670A5
:1008D0009A19517B506802F1080A12898DF85E104E
:1008E00088F87E7017A988F87490C8F88040CDF811
:1008F00024C0ADF85C208DF85F5005F00CFF134B61
:100900009AF8021098593A4605F0A3FD2046394658
:100910004A460DF0F9FA1449089BDDF824C0C8F8DE
:10092000841012496344C8F8881003F18401C8F8A0
:100930008C7020460A1D0DF02FFB059B4B44059340
:1009400079E000BFFC270020E9000020E4910108C5
:1009500000040040000C0140002C0140C0000020B9
:1009600085610008656200088D6400085D6100080B
:10097000032D46D19DF84730964D974ED3B19DF843
:100980004830964F95F82A8053B1954BBDF85420C6
:100990002046B3FBF2F2082192B2BDF8563003E0D4
:1009A00020464FF6FF72082105F0A8FF46F8280000
:1009B000C76020E0BDF8542095F82A70B2F5FA7FA0
:1009C000BDF856300BD986492046B1FBF2F208211A
:1009D00092B205F093FF834B46F827000AE0824964
:1009E0002046B1FBF2F2012192B205F087FF7B4B6A
:1009F00046F82700C36095F82A30013385F82A307D
:100A000019E0042D17D1BDF84E20774B714D93FBA3
:100A1000F2F22046BDF85030012192B295F82960DB
:100A200005F06CFF95F8293005EB86060133C6F812
:100A3000540185F82930069B079A93427FF458AEFB
:100A4000644F6A4E97F82930002487F87431684B58
:100A500034701D78A5F11703022B18D83B6A0021CA
:100A6000185903EB040811F097FF10B17B6A5BBBC8
:100A700025E0604B04EB030E98E80F008EE80F00B2
:100A8000337810340133C02C3370E7D1EEE75A4B82
:100A900013F835C003EBC503D3F8048086F800C013
:100AA000B8F1000FE2D06445E0DA524A230103EBCB
:100AB000020E43440FCB01348EE80F00F3E74F4F93
:100AC0003B68DB0424D41DE04D4B4E4A13F835003F
:100AD00003EBC5035C681070002CF0D00023834248
:100AE000EDDAC3EBC3016218D2F800C0DFF83CE1D5
:100AF000013341F80EC001EB0E079188B98092795D
:100B0000BA71ECE705F0EF03082B3F4B24D125E049
:100B10003378012BF6D93D4C04EB031303F1100697
:100B20001034B442EED054F8100C4FF07C5111F058
:100B30009FFD4FF07C5144F8100C54F8140C11F048
:100B400097FD4FF07C5144F8140C54F80C0C11F044
:100B50008FFD44F80C0CE3E70E2D08D11A78182D00
:100B600042F010021A7008D10BF0E6F805E01A788E
:100B7000192D22F010021A70F5E70BF0C1F83B684E
:100B8000234D5E035EBF234B01221A70224A234E7F
:100B90001378234843F0040313702B784FF48052EA
:100BA000022B34BF142310238DF85E304FF0020364
:100BB0008DF85F30B369ADF85C2043F00403B36196
:100BC00034BF0024012417A905F0A5FD154B7CB303
:100BD000154A2EE0C0000020F817002075620008BA
:100BE00000127A008562000840420F007C16002047
:100BF0006017002094160020A49E0108901B00207E
:100C0000A87B0108F2170020642400209C16002015
:100C100025300020C80B0020FC2F002000100240CF
:100C2000000801400C30002091B10008821700201C
:100C3000BE4A00201A600AF035FBBD4BBD4C93E85C
:100C40000300B3698BE8030043F00803B36117980E
:100C500018A905F060FDF3694FF0030943F48043E0
:100C6000F3613369204643F48043336118238DF8E0
:100C70005E3059464FF42043ADF85C304FF0040A23
:100C80008DF85F9005F047FD4FF4804320465946AC
:100C90004FF48058ADF85C308DF85EA005F03BFD58
:100CA0001023204659468DF85E30ADF85C8005F083
:100CB00032FD3369322043F480433361336923F4D6
:100CC000804333619C4B1A8802F4415242F44572CE
:100CD00042EA09021A80998B072221F40061090473
:100CE000090C99831A821A8892B242F040021A8043
:100CF0009F23C4F810808DF83C3000238DF83D30E0
:100D00008DF83E308DF83F300AF0ABFA5246C4F809
:100D1000148058460FA910F0EBFDC4F810809DF820
:100D20005E309DF85D201B0243EA02439DF85F2080
:100D30001343824A934214D032200AF092FAC4F844
:100D40001480F52010F00AFEFF2010F007FE702836
:100D5000C4F8108005D12B78022B04BF784B83F8A0
:100D600000902B78032B0CBF1F20022008F024FCDE
:100D70002B78032B03D0012006F073F907E0022043
:100D800008F096FC0028F6D04388002BF3D095F8A5
:100D900000906C4D4FF0100B284600215A463C68DD
:100DA00014F02DFD4FF6FF73ADF83C30022304F430
:100DB000004804F400674FF0000A1C408DF83E30F4
:100DC0008DF83FA00DD060480FA9ADF83CB00BF0F6
:100DD0002FFF04232B700124072385F801A0AC709A
:100DE000EB70B8F1000F0ED0022357480FA9ADF8F1
:100DF0003C300BF01DFF0123E2182B71AB71072370
:100E00006C71EB71D4B2B9F1010F0FD920234E48A8
:100E10000FA9ADF83C300BF00BFF052301222B721C
:100E2000AA72631C07226C72EA72DCB27FB10223E1
:100E300040480FA9ADF83C300BF0FAFE092301221F
:100E40002B73AA73631C07226C73EA73DCB273689A
:100E50003E4843F44043736073693C4F43F00103E1
:100E60007361B36943F40073B3610BF0BDFC17A861
:100E70000AF062F9364B00261793364B012C189373
:100E800094BF334680231C934FF480731D934FF41B
:100E900080631E93202317A91F9338464FF40053F5
:100EA0001A94209319961B9621960AF052F93B68E2
:100EB000294A43F001033B605368012C23F470235B
:100EC00094BF0021012123F4807343EA012353607E
:100ED0009168224B013C0B40314643F4602343F0C0
:100EE00002039360D36AE4B223F4700343EA045428
:100EF000D46201236A18907800286BD06C5C581C6F
:100F0000092CC0B2D278144F2AD9A4F10A06D7F816
:100F10000CC006EB46064FF0070E0EFA06FE2CEA52
:100F20000E0EB2404EEA0202FA6026E0A5B10008B9
:100F300058710108000C01400038004015202000C5
:100F400025300020E41A002000080140080002407B
:100F50004C240140F41A002000240140FDF7F1FF69
:100F60003E6904EB440C4FF0070E0EFA0CFE26EA25
:100F70000E0602FA0CF232433A61062B3A4E0CD8B6
:100F80005A1E776B02EB82021F23934027EA030766
:100F900004FA02F33B4373631BE00C2B0CD8DA1FFB
:100FA000376B02EB82021F23934027EA030704FA00
:100FB00002F33B4333630CE0A3F10D02F76A02EB4B
:100FC00082021F23934027EA030704FA02F33B43FC
:100FD000F3620346043110298CD1234B9A6842F402
:100FE00080729A609A6842F001029A609A6842F0B0
:100FF00008029A6099681C4A0D0739D5FAE7013A48
:10100000092A3FF61DAAD8F82C0004935946C7F8C0
:1010100014A0CBF80000039805F07DFB039B3C2057
:101020001A46082313610AF01CF9049BC7F810A0A4
:101030001F4695F891319F42BFF6FCA9039BDFF84C
:101040002CA04FF00808CAF810807820C3F814804C
:101050000AF0FCF8039BCAF814807820C3F81080CB
:101060000AF0F4F80137E4E700240140000C0140E5
:10107000936843F004039360A84B9A6812F004024B
:101080000392F9D19A6842F4A0029A60A44BB3F893
:101090005801002840F03686B3F95A21002A40F062
:1010A0003186B3F95C31002B40F02C869D4D2B68C6
:1010B0009C0320D5C8200AF0D4F8AE2005F051FFDB
:1010C00008B105F053FF984C84F87501C8200AF068
:1010D000C8F8964B0021C4F87831954C0C22204674
:1010E00014F08DFB0223E3700EF06DFF0AF092F80E
:1010F000904B0344A360904E894C336894F85F0191
:1011000094F8691194F86A21B3F9623009F052FB3E
:10111000059610B901200AF027F9884A0A261378A3
:1011200043F002031370864B10225A6108221A61A1
:10113000834F1920FB68013E83F01003FB60FB68BE
:1011400083F00803FB600AF08CF801200AF0AAF88B
:1011500019200AF086F800200AF0A4F816F0FF061D
:10116000E6D108233B611026764B3E611B681807C9
:1011700007D5754B7E611B689847744B01223E6111
:101180001A70734B00271E68DFF8FC81307B11F06A
:101190001BFA704911F06CFA09F016F86E4B1860E2
:1011A0006E4B188811F010FA01464FF07E5011F086
:1011B00013FB6B4B674918606A4B186911F058FABA
:1011C000694B1860307811F0FFF901464FF07E50FE
:1011D00011F002FB654B014618604FF07E5011F094
:1011E0003DF9634B4FF07E521860624B38469A606F
:1011F0001F605F60604B9A601F605F6008F0E4FFF3
:101200000646384608F06EFF31460746304611F074
:101210002FFA39468246384611F02AFA314681467D
:10122000504611F025FA39468346484611F020FA17
:101230000146584611F014F93146C8F80000384606
:1012400011F016FA3146069011F012FA069B834609
:101250003946184611F00CFA0346584619460693CB
:1012600011F0FCF8069BC8F804001946584611F026
:10127000F7F83946C8F80800504611F0F9F9314638
:101280000746484611F0F4F90146384611F0E6F8F1
:101290003A4F3B4B0026C8F80C00FF2138461B2272
:1012A0001E7014F0ACFA38463E70264E354B32684C
:1012B000012112F0020F18BF797019701FBF0321AE
:1012C00019700221B970510741BF19784F1C1F7066
:1012D000032748BF475412F00A0F0CD01A78042194
:1012E0008154511CC9B205274754D11C02321970D0
:1012F000D2B2062181542F6894F805E0BA0641BFA6
:101300001A78511C1970072148BF8154BEF1080F8B
:101310003CD0BEF10E0F3ED138E000BF00240140AA
:10132000FC270020901B0020C00000208429002002
:10133000E00D0020404B4C00D40E0020FC2F00207C
:10134000000C01400816002018160020D0050020CF
:101350006824002035FA8E3C602400200C00002018
:1013600018240020541500201C2400207C24002078
:101370006C2400208024002070240020950E002082
:10138000D6230020940E0020502400201A78511CEF
:1013900019700B2181541A7817F4803F4FF00C0C10
:1013A00000F802C002F101011CBFDFF8D4C2023212
:1013B000C9B219701FBF8CF80020B04A4FF00E0C54
:1013C00002F801C07A0748BF1A784FF0120841BFEF
:1013D000511C197010218154A94A17F4806F11789B
:1013E00001F1010C5FFA8CFC82F800C000F801806A
:1013F0000BD094F81882B8F1000F06D002311170AA
:101400009E494FF0130801F80C80B90541BF1178CF
:1014100001F1010C82F800C04FF0150C48BF00F834
:1014200001C0BEF1180F14D111784FF0160C00F85E
:1014300001C001F1010C5FFA8CFC4FF0170800F8B5
:101440000C8001F1030C0231C9B282F800C000F82F
:1014500001E0390341BF117801F1010E82F800E08B
:101460004FF0190E48BF00F801E0F90541BF1178AF
:101470004F1C17701A2248BF42541A78511C197019
:1014800014238354002198227E4814F0B8F910F0F8
:10149000FBFA7D497D4BB4F84E2119607C4B7D48A9
:1014A0001A807D4A0023138093700160059A7B495E
:1014B000D2F800E00B70B4F896110EF185021FFA15
:1014C00081F8774FDFF81CC23868DFF81C9200F50E
:1014D000967049F823002CF813800133122B6046D4
:1014E000EFD1D5F800C00EF1D50E1CF4805F08BF17
:1014F000B4F89C81A0F806801378F3B992F80280C2
:10150000D378984519D2B8F1000F08D008F1FF3808
:1015100008EB880808EB880808F5617306E00133DA
:1015200003EB830303EB830303F5617392F80180FC
:101530009BB208F1040820F8183004327245DBD160
:101540001CF0080F00F0008194F89031062B00F297
:10155000F580DFE803F004070E355172720045F2A2
:10156000F05201E042F6F8224E4B1A8010F018FBC0
:10157000E3E042F6F8224B4B09011A800A2391FB63
:10158000F3F10023A1F5B061474A42F8231001337B
:10159000122BF9D1454A464940201160454A137043
:1015A00008F060F9002800F0C98001234FF0070916
:1015B00090F9000040218DE808023F4A3F4BB7E018
:1015C00042F6F822374B40201A803D4A374B1A60CA
:1015D000384B10221A7008F045F9002800F0AE8050
:1015E00001234FF0000890F9000040218DE8080128
:1015F000344A4FF4E1339BE042F6F822294B402075
:101600001A80314A294B1A602A4B08221A7008F0B6
:1016100029F9002800F0928001234FF0000C90F986
:10162000000040218DE80810284A4FF4E13307F00C
:10163000EFFF274BC3F87C017CE042F6F821194A02
:10164000062B11801B494FF00C02DFF8A0C0DFF819
:10165000A0E0204C20480A704CD0002323708CF866
:1016600000308EF800301B2303701C4B4FF4E13424
:101670001A701B4B05221A7049E000BF950E00201E
:10168000940E00206427002084290020D00D002023
:10169000D40D00208C1B0020A01B00200B0D00206F
:1016A0009C1B00203A070020941900203C000020D9
:1016B0001DC50008E42F002099C70008A08601007E
:1016C00009C50008EDC60008F1C40008A1C600085D
:1016D000C0000020201A0020221A0020211900201A
:1016E000231A00203E270020540D0020221900203C
:1016F000211A0020002121708CF800108EF80010B3
:1017000021210170B649B74C0A70B74A1370B74A25
:10171000B74B40201A6008F0A5F878B101234FF0CC
:10172000000E90F900008DE808402346B14A4021A0
:1017300007F06EFF003018BF012028B9082008F01C
:101740006DFDAD4AAA4B1A602B68AC4A13F4804F6A
:101750001FBF12211170AA48A54918BF086042F2A4
:101760000101194099B144F62060A6490880990406
:1017700041BF08211170A4489D4948BF0860DC079B
:1017800041BF0C211170A148994948BF08601178E8
:101790009805A1F10401517052D59D4A9D4C049BBE
:1017A0004FF01008236093699B4843F00103936155
:1017B000049B0EA91B888DF83A80ADF838300223BF
:1017C0008DF83B3004F0A7FF236893485B880EA98F
:1017D000ADF8383004238DF83A3004F09CFF2368CC
:1017E0000120197A04F082FF23688C4A5B684FF06D
:1017F0000009536117A88DF861804FF00108179315
:101800008DF860908DF862800BF0D4F923680FA8F2
:101810005B7A8DF83E908DF83C3003238DF83D3097
:101820008DF83F8010F046F83B687D4A3C3B1360E2
:1018300033684FF0FF3243F010033360794B1A6086
:10184000794B7A4A7A4C13607A4A803313602B685A
:101850000026D903267040F1B08040F22A38DFF824
:10186000FC91DFF8ACA10CF01DF801274246484678
:101870003146277013F0C3FFDAF818306E4843F092
:101880000403CAF818304023ADF8383018238DF817
:101890003B300EA903238DF83A300BF0C9F9DAF882
:1018A0001C30664A43F00203CAF81C30644B654C96
:1018B0001B68AAF6947AB3FBF2F32288013B22F468
:1018C0005C721204120C22809BB21D22A285238519
:1018D000A782238C23F001031B041B0C2384238C7D
:1018E000A188228B23F0020322F0730212041B044E
:1018F000120C1B0C89B242F060023B43A180228390
:10190000A6862384238B23F008031B041B0C43F0BF
:1019100008032383B4F844306FEA43436FEA534328
:101920009BB2A4F84430DAF8A83F3B43CAF8A83F7A
:1019300050460AF059FF17A809F0FEFB424BCDF8BC
:101940006090179380231C934FF480734FF010091D
:101950001D9350464FF4005317A92093CDF864907F
:10196000CDF868801B961E961F96219609F0F1FB14
:10197000A3890FA89BB243F40073A381DAF8003067
:1019800043F00203CAF800308DF83C908DF83D70AA
:101990008DF83E608DF83F700FF08CFF2B4B039954
:1019A0001A682B4B43F821200B460133202B03935D
:1019B000F4D104F0BDFD04F0BBFD2B685A0540F1E5
:1019C0008680244C244BD4F8AC6404201E6007F0BD
:1019D00049FF0421C4F8B00407F020FF40E000BF35
:1019E0002119002090D00300231A002019C40008F8
:1019F0003C00002081C500087DC50008E42F0020C0
:101A00004DC500083A0700206DC500085DC50008F7
:101A10000010024008070020000C014000040140B3
:101A200004070020000F0020242A0020EC140020CE
:101A3000530C0020E81400200008014000366E011D
:101A40004C00002000040040340400406071010894
:101A5000540C0020C0000020D40B002040020020C5
:101A60008C4B84F8B40408201E6007F0FBFE8A4B00
:101A70000821186007F0D2FE884D2C22002184F83E
:101A8000B504284613F0BBFE7C232B708E236B70AD
:101A9000E023EB7010207D2385F82B30C4F8B86468
:101AA00007F0E0FE1021C4F8BC0407F0B7FE84F88C
:101AB000C0042020C4F8C46407F0D4FE2021C4F878
:101AC000C80407F0ABFE84F8CC040EF053F9744B55
:101AD000744C1B78022B65D1734A00251388322081
:101AE00023F040031B041B0C138013884FF4805613
:101AF00023F038031B041B0C138013889BB243F0A4
:101B0000400313809F238DF83C308DF83D508DF8B5
:101B10003E508DF83F5009F0A4FB8DF85D50634DA9
:101B200004226E6117A80FA90FF0E2FE2E619DF846
:101B30005E309DF85D201B0243EA02429DF85F3053
:101B400013435B4A934219D00AD8A2F51A42033ACA
:101B500093420CD002F51A420232934209D01CE0A3
:101B6000544A934205D00132934207D015E0202316
:101B700000E0802323804FF4807302E04FF48073F1
:101B800023806380A38822881B02A3605343E36001
:101B9000494B012283F8CD2404E000232380638095
:101BA000A360E360E4680CB3E40A26460027A7427A
:101BB0000ADA3D196D100DF15C08E8024146102269
:101BC00005F006F80F2806DC0CF0AEF83A4BF602EA
:101BD000C3F8D0640AE0002358F82320013255D11D
:101BE0000133042BF8D12E462C46E0E7334C344A1F
:101BF000236813F4002318BF0123137009F00AFBB4
:101C0000304B1860304B5A791946052A02BF2F4BCA
:101C10004FF4C8721A802E4B4FF47A721A802D4BF3
:101C2000C8221A802C4A137843F0080313702B4AF9
:101C3000137823F00203137040F602032268134066
:101C40006BB12748274B1860274B03201870274B90
:101C50000120187026480023038026480380930340
:101C600041BF254B03221A71DA7844BF42F00102CA
:101C7000DA708B6801222360204B1A70204A137897
:101C800063F07F03137023B0BDE8F08F6F1C25460F
:101C9000AAE700BF100C00202C0C0020E00B002055
:101CA000253000201000002000380040000C0140CA
:101CB00018BA20001740EF00C0000020901B002041
:101CC000702500200C070020FC270020EA230020BC
:101CD0001E3000201C300020642400202130002011
:101CE00076290020DC1A002058250020480000201A
:101CF000480E00204A0E0020E00D0020C80B0020F6
:101D0000FC2F0020424B00221A7000B210F05CFC45
:101D1000404910F0ADFC404C0646B4F95A0110F0B1
:101D200053FC3C4910F0A4FC0546B4F95C0110F0EA
:101D30004BFC384910F09CFC0446304608F044FA4D
:101D40008046304608F0CEF90646284608F03CFAB0
:101D50000746284608F0C6F90546204608F034FA3A
:101D60008246204608F0BEF941468146504610F0B2
:101D70007FFC41468346484610F07AFC5146059068
:101D8000304610F075FC49460690304610F070FC65
:101D900039460790504610F06BFC204C49462060B5
:101DA00007F1004010F064FC29466060A5600698C9
:101DB00010F05EFC0146059810F052FB2946E060E9
:101DC000079810F055FC0146584610F047FB39467D
:101DD000206106F1004010F04BFC29466061584636
:101DE00010F046FC0146079810F038FB2946A06128
:101DF000059810F03DFC0146069810F031FB414675
:101E0000E061384610F034FC2062FFF74FB900BFA4
:101E10003400002035FA8E3CFC270020B81A002040
:101E2000A0492DE9F04F0A689F4C02F59C432033EE
:101E300023609E4B89B01E780191C6B19C49096808
:101E40008A4240F20381013E1E70FFE0D9F8003063
:101E5000072D98BF595D974B88BF29461B68964848
:101E60009847032D0CD904EB4505A8800136924B09
:101E7000F5B21A78DFF86492AA421946E6D820E053
:101E8000D9F8002005F10E0302EB83039988DA8864
:101E90000028E8D04FF47A73401A5843531A90FB45
:101EA000F3F040F6C90300F57A70984205DC40F281
:101EB000EE239842B8BF184601E040F6CA0080B24F
:101EC000D1E742F201087D4B1B6803EA0808B8FA23
:101ED00088F87B4B4FEA58181B68B8F1000F06D101
:101EE00094F8292084F82820764A5078107094F8C5
:101EF00028701FB1734A177887F0010794F82BB048
:101F00000326BBFBF6F60F2206EB460684F82A20D2
:101F1000C6EB0B06D9F8002091F800A0DFF8C491B9
:101F2000F6B20025554559DA4FEA450C1FB166490E
:101F300031F8150000E03846918ADFF8ACE18142C3
:101F400002D8D18A81421ED25EF8250056498342CA
:101F500003D25E4931F80C0019E0E8B20392029313
:101F600004910AF0E9FF032D029B039A0FDC049908
:101F70004FF0010C91F82AE00CFA05FC2EEA0C0E49
:101F800081F82AE003E003F596714EF82510B8F1C8
:101F9000000F1CD194F8BC1029F8160031B9BBF120
:101FA000020F14D94049012081F8BC00B9F8021091
:101FB000B9F800000844B9F804100844444980B254
:101FC00021F8150000B2032190FBF1F080B23F49E7
:101FD00009F1060921F815000135A3E794F82A2034
:101FE0003749A2F10F077A427A4184F8D620394B5B
:101FF0006AB1394A1268560109D40A68D9689A60E8
:10200000521AC82A1DD9012283F8212019E02D4A2D
:102010000120507010700A689968DA605B68521A83
:102020009A4282BF2B4B002283F821200025554580
:1020300007DAE8B20AF080FF244B23F815000135D7
:10204000F5E794F82B30013384F82B301B4E3368BE
:10205000DD0405D5204B1B68D80701D40FF0F6FB33
:10206000019B1F681D4BD3F800E09EF80A00002872
:102070003CD0164A9EF80C30013832F810001BB1E3
:10208000C0F53B60083080B200B2A0F57A70B0F5C0
:102090007A7FA8BF4FF47A7020EAE07010F094FACB
:1020A0000F4959E008300020E00C0020981B002068
:1020B000941B00203C000020E42F0020901B0020F7
:1020C0009C1B002008000020E40C00203E2700207C
:1020D0009E0D0020A01B0020900E00208C1B0020D5
:1020E00000007A440C0D0020540D002033681904C0
:1020F0003BD5D4F8D830934DFB1A002B35DB07F5D0
:102100009C432033C5F8D8308F4B5A798F4B33F826
:1021100012108AB29EF80B1092FBF1F195F8DC20B8
:10212000013202F00F0385F8DC302B4483F8DD1018
:102130000346874A825C0130134410289BB2F8D1D1
:102140001BB293FBF0F000B26428A8BF642020EA21
:10215000E07010F039FA7F4910F03EFB7E4910F034
:1021600087FA10F071FC7D4B188033687C4D13F4B6
:10217000807F00F00E817B4BDFF8EC919F4205D908
:1021800099F8022012B9012289F8022099F8022058
:10219000002A00F0FE80744A95F8008092F82170C1
:1021A000C8F380087A1E57425741704A002F924662
:1021B000116818BF4FF0000BC1F38063019308BF93
:1021C0004FF0030B99F82020052A00F2DC80DFE8AD
:1021D00002F0034E537988A5B8F1000F3AD0D4F835
:1021E000F000B4F8F41007F0DAFB012809D16049D7
:1021F000604A09681268C988642000FB0122C9F896
:102200001020019B6BB15A4A126812794AB10FF043
:10221000E1FE032289F820204FF47A72C9F81C20CD
:10222000D0E7002F40F0AF80524AD9F81010106864
:102230004D4A88420AD902920FF0CCFE029A03213D
:1022400082F8201040F6B831D161BBE7012182F855
:102250002010B7E7019B4FF4806013B107F0CEFF69
:1022600001E007F0BBFF0022C9F810208BE0002F2F
:1022700049D10FF0AFFEA5E727B1052289F820204C
:10228000012000E03846B8F1000F0CD0D4F8F0205F
:102290004FF0020BD189384A118051809180344926
:1022A00009684988D180334A1168D9F814209142CD
:1022B00002D8B8F1000F63D147F23052C9F81C20A0
:1022C000032221E02A7842F002022A700FF0BEFABF
:1022D000284AD9F81C1012680A44C9F818200422A8
:1022E00012E0244A9FB11168D9F8182091424AD9C6
:1022F000224A92781AB9DAF80020D30743D42A7810
:1023000022F002022A70052289F820205AE712687A
:10231000D9F81C100A44C9F8182034E01449154AA9
:1023200009681268C988642000FB01224FF48060AC
:10233000C9F81020002289F8202089F8032007F02E
:102340004DFF3FE7E00C0020E41A0020F41A0020C3
:10235000BD0D00200000C84200C07F44040F0020D3
:1023600021300020404B4C00A01B0020900E00208C
:10237000F82F00209C1B00203E2700200800002092
:1023800000287FF41FAFBBF1000F02D0584608F0C1
:10239000A3FF904F07F5C470B7F84E1107F0FFFA8E
:1023A0000197834668B90FF007FE8B4B0022C3F8F4
:1023B00000B0C3F804B0C3F808B0884B1A605A6084
:1023C0009A602B785F0736D53368D80633D5844BAF
:1023D0001B78D9062FD4834B9B789BB1019B93F834
:1023E000E031BBF1000F15D17BB17F4B1A68D4F8F7
:1023F000F8309B1A002B08DA0FF028FA7B4B83F891
:10240000FCB018E0BBF1000F0DD1102008F064FF04
:1024100001230EE03BB1744A4FF47A71126801FB5C
:102420000323C4F8F83094F8FC3023B108F040FFDF
:10243000002384F8FC30019B002293F8DEA193F87E
:10244000DF11B3F898E1B3F89AC1134668489B08C6
:1024500030F9127001327745C4BF63F07F03DBB2FD
:102460006745B8BF43F04003042A8146EED194F893
:10247000FD205E489A4205D190F8FE20F92A04D842
:10248000013200E0002280F8FE2084F8FD30554B38
:10249000584F9A789846E2B93B68DA0708D5BBF1FD
:1024A000000F16D12B78DB0713D50FF031F810E0B1
:1024B0002B7858070DD54D4B93F828304BB14E4B28
:1024C000DB7833B911B10FF0C1F902E0BBF1000FB5
:1024D000F9D094F8FE30454A142BDFF838B140F0BB
:1024E000AB8098F802301AF1000A18BF4FF0010AC9
:1024F0006BB392F8FD305F2B11D12B7803F00403FE
:1025000003F0FF0113B10FF0A1F908E00B200391D4
:10251000029208F0E1FE029A039982F8FE10BAF1E5
:10252000000F14D094F8FD307D2B10D12B7803F0E0
:10253000040303F0FF0213B10FF088F907E00B204A
:10254000029208F0C9FE294B029A83F8FE202B78EC
:1025500003F0040303F0FF01002B6DD194F8FD306C
:10256000224A572B10D1254B4FF47A721A80244BF4
:102570001B685A0742BF234A0A21118013F008033F
:102580005AD1214A138057E03068400716D55A2B9C
:1025900014D11E4B187820B119701D4B01221A70EE
:1025A0004AE092F8FF3083F0010382F8FF300BB16C
:1025B0000C2000E00D2008F08FFE3DE05D2B00F0C8
:1025C00069845B2B00F068845E2B25D1032000F02A
:1025D00064BC00BFFC27002030230020E422002040
:1025E00064240020080000209C1B0020E00C002038
:1025F0003E270020900E0020A01B00201E3000204F
:10260000081600201C300020F40E002015240020A5
:1026100016240020D40E0020562B01D108F0C0F85B
:1026200098F80230002B00F04E8494F8FD306F2BA8
:1026300040F043840EF06CFF3368580732D594F8AD
:10264000FF30A3B12B78590711D5019BB9F90620AA
:10265000B3F898319A420ADD3B6813F0010301BFD9
:10266000AC4A32211180AC4A08BF82F8FF303B6887
:10267000DA030AD5A94B1A782AB9A94A127812B9ED
:10268000A44A3221118001220BE0A54A13784BB1F4
:102690002B7803F0040303F0FF011BB9A14B117069
:1026A00001221A70DBF8009000233B6009F18708D3
:1026B00009F1D70A98F8002098F8013018F8010CB1
:1026C0009A420BD2414607F035F938B118F8022C7E
:1026D000012303FA02F23B6813433B6008F104084C
:1026E000D045E7D1904B1B7853B1904FDFF854920F
:1026F0003B68DFF8548213F0020F40F0388330E378
:1027000009F1D60709F58F783A787B7817F8010C2C
:102710009A4225D2394607F00DF908B397F804C05C
:102720000C21BB7801FB0C41814A013B03EB4303C5
:102730001344D1F8102197F803909A4276480FD0AD
:10274000C1F81031002390F83C21C1F81431012365
:1027500003FA0CF322EA030381F80C9180F83C3170
:1027600006374745D0D1734BDFF8E0A1D3F800809E
:10277000714B4FF0000B1B68029394F828300393C1
:10278000DAF80020002A00F0E38292F80090B9F114
:10279000000F00F0DD82DAF804300299CB1A002B2A
:1027A0000CDB01F5FA73CAF8043094F83C110123EC
:1027B00003FA0BF321EA030384F83C31039B002B5B
:1027C00000F0C6821AF8043C51780433DBB20029C9
:1027D00040F07F82594931F91310594BB3F89631C3
:1027E00003F1C800814201DD977814E0C83B9942AB
:1027F00002DA91784F420EE094F83C21012303FA6B
:102800000BF322EA030384F83C31029B03F5FA73CD
:10281000CAF804309CE294F83C3143FA0BF3DB072E
:1028200000F19682002FCCBF0220012008F084FD29
:1028300009F1FF32384B132A00F28282DFE812F0EE
:10284000140023003200440061008800ED005201B2
:10285000B701EA0119028002440055008800ED002A
:102860005201BF002401890198F8001040460F442E
:10287000FA2FA8BFFA2727EAE77788F8007007F051
:102880003FF801201EE098F8011040460F44642FE5
:10289000A8BF642727EAE77788F8017007F030F8C7
:1028A00002200FE098F8031040460F44642FA8BFA1
:1028B000642727EAE77788F80370D3F8401106F019
:1028C000D7FF03203946D1E198F805100D2039448F
:1028D0006429A8BF642121EAE17188F8051008F095
:1028E00085FCB9F10D0F00F02B8298F804100E2032
:1028F00039446429A8BF642121EAE17188F80410F1
:10290000B4E198F806100520394481F3080188F8ED
:102910000610ABE1FC230020E00C00201424002072
:10292000152400201624002023300020900E0020C3
:10293000487401080C0F00209C1B00203E2700203B
:10294000FC270020081600208C0E0020F00D00202F
:10295000D3F844311A78022A22D1384604930FF072
:1029600033FEA9490FF038FF049B596A05930FF015
:1029700077FD0021049010F019F8059B48B9049ADE
:10298000A149104610F030F8049A059B10B19E4AF8
:1029900000E000225A620F20114607F01BF80AE0FF
:1029A00099780F203944C829A8BFC82121EAE171CC
:1029B000997008F01BFCB9F10F0F00F0C181934B27
:1029C000D3F8449199F80030022B1AD138460FF011
:1029D000FBFD8D490FF000FFD9F820100FF040FDEE
:1029E000002107460FF0E2FF30B9384686490FF064
:1029F000FBFF10B1844F00E00027C9F820701220BF
:102A000057E199F8011012203944C829A8BFC821FC
:102A100021EAE17189F8011028E1D3F844311A78EC
:102A2000022A22D1384604930FF0CEFD76490FF0EA
:102A3000D3FE049B196B05930FF012FD0021049047
:102A40000FF0B4FF059B48B9049A6F4910460FF088
:102A5000CBFF049A059B10B16B4A00E000221A6379
:102A60001020114606F0B6FF0AE0197B1020394409
:102A7000C829A8BFC82121EAE171197308F0B6FB83
:102A8000B9F1100F00F05C81604BD3F8449199F8D4
:102A90000030022B1AD138460FF096FD5A490FF03C
:102AA0009BFED9F82C100FF0DBFC002107460FF03D
:102AB0007DFF30B9384654490FF096FF10B1524FA0
:102AC00000E00027C9F82C701320F2E099F80B10F1
:102AD00013203944C829A8BFC82121EAE17189F827
:102AE0000B10C3E0D3F844311A78022A22D13846B9
:102AF00004930FF069FD46490FF06EFE049BD96BFD
:102B000005930FF0ADFC002104900FF04FFF059BE3
:102B100048B9049A3C4910460FF066FF049A059B99
:102B200010B1394A00E00022DA631120114606F0A4
:102B300051FF0AE0997D11203944C829A8BFC82156
:102B400021EAE171997508F051FBB9F1110F00F01C
:102B5000F7802E4BD3F8449199F80030022B1AD10C
:102B600038460FF031FD2A490FF036FED9F83810FB
:102B70000FF076FC002107460FF018FF30B93846F9
:102B800021490FF031FF10B11F4F00E00027C9F8B5
:102B9000387014208DE099F8151014203944C82994
:102BA000A8BFC82121EAE17189F815105EE0D3F8C9
:102BB000449199F80030022B1AD138460FF004FDE9
:102BC00011490FF009FED9F828100FF049FC002137
:102BD00007460FF0EBFE30B938460B490FF004FF03
:102BE00010B1094F00E00027C9F82870092060E003
:102BF00099F8031009203944C829A8BFC82121EA3F
:102C0000E17189F8031031E00000C842E00C0020B7
:102C100000007A44D3F8449199F80030022B1AD17D
:102C200038460FF0D1FCBA490FF0D6FDD9F8341070
:102C30000FF016FC002107460FF0B8FE30B93846F9
:102C4000B3490FF0D1FE10B1B14F00E00027C9F831
:102C500034700A202DE099F80D100A203944C82953
:102C6000A8BFC82121EAE17189F80D1008F0BEFA69
:102C700066E0D3F8449199F80030022B1DD1384614
:102C80000FF0A2FCA3490FF0A7FDD9F840100FF0F8
:102C9000E7FB002107460FF089FE30B938469C4912
:102CA0000FF0A2FE10B19A4F00E00027C9F8407063
:102CB0000B20394606F08EFE42E099F817100B20E3
:102CC0003944C829A8BFC82121EAE17189F8171041
:102CD000CCE7012934D190788F4A32F91370B7F5D7
:102CE000617F05DB40F633039F42A8BF1F4601E02A
:102CF0004FF46177B9F10C0F22D14FF4966393FB37
:102D0000F0F0A7F5617797FBF0F7844AFFB21378EC
:102D1000BB4215D0042F34BF3B4602231370019AE7
:102D200009FB03237E4A03F2B273136007F04EFBE4
:102D30004846394608F05AFA781CC0B208F0FCFA46
:102D400094F83C21012303FA0BF3134384F83C313C
:102D50000BF1010BBBF1040F0AF10C0A7FF410AD6B
:102D6000C3E43368D80511D56E4BDB7873B1D9F85D
:102D7000003099070AD5B8F8003013F0010A0AD1DB
:102D80000FF01AF9012007F039FA04E0012007F0EA
:102D900025FA012300E000233A6852070DD563B1FC
:102DA000012007F01BFAB8F80030980708D40FF09C
:102DB00003F9022007F022FA02E0022007F00EFADF
:102DC000B8F80030584A13F0030F4FF0100114BF49
:102DD00051611161D9F8002012F00A0F24D03A682D
:102DE000D10609D55A070AD4042007F007FA4F4B39
:102DF0001B88A4F8483102E0042007F0EFF93B6893
:102E00009B0607D5B8F80030580606D4402007F0D6
:102E1000F5F902E0402007F0E1F93B68590642BFAE
:102E2000424B1B88A4F84A313B684FF480701A0566
:102E300002D507F0E3F901E007F0D0F93C4B5A79ED
:102E40001C46082A01D00E2A02D1402007F0C6F9FC
:102E500033685B0540F1A58094F818321BB92B78D4
:102E600013F0040F02E03B6813F4002F0BD0314B3A
:102E700000221A703C2008F02DF9002800F0918003
:102E80000EF074F8F6E70CF075FF09B0BDE8F04FEE
:102E90000EF0FABD012000E002205FFA80F8019AEE
:102EA00008F1FF3382F8B03707F0EAF907F0B2FA19
:102EB000404608F041FAFFF7BFBBBAF1000F02D05D
:102EC0007E2B3FF4B7AB94F8FD301B4A972B05D10E
:102ED0001A4B4FF4C8721A80FFF7AEBBA72B06D16E
:102EE000174A137843F004031370FFF7A5BB0021C2
:102EF000BB2B079101D1022303E0B72B04D14FF67E
:102F0000FE73ADF81E3023E0BE2B1BD102231DE063
:102F10000000C84200007A443E27002030250020EF
:102F20000C0F0020A01B0020000C0140F40E00201C
:102F3000FC27002024160020E00C0020EA230020BB
:102F400064240020BD2B1AD14FF6FE73ADF81C305F
:102F5000DBF80030BDF81C10B3F864200A44A3F875
:102F60006420BDF81E10B3F866200A44A3F866205A
:102F700007F016FC002384F8FE30FFF75DBB792BC9
:102F800004D192F8033123F0010306E07A2B7FF499
:102F900053AB92F8033143F0010382F80331FFF79A
:102FA0004BBB09B0BDE8F08F704B2DE9F04FB3F982
:102FB00006106F4B91B01F6801937A8991420EDB26
:102FC000B1F5FA6FFC79BFBF8B1A6343A2F5FA64BF
:102FD00093FBF4F4ACBFC4F16404643400E06424F3
:102FE000644B654A1868B2F896A1054692F95E21CD
:102FF000049092B205920293002240F2E6305B4BBD
:103000004FEA420B33F912300393CAEB030303F286
:10301000F316864203D8002BB8BF5B4201E04FF4A1
:10302000FA73022A00934FF06400049B534E31D090
:1030300093F81DE1BEF1000F06D0009B7345CCBF95
:10304000CEEB030300230093009BDFF84CE193FBDE
:10305000F0FC6FF063093EF81C8009FB0C390CF1A1
:10306000010C3EF91CE00FFA88FCCCEB0E0E0EFBB7
:1030700009FE9EFBF0FEC64426F80BE0BE1836792A
:1030800073433F4E93FBF6F364339BB2634393FB6E
:10309000F0F030E093F81EE1BEF1000F06D0009B87
:1030A0007345CCBFCEEB030300230093009BDFF8F6
:1030B000E48093FBF0F06FF0630C38F910E00CFB48
:1030C0000039013038F91000059BCEEB000000FB01
:1030D00009F999FBFCF9CEEB090909FB03F9009BFF
:1030E000A6F80490B879002BB8BF5B42434324484C
:1030F00093FBF0F064306B784FF0640E434393FB26
:10310000FEF3204E022AB354EB7A1F4E00FB03F36A
:1031100093FBFEF3B3546B7D184E00FB03F090FB62
:10312000FEF01A4B98541A4B0FD183F802E0039B20
:1031300053450EDB104CB4F8982191422EDBB1F5CB
:10314000FA6FA8BF4FF4FA6129E09C54039B5345E2
:1031500004DA36F80B305B4226F80B300132032AD2
:1031600005F101057FF449AFE4E700BF3E270020E9
:103170000C0F0020D40E0020FC2700208A1600200F
:103180000CFEFFFFF02200203E0E00200423002052
:1031900020230020300E00201A1500201146891A25
:1031A0004FF47A735943C2F5FA62B1FBF2F1642726
:1031B00091FBF7F2DFF898E26FF063033EF812003C
:1031C00003FB021101323EF9122003B2D21A51431D
:1031D00091FBF7F30344F3808C4B8D4D1B885F0606
:1031E0003BD58C4A8C4B10881B88181A00B20FF004
:1031F000EBF98A490FF03CFA074606F0E5FF8046F6
:10320000384606F06FFF0746B5F902000FF0DCF90B
:103210008146B5F900000FF0D7F9414682460FF01C
:1032200027FA3946834648460FF022FA01465846A7
:103230000FF014F90FF0E2FB4146288048460FF0EA
:1032400017FA3946804650460FF012FA01464046BA
:103250000FF006F90FF0D2FB6880714F3B689D07B5
:103260006CD545F207216F4B6F4D1A686B69D31A05
:103270008B4263DD6A6109F047FE6C4BDFF8D49145
:103280001A789846032AB9F8003020D10A2B28D999
:103290000023282088F8003007F0E3FF09F034FE0F
:1032A000634B188809F01AFE624B1A68D37890FBBA
:1032B000F3F001300828604BA8BF0820187053793C
:1032C00080B243432B8313795843688309E00A2B68
:1032D00007D80323584A88F80030002313702B8343
:1032E0006B8398F80030514A012B0CD002D3022B8B
:1032F0001BD023E02A8BB9F800309A421EDD01234F
:1033000088F800300FE0B9F800106B8B8B4202DDBB
:10331000022313700FE0444B1B8B0133994202DDF3
:10332000002313700AE0082006E06B8BB9F8002038
:1033300001339A42E3DC072007F0CEFFD7F800B054
:103340003E4D1BF4006F00F0A080364B364F1B68DB
:10335000FA69C2EB030845F20722904540F39580D5
:10336000FB61344BB6F906C0D3F80090B4F84E11A7
:1033700099F80A30ACF57A7C012B314E03D06BD32F
:10338000022B20D06AE02F4B396A5A7B2E4B082043
:1033900033F8122091FBF0F392B2C91A8B183B62FA
:1033A00093FBF0F3BA8440F6E4429BB25343B9F87E
:1033B0000820C2EB13334FF47A725343B9F9062055
:1033C00093FBF2F349E02B78B9F808A05807C6F848
:1033D00000A043D51D48CDF800C006F0E0FADDF8A6
:1033E00000C020B91BF0100F18BF4FF0000C0CFBF1
:1033F0000CF3322293FBF2F3B9F9062063445A43EB
:103400004FF47A7392FBF3F3534426E08C0E0020C2
:103410008A1600202A0E0020F40E002035FA8E3C79
:10342000901B002008300020300E0020582500207E
:10343000FC1A0020DC1A0020480000202130002067
:10344000080F0020E41A0020F41A0020842900202C
:1034500002150020881B0020002333603368D7E961
:103460000A0103FB08F84FF47A7398FBF3F810EBAA
:10347000080241EBE873C7E90A2310461946944A4B
:1034800000230FF001FB934B1860934F3B680097AC
:1034900013F4805F02D00A2007F01EFF8F4E3268BF
:1034A000002A58D08E498F4B08681F68894687428A
:1034B000984650D88C4BDFF83CA21878516808BB6E
:1034C00001201870BAF80030CB5C5BB31378013B75
:1034D00000FA03F2D4F8DC371A4201D107F0E2FE19
:1034E000824B01221A7009F079FDBAF80030CBB98D
:1034F00033681B78053B012B14D807F08BFE7C4BFF
:1035000018600FE04FF0000B83F800B0BAF80030FD
:10351000CB5C3BB1584607F0C5FE744B83F800B056
:1035200009F05CFD3368BAF800205B6871499B5C68
:10353000FE2B02D100230B800DE0FF2B02D107F000
:10354000B7FE08E0D9F800000A2606FB03030132A3
:10355000C8F800300A802B78590703D5664B08223B
:103560005A6138E0009A1268D2075EBF634A43F09E
:1035700001031370624B5D4A1B781F075EBF2B78F7
:1035800023F001032B705F4B1B6813F0040F02D074
:103590005D49098851B95D49098809B19E0705D47B
:1035A0005B4B1B88003318BF012333B10223137018
:1035B0002B7823F001032B7004E02978C80758BF4B
:1035C0000223137007F026FE524B1B68C01A002816
:1035D00001DB09F003FD504F0CF0CCFB3E78002ED0
:1035E00000F0E1804D4B1A689846002A00F0E7860B
:1035F000D8F8000007F020FF002800F0E086474BD5
:10360000474C186807F015FF092801D03F2852D110
:103610004FF0000A55462668DFF8189136B1414848
:10362000D9F80010324612F037F910B9CA4605B978
:103630004D463D4B09F110099945EFD3EDB1D5F851
:1036400000C0DAF8009023681CF803E019F80300C2
:10365000704512D15A1C334958B92D2B09D8DFF8BF
:10366000C0E0CEF800204FF0200E01F803E08854AF
:1036700003E001F803E02260E5E723680BB155455C
:1036800010D02A480DF066FD554507D855F8100BA7
:103690000DF060FD09200DF055FDF5E724480DF013
:1036A00059FD002623689E42A2D21E4B985D0DF064
:1036B00049FD0136F6E72368002B40F066860428B2
:1036C00040F08886174804F0ABFD00F078BE00BFDC
:1036D000407E0500E01A0020900E002078160020A1
:1036E0009C1B0020701600206C160020C41B0020BC
:1036F0002827002074160020000C014021300020F3
:1037000064240020081600201C300020EA2300203A
:103710001E300020C81B002023300020542500202C
:10372000E4140020B4140020E87A0108A2940108EF
:10373000A794010818790108D9F80000DFF894A3CC
:1037400007F07AFE28B3DAF8000007F072FEDBF823
:103750000030024693F84810A9BB24286CD10122FE
:1037600083F84820DBF80030DFF89CA393F848206A
:10377000062AE1D193F8490001F00EFE83460028A5
:1037800000F083800DF03EFCD8F80030002283F872
:103790004820CE4B93F83530002B40F0E4854C3672
:1037A000982E00F00C86CA4BF21892F84A100129A4
:1037B000F5D1DFF85483F358C8F80020C54AC34652
:1037C00013609146B8E7012904D14D2814BF0022A7
:1037D0000222C5E7022904D13C2814BF002203229B
:1037E000BEE703290CD140284FF0000102D983F82D
:1037F0004810B7E758711971D97198710422AFE771
:10380000042906D1997983F849004A409A71052222
:10381000A6E70529A6D1587919798842987906D959
:1038200050409871481C18710B441A729AE79042E4
:103830000CBF0622002293E72B78A7495B0791D49F
:103840002328DAF8003013D1009001203870A34803
:10385000039103609D480363A1480DF07BFCA148E0
:103860000DF078FC0399009A0B7843F002030B707B
:103870009D4B1B681B78934201BF9C4A9C4B1A606E
:103880009C4A04BF9C4BDA606CE7DAF8002092F89F
:1038900049304A2B00F062855CD8332B00F05B8402
:1038A00021D8292B00F0F58309D8252B00F0CC83F3
:1038B000272B00F0D083232B40F0888552E22D2B5C
:1038C00000F0F88307D82B2B40F080850DF06EFBBD
:1038D000607100F043BD2F2B00F0AA84312B00F063
:1038E000C78400F073BD3E2B00F036811DD8372B06
:1038F00000F0658404D8352B00F06D8200F066BDC1
:10390000392B00F0B5833C2B40F06085DFF8EC915B
:10391000D9F800A00DF04AFB8AF80000D9F8003071
:1039200018780CF0E9F900F019BD432B00F024845D
:1039300006D8412B40F04A854FF0000900F010BC3A
:10394000442B00F0CA84482B40F040850AF03AFA34
:1039500000F004BDD02B00F055835FD8CA2B00F0D7
:10396000048116D84E2B00F0C883C82B00F0A2802B
:103970004C2B40F02B850DF019FB84F8D6010DF08F
:1039800015FB84F8D7010DF01BFBA4F8D80100F05B
:10399000E5BCCD2B00F0418304D8CC2B00F05A823B
:1039A00000F014BDCE2B00F04183CF2B40F00E85EC
:1039B0000DF006FB6FF4AF6E00EB0E039BB2C62B4F
:1039C00098BFA4F896010DF0FBFAA4F840010DF0A1
:1039D000F7FAA4F842010DF0F3FAA4F844010DF04F
:1039E000EFFAA4F8D8010DF0E1FA0DF0DFFA0DF0CE
:1039F000DDFA0DF0DBFA84F885010DF0D7FA84F8D2
:103A000092010DF0D3FA3D4BD3F800900DF0D8FAA7
:103A100000EB80004000A9F8620029E3D82B00F0F9
:103A200033810FD8D32B3FD003D8D22B29D000F02D
:103A3000CDBCD42B00F06D82D62B40F0C7844FF064
:103A400000095BE2F22B00F0B28212D8EF2B40F0BB
:103A5000BD84DFF8A890D9F800A00DF0B1FAAAF85B
:103A60006600D9F800900DF0ABFAA9F8640000F0F8
:103A700075BCF32B00F03684FA2B00F0E18200F0E5
:103A8000A5BC2B7803F0040303F0FF09002B40F0E2
:103A900065840DF08BFA022884F8B00740F2B882F2
:103AA000174B83F8B097B3E20DF08AFA154B1880E4
:103AB00000F054BC92F805904FEA5909B9F1120F81
:103AC00024D907F003FB00F049BC00BF300E0020F2
:103AD000642700205025002021300020542500209C
:103AE000D7940108A794010828160020EFBEADDE88
:103AF000F04F00200400FA0500ED00E0D40E002095
:103B0000FC270020280E00204C2500204FF0000A42
:103B1000CA4507D20DF054FA07AB23F81A000AF190
:103B2000010AF5E74A4600234B4507DA07A931F8B1
:103B30001300BD4921F813000133F5E7122A05D01F
:103B4000B94B002123F812100132F7E7B74B0122DD
:103B500083F8342000F002BC0DF028FA84F8E0016C
:103B60000DF024FA84F8DF01F8E3B14B81461A68BE
:103B70009A461278022A6CD1DFF8B4A209F1080B38
:103B8000DAF8003000930DF011FA0EF019FDA94992
:103B90000EF022FE009B43F82B00DAF800B00DF087
:103BA00005FA09F10A030BEB830B0EF009FDA2499C
:103BB0000EF012FEDAF80030CBF8040000930DF09E
:103BC000F5F90EF0FDFC9D490EF006FE09F10E0B15
:103BD000009B09F10109B9F1030F43F82B00CBD188
:103BE000B9F1070FDAF800B01AD10DF0DFF90EF0D5
:103BF000E7FC90490EF0F0FDCBF84400DAF800B095
:103C00000DF0D4F90EF0DCFC8A490EF0E5FDCBF89E
:103C10004800DAF800B00DF0C9F98BF84C0012E05A
:103C20000DF0C4F9CB448BF80100DAF800B00DF0C8
:103C3000BDF9CB448BF80B00DAF800B00DF0B6F903
:103C4000CB448BF8150009F10109B9F10A0FC7D16E
:103C500084E3DAF800B00DF0A9F9CB448BF8010049
:103C6000DAF800B00DF0A2F9CB448BF80B00DAF8CB
:103C700000B00DF09BF9CB4409F10109B9F10A0F2D
:103C80008BF81500E5D169E38146DFF8A4A109F1BD
:103C9000080BDAF8003000930DF092F90EF090FC6A
:103CA00066490EF099FD009B43F82B00DAF800B04E
:103CB0000DF086F909F10A030BEB830B0EF080FC83
:103CC0005E490EF089FDDAF80030CBF8040000936D
:103CD0000DF076F90EF074FC58490EF07DFD09F1F7
:103CE0000E0B009B09F10109B9F1030F43F82B00FA
:103CF000CBD1B9F1070FDAF800B01AD10DF060F9A5
:103D00000EF05EFC4D490EF067FDCBF84400DAF88A
:103D100000B00DF055F90EF053FC48490EF05CFD73
:103D2000CBF84800DAF800B00DF04AF98BF84C00F7
:103D300012E00DF045F9CB448BF80100DAF800B041
:103D40000DF03EF9CB448BF80B00DAF800B00DF023
:103D500037F9CB448BF8150009F10109B9F10A0FC5
:103D6000C7D1FBE20DF022F9132883463FF6A9AE36
:103D7000DFF8BCA0DAF800900DF018F90023304904
:103D80000C2202FB0312117A814220D1137809EB35
:103D90008B0989F885300DF009F989F886000DF056
:103DA00005F989F887000DF001F9264A264B89F8B4
:103DB00088001A60DAF80000244B00211860853072
:103DC00005F0DCFD224B80F001001870C6E20133E3
:103DD0001C2BD4D175E60DF0E9F80B2882463FF68E
:103DE00070AE134BD3F800900DF0E0F803283FF6C7
:103DF00068AE062303FB0A9989F8DA000DF0D6F8BD
:103E000089F8D5000DF0D2F889F8D6000DF0CEF87B
:103E100089F8D7000DF0CAF889F8D8000DF0C6F877
:103E200089F8D9009AE200BFDC190020300E00208A
:103E3000D40E0020000020410000C84200007A4457
:103E4000B47401083C290020200E0020240E00201C
:103E50000A0000205379092B7FF633AE019BD3F87B
:103E600000900DF0A3F8019B89F80000D3F80090B2
:103E70000DF09CF889F801000DF098F8019B64287A
:103E80001B68A8BF642018710DF090F8019B64288E
:103E90001B68A8BF642058710DF088F8019BFF28AB
:103EA0001B68A8BFFF2098710DF080F8019B642863
:103EB000D3F8009028BF642089F807000DF076F849
:103EC000019B89F80200D3F800900DF06FF8019B78
:103ED00089F80300D3F800900DF072F8D8F800309C
:103EE000A9F80A005B790A2B40F23882DB4BD3F841
:103EF00000900DF05BF889F808002FE20DF060F8F3
:103F0000D74B23F8190009F10109B9F1080FF5D1D0
:103F100024E253790F2B7FF4D4AD0DF047F8072836
:103F200081463FF6CEAD029BD3F800A00DF048F8D5
:103F30000E2303FB09F9029BCA44AAF82501D3F812
:103F400000A00DF03DF8CA44029BAAF82701D3F85F
:103F500000A00DF035F8CA44029BAAF82901D3F855
:103F600000A00DF023F8CA44029B8AF82B01D3F875
:103F700000A00DF01BF8CA44029B8AF82C01D3F86C
:103F800000A00DF013F8CA44029B8AF82D01D3F863
:103F900000A00DF00BF8CA44029B8AF82E01D3F85A
:103FA00000A00DF017F8D144C9F82F01D6E10CF0AC
:103FB000FDFF0F2881463FF684AD0CF0F7FFC9EBFB
:103FC000C90904EB090383F8D00003F1D0090CF010
:103FD000EDFF89F801000CF0E9FF89F802000CF010
:103FE000E5FF89F803000CF0E1FF89F804000CF00C
:103FF000DDFF89F805000CF0D9FF89F8060007F00D
:104000009BFEABE12B78580700F1A8810CF0BAFABF
:1040100006F036F906F0FEF9A0E12B78590700F119
:104020009D81904B4FF4C8721A8097E12B785A0704
:1040300000F194818C4A137843F0040313708DE1EE
:104040002B785B07E4D5C1E1A0600CF0C3FFA36847
:104050001843A06082E10CF0B3FFA4F858010CF003
:10406000AFFFA4F85A010CF0ABFFA4F85C0175E1B6
:104070000CF09CFF84F87A010CF098FF84F87E0124
:104080000CF094FF84F87D010CF090FF84F87F0120
:1040900064E10CF095FFA4F880010CF091FFA4F806
:1040A00082010CF083FF84F884010CF089FFA4F8EE
:1040B000860153E10CF07AFF84F890010CF080FF48
:1040C000A4F89A010CF07CFFA4F896010CF078FF9C
:1040D000A4F898010CF06AFFDAF8003084F8910136
:1040E0005B79082B40F23A810CF06AFFA4F89C013E
:1040F0000CF066FFA4F89E0130E192F805900323CE
:10410000B9FBF3F9B9F1120F3FF6DBACDFF85CA1B4
:104110004FF0000BCB4580F021810CF047FF8AF86F
:10412000A0010CF04DFF40F2ED23984205DD40F672
:10413000CA039842A8BF184601E040F2EE20A0F260
:10414000EE20192390FBF3F00BF1010B8AF8A1018B
:104150000AF1020ADEE70CF029FF84F89201FDE083
:104160000CF024FF04EB090309F10109B9F1080F70
:1041700083F88801F4D1F1E00CF018FFC4F808B01E
:1041800060710CF027FFA3681843A0600CF00EFFCD
:1041900084F890010CF014FFA4F858010CF010FF03
:1041A000A4F85A010CF00CFFA4F85C010CF008FF15
:1041B000A4F880010CF004FFA4F88201CEE053794A
:1041C0004FF0070AB3FBFAF2C2EBC2029A1A12F0DE
:1041D000FF0F7FF476ACB3FBFAFA0AF1FF3A5FFA0D
:1041E0008AFABAF1FF0F00F0B9800CF0DFFE5FFA37
:1041F00080FB4FFA8BF005F05BFA814600283FF414
:1042000060AC80F800B00CF0DBFEA9F802000CF006
:10421000CDFE89F804000CF0C9FE89F805000CF009
:10422000C5FE89F807000CF0C1FE89F80600D4E746
:10423000DFF8389009F1400A0CF0C2FEA9F8A80294
:104240000CF0B4FE89F8AA020CF0B0FE09F10409E2
:1042500089F8A702D145EFD180E000BF0C0F002004
:1042600032250020EA23002064240020FC270020BF
:104270000CF09CFE1F2881463FF623ACD8F8003096
:104280005B79082B7FF41DAC0CF09AFE09F18A09CA
:1042900004EB890A00F03F00AAF802000CF090FE3F
:1042A000BAF80230800100F4FE501843AAF8020068
:1042B0000CF07CFE000104F829000CF077FE14F8E5
:1042C000293000F00F00184304F829000CF06EFEAE
:1042D0008AF8010009F0E6FA40E0704B012283F809
:1042E00035203BE00CF062FEFF28824622D10023FD
:1042F0008DF81B309DF81B30052B14D89DF81B0042
:10430000674A9DF81B30012102EBC3035B6852F83A
:104310003000994089B2482205F0AEF89DF81B3074
:104320000133DBB2E4E75F484FF48051042205F02B
:10433000A3F813E005283FF6C4AB00200CF086FE7E
:104340000CF060FED9F8000007F070F818B93220C0
:1043500006F087FFF6E7504605F09CF800200CF0C9
:1043600075FEFFF70FBA504B985907F05FF818B970
:10437000322006F076FFF6E707F09EFC05F056FFC8
:104380004A4A4B4BDA60FFF70ABA0C2824D00A28B5
:104390002BD1484D48480CF0DDFE2846232111F072
:1043A00064FA08B1401B20602368002B40D14148CB
:1043B00000213022236011F022FA3B787BB93F4B79
:1043C0009B68002B67D03E48984764E006F07EFE6D
:1043D000FFF7D8B90C2804D13A480CF0BBFE3A4894
:1043E0000DE07F2812D1FFF703B90D28D1D07F2827
:1043F00009D1304A013B002134482360D1540CF0EC
:10440000A9FEFFF7F5B82F2B3FF6F2A8A0F1200286
:10441000D2B25E2A3FF6ECA813B920283FF4E8A8F0
:104420005A1C2260234AD0540CF08CFEFFF7E0B8EF
:104430005A1EA95C202901D11346B6E71D4A002166
:104440002360D154224B234DD3F800A0D5F800B0FF
:10445000DFF86090584611F016FA06465946324683
:10446000484611F019FA1C4A28B919F80630534485
:104470005B78590703D010359542E7D306E09542A3
:1044800004D2701CEB684844984702E013480CF0D3
:1044900061FE00238BE711B0BDE8F08F300E0020E5
:1044A00050A0010800080140642700200400FA051C
:1044B00000ED00E0B41400206CA3010854150020A6
:1044C000660E0020AC940108A7940108D39401085B
:1044D0005000002018790108E87A0108B794010813
:1044E0006B4B6C4A2DE9F04F5E8914684FEA062A3F
:1044F000B4EB0A0A9C884FF000054FEA04481C8977
:104500004FF0000BA4FB0A6765EB0B0B04FB0B776A
:10451000F40944EA476418EB04065C884FF000098C
:104520004FEAE7154FEAC438DC8849EB050787B046
:10453000CDE90467A4FB0A6704FB0B77340A44EA5D
:10454000076418EB04064FEA27259C894FF0000901
:1045500049EB0507CDE90067AAFB046704FB0B776D
:10456000F40D44EA472414F5FA664FEAE75545F19D
:104570000007B6F5FA6F77F10003CDE902679646BA
:1045800066DADDE90489A4FB046704FB05F34FF058
:10459000050C07EB4307A6FB0C230CFB07335F104E
:1045A0004FEA3206B8EB06084FEA920646EA8376EF
:1045B00069EB07099F10DDE90023921B63EB0703FA
:1045C000CDE90023DDE90267334A4FF0FF3396421D
:1045D00077EB0303CDE9048927DA40F6AC520023D8
:1045E000A4185D4104FB05F3A4FB04456FF006022B
:1045F00005EB4305664202FB0566A4FB0223334438
:1046000018EB020649EB0307CDE904670B26A4FB70
:10461000062306FB0533DDE900455B104FEA320255
:10462000A41A65EB0305CDE90045DDE902450AFB67
:104630000BF3AAFB0AAB0BEB430B4FEADA7242EA2D
:104640004B02A41A4FEAEB7365EB0305CDE9024573
:10465000DEF80440009B019DA4FB032304FB05330B
:104660004FEA525848EAC3284FEA6359DDE9042368
:10467000B8EB020269EB03039946D30B43EA4943C3
:1046800000B1036009B1029B0B6007B0BDE8F08F79
:1046900080150020680E002024FAFFFF2DE9F04F5E
:1046A00087B06C4C02916C4922888E680546C2EB3B
:1046B00026135B435200C2EBE602B4F902601B13FF
:1046C0005643B4F90420B4F90A0053439B1303EB97
:1046D000E62606EB860380331B12B6F5FA384FEA5E
:1046E000E6770493CB6847F1FF39A8FB08AB039347
:1046F00008FB09F3B4F908200BEB430BE389A6612F
:104700000593D31708FB03F102FB0911A8FB022351
:104710000B44C1171F030AFB01F300FB0B33AAFB79
:1047200000011603194447EA1257020A42EA0162DD
:1047300092194FEA2123E6887B410032A2FB060151
:1047400043F5004306FB03114B100093CB17019375
:10475000DDE900231343B4F810E0B4F80CC06DD0C9
:104760000FFA8EF0C1170AFB01F1AAFB002300FB30
:104770000B11BDF914600B44F71708FB07F106FB9A
:104780000911A8FB06670F4479047004801841EAF8
:10479000D6315941039B0FFA8CF8C3F5801E72463F
:1047A000D317002212184FEACE764FEAC3774FEAAA
:1047B000C8034B4147EA5E07B61A67EB030740F6AA
:1047C0003543A6FB030103FB0711DDE900230EF0CF
:1047D0005BF9B4F916204E1302FB06FE470B47EABD
:1047E000C147D31707FB03EEA2FB072356437344CD
:1047F00007FB0366A2FB07233344560E46EAC316A3
:104800008219B4F914604FEA636741EB07037143FF
:10481000F71700FB0717A6FB00013944C60C46EA50
:10482000413692194FEAE1474FEA1221B4F91220BA
:104830007B4141EA036113010B4400E000230DB109
:104840001B0A2B60029B13B11A46049B136007B02E
:10485000BDE8F08FEC150020680E0020704770470F
:104860002DE9F041324C334D62892B8AB4F9048032
:104870009A1A2389B4F902E05A43B4F91230D613D4
:10488000B4F91420DB02324493FBF2F232440A26DC
:10489000E2615643A2F57A6202FB02F3B4F90EC05C
:1048A00002FB0EFE02FB08F2B4F90C801B130CFB9A
:1048B00003FC03FB08F31B1403EB62320232E388B0
:1048C000921002F5004253434CF25032B4F920707A
:1048D0004FEAEE2EB4F900400EEBEC2C0CEB840406
:1048E000BC406D690234A5EBA4043A4162434FEA2F
:1048F000D3384EBFB2FBF8F35400B4FBF8F340F6E4
:10490000DE3448BF5B001A12524362430A4C083639
:104910005C43241404EB224202F6CF62361103EB0F
:10492000221300B1036001B10E60BDE8F08100BF49
:1049300094150020680E002043E3FFFF13B50C4BD5
:1049400004465B681B20022101AA984770B19DF8BC
:1049500004209DF8053043EA022303F54E5310333B
:104960004FF48C7293FBF2F32333238002B010BD1B
:104970006C150020054B1A7E02F0FF0122B10122C6
:10498000027000221A76704701707047680E00208E
:1049900037B5104B04465D68187806216A46A8476B
:1049A000A8B19DF800209DF80130012043EA0223C0
:1049B00023809DF802209DF8033043EA02236380A0
:1049C0009DF804209DF8053043EA0223A38003B03C
:1049D00030BD00BF6C15002013B5104B04465B685A
:1049E0003B2006216A469847A8B19DF800209DF813
:1049F0000130012043EA022323809DF802209DF824
:104A0000033043EA022363809DF804209DF80530BB
:104A100043EA0223A38002B010BD00BF6C15002042
:104A2000B0F5807F0ED0BB280ED861280ED829287B
:104A30000ED813280ED809280ED8002814BF062037
:104A40000020704700207047012070470220704707
:104A500003207047042070470520704710B5224C92
:104A60002368998A89B211F4706F1EBF1F4A012012
:104A7000507611F4E06F2BD01A8B9A88890522F4B6
:104A800080624FEA02424FEA12429A8020D41A888A
:104A900092051DD41A88D0050FD51A88D105FCD4EB
:104AA0001A8892B242F400721A801A889205FCD4D5
:104AB0000F4B187802F0D5FA0AE01A8892B242F445
:104AC00000721A809A8822F440721204120C9A80A2
:104AD0002268938A23F470631B041B0C9382054B9A
:104AE00000221A7010BD00BF8C140020680E002038
:104AF00090140020A4140020054A08B5138801333F
:104B00009BB21380034B187802F0ABFA002008BD6B
:104B10008A0E00209014002008B54FF4804008F061
:104B200079F8012801BF044B4FF480425A61034BCE
:104B300008BF987608BD00BF00040140680E002041
:104B400010B5074C2368186908F064F830B1236881
:104B50001A69044B5A61044B01221A7610BD00BF3A
:104B60007815002000040140680E0020F8B50E46BC
:104B70001746084C4FF48055656140F080000CF0FA
:104B8000EDFE3846002132460CF0B2FE25610120D0
:104B9000F8BD00BF000C014070B50E46054C4FF447
:104BA000805565610CF0DAFE30460CF0D7FE2561C9
:104BB000012070BD000C014070B5FFF731FF104CB3
:104BC0000546192006F04DFBA368152000219847E3
:104BD00010B9022006F0C8FB45F01801A368C9B25D
:104BE00016209847A368002117209847A368012141
:104BF0003D209847A3683E200121BDE8704018473A
:104C00006C150020F0B5274D85B0EB7E002B46D10A
:104C1000254C2368002B42D01A68244E12B1B1698A
:104C20000A43B2619A889868ADF8002002228DF894
:104C30000320694604228DF8022001F06CFDB3695F
:104C4000002743F00103B36123680126187B197D17
:104C500001F04CFD2368164993F9150006F0CEFBD0
:104C60002368144A1B695361029308230DEB030068
:104C70008DF80D308DF80C708DF80E6007F09AFFEE
:104C8000236801A85B7D8DF806708DF8043003233E
:104C90008DF805308DF807600CF00CFEEE7605B04F
:104CA000F0BD00BF680E0020781500200010024003
:104CB000414B00080004014037B50446FFF7A2FF4E
:104CC000274B1A68274B9A420ED14FF40053ADF888
:104CD000043002238DF80730042323480DEB030131
:104CE0008DF8063001F017FDFFF78CFF2046FFF727
:104CF00097FE05461D4C8021A3686B2098476420D1
:104D000006F0AFFAA368072168209847642006F0F0
:104D1000A8FAA36800216B209847642006F0A1FA46
:104D2000A36801216B209847A36818211B2098478E
:104D3000A36810211C209847A36829461A20984789
:104D40000B4AA368117819209847A36812213720CD
:104D50009847A36801213820984703B030BD00BFB1
:104D600030000020001BB700001001406C1500202F
:104D70000C16002008B5FFF745FF024B4FF4805298
:104D80001A8008BD0C00002070B50446FFF73AFFFA
:104D90002046FFF745FE0546144C8021A3686B2092
:104DA0009847642006F05DFAA36803216B209847BA
:104DB0000F4AA3681178192098470F2006F051FA7E
:104DC000A36829461A209847A36818211B209847F2
:104DD000A36810211C209847A36802213720984718
:104DE000A36838200121BDE8704018476C150020E9
:104DF0000C16002008B5FFF705FF074B5B7813B1D1
:104E0000012B03D008BD4FF4006201E04FF4805243
:104E1000024B1A8008BD00BF681500200C0000205E
:104E200010B54000204CC0B220702048204C0170CA
:104E3000204800210170012020701F4C23601F4C6E
:104E400023601F4B1A701F4A1F4B107059761F4961
:104E5000086811461A4630B383889C0515D4038828
:104E6000DB050DD447F230530488A40502D5013B7D
:104E7000FAD112E08BB103889BB243F480730380B4
:104E800083889BB243F44073838047F230530878A1
:104E900010B1013BFBD100E013B9BDE810402BE697
:104EA000507E80F0010010BD961400209414002064
:104EB000921400209C14002098140020A0140020BC
:104EC00095140020A4140020680E00208C140020EB
:104ED00007B5002101AB03227720FFF7A1FF9DF862
:104EE00005309DF804001B0243EA00439DF80600CC
:104EF000184303B05DF804FB08B5FFF7E9FF014B69
:104F0000586008BD680E002008B5FFF7E1FF014BAF
:104F1000186008BD680E002007B5F7216B46062211
:104F20007620FFF77DFF9DF800309DF801101B03F0
:104F300043EA01139DF80210094A43EA1113D360B2
:104F40009DF803309DF804101B0343EA01139DF8FC
:104F5000051043EA1113936003B05DF804FB00BF32
:104F6000680E00200F4B13B51B780F4C0BB1A37EBE
:104F7000B3B1032201AB7720F621FFF751FF9DF873
:104F800005309DF804201B0243EA02439DF80620E9
:104F90001343064AB2F92020C2F10802D3406361EC
:104FA00002B010BD2C000020680E002094150020D7
:104FB0000A4B13B51B780A4C0BB1A37E63B10222D6
:104FC00001AB7720F621FFF72BFF9DF804209DF819
:104FD000053043EA0223238202B010BD2C000020DA
:104FE000680E002030B505460C4613462946224679
:104FF000BDE83040682013E713B5062204460121BE
:105000001C206B46FFF70CFF08B39DF801309DF89C
:105010000020042143EA022242F38D0292FBF1F2C6
:105020009DF8023022809DF8032042EA032242F3D9
:105030008D0292FBF1F29DF8043062809DF805200C
:1050400042EA032343F38D0393FBF1F3A38002B001
:1050500010BD13B506220446022118206B46FFF747
:10506000DFFEB8B19DF800309DF801209B0803EBEE
:10507000022323809DF802309DF803209B0803EB58
:10508000022363809DF804309DF805209B0803EB04
:105090000223A38002B010BD314B2DE9F3411B78F0
:1050A0000546002B3BD0002426462746A046013467
:1050B0005320322108226B46E4B2FFF7B1FE08B953
:1050C000002049E09DF801209DF80030202C03EBE2
:1050D00002231BB29DF8032098449DF8023003EB95
:1050E00002231BB21F449DF805209DF8043003EBFA
:1050F00002231BB21E449DF8073003F07F0301D04A
:10510000002BD4D198FBF4F897FBF4F796FBF4F658
:10511000144BA5F800806F80AE801C771CE05320F4
:10512000322106226B46FFF77BFE0028C8D09DF88F
:1051300001209DF8003003EB02232B809DF8032013
:105140009DF8023003EB02236B809DF805209DF84B
:10515000043003EB0223AB8002B0BDE8F08100BF56
:105160007E150020680E002013B502AB03F8012D58
:105170004000214AC0B21070204A0020117020491E
:1051800001220A701F4908701F490B601F490B60FC
:105190001F4B20491A700A701F4B204A587610681E
:1051A0001A4630B383889C0515D40388DB050DD4DB
:1051B00047F230530488A40502D5013BFAD112E02E
:1051C0008BB103889BB243F48073038083889BB2C6
:1051D00043F44073838047F23053087810B1013BA9
:1051E000FBD100E013B9FFF787FC02E0507E80F0AE
:1051F000010002B010BD00BF9614002094140020DE
:105200009C14002092140020A01400209814002068
:1052100095140020A4140020680E00208C14002097
:105220007720482101229FE77720582101229BE720
:105230007620F421312297E7064B002193F82020B5
:10524000054B9201343299767720F42102F0FC026A
:105250008AE700BF94150020680E0020034B00224F
:105260009A767720F4212E227EE700BF680E002078
:1052700003460A466820194676E713B500222A211C
:105280001C20FFF771FF0E2102221C20FFF76CFF8C
:105290000F2103221C20FFF767FF2B2112221C2065
:1052A000FFF762FF164A02249369164843F004038D
:1052B00093612023ADF8043004230DEB03018DF836
:1052C00006308DF8074001F026FA22462C211C20DA
:1052D000FFF74AFF2D2101221C20FFF745FF2E2159
:1052E00000221C20FFF740FF2A2105221C20FFF787
:1052F0003BFF054B4FF480721A8002B010BD00BF17
:1053000000100240000801400C00002008B50F21E9
:1053100008221820FFF728FF0E2218201021FFF77F
:1053200023FF024B4FF480521A8008BD0C0000206E
:1053300008B5134B53201B782D2108227BB1FFF7B2
:1053400013FF31210A225320FFF70EFF2C210C22DC
:105350005320FFF709FF53203821902209E0FFF77F
:1053600003FF31210A225320FFF7FEFE53202C2198
:105370000A22FFF7F9FE40F20912024B1A8008BD1B
:105380007E1500200C00002001F066BFFFF766BB11
:1053900001F062BFFFF762BB2DE9F0474728A0B0DC
:1053A000044600F0628600F2CE802E2800F01186BE
:1053B00067D8222800F0C18423D8032800F0378260
:1053C00014D8012800F02882022840F083860420A7
:1053D0000BF03CFE43200BF006FE4C200BF003FECE
:1053E00046200BF000FE4C2000F0C8BD042800F061
:1053F0002882052840F06E861A200BF027FE002434
:1054000031E2282800F0828515D8242800F069852B
:10541000262840F05F86E44C06200BF017FEB4F817
:1054200058010BF016FEB4F85A010BF012FEB4F856
:105430005C0100F045BD2A2800F07B852C2840F057
:105440004986D94C0C200BF001FE94F890010BF02A
:10545000CAFDB4F89A010BF0FCFDB4F896010BF00C
:10546000F8FDB4F898010BF0F4FD94F891010BF0FD
:10547000BAFDB4F89C010BF0ECFDB4F89E0100F00D
:105480001FBD3A2800F0E6821DD8342800F077844A
:105490000DD8302800F0B385322840F01B8601205B
:1054A0000BF0D4FDC04B93F8920100F067BD362895
:1054B00000F07585382840F00D8604200BF0C6FDFD
:1054C000B94C00F014BD402800F05B8511D83B2892
:1054D00000F02C843D2840F0FD85B34C02200BF0F9
:1054E000B5FD94F8E0010BF07EFD94F8DF0100F0CB
:1054F00045BD452800F0DB8500F2A685422840F036
:10550000E985A94C10200BF0A1FD60790BF06BFD33
:10551000A0680BF0A7FD94F890010BF064FDB4F8BF
:1055200058010BF096FDB4F85A010BF092FDB4F857
:105530005C010BF08EFDB4F880010BF08AFDB4F82D
:10554000820100F0BDBC6F2800F0DE8200F2E68030
:10555000662800F0C48100F2BB804D2800F0EF8483
:1055600015D8492800F0AA824B2840F0B3858E4C0C
:1055700004200BF06BFD94F8D6010BF034FD94F889
:10558000D7010BF030FDB4F8D80100F099BC6428C5
:1055900000F08281652840F09D85844C0B200BF043
:1055A00055FD20880BF055FD608880B20BF051FD51
:1055B0007F4B1B68C3F3C000C3F38002800040EA46
:1055C0004200C3F340021043C3F3401240EAC2005A
:1055D00003F0100318430BF03CFDA288A36802F00F
:1055E000080103F4475949EA010903F4804149EAF3
:1055F000010903F4004149EA010903F4803149EA51
:10560000010903F4003149EA010903F4802149EA60
:10561000010903F4002149EA010903F4801149EA70
:10562000010903F0007349EA0303DFF8889112F0DF
:10563000010F99F8009018BF4FF00208C9F38009D4
:1056400008BF4FF0000843EA090312F0020F43EAD3
:10565000080314BF4FF0040C4FF0000C12F0040FBD
:1056600043EA0C0C14BF4FF0100E4FF0000E12F076
:10567000400F14BF202700274CEA0E0E12F0100F27
:1056800014BF4FF4007600264EEA070712F0200FF1
:1056900014BF4FF4806500253E4312F4807F14BF91
:1056A0004FF400600020354312F4007F14BF4FF424
:1056B00000110021284312F4806F41EA000114BF59
:1056C0004FF08063002300201943247B0346F3E05E
:1056D000692800F0A2810AD8672800F0298168288B
:1056E00040F0F88410200BF0B1FC00248DE16D280F
:1056F00000F0A68100F2B4816C2840F0EB842B4CC2
:1057000006200BF0A3FCB4F868000BF0A2FCB4F880
:105710006A000BF09EFCB4F86C00D1E3772800F02F
:10572000978354D8732800F0B38345D8702800F0CD
:105730001D82722840F0CE841B4C16200BF086FC94
:10574000B4F896010BF085FCB4F840010BF081FC35
:10575000B4F842010BF07DFCB4F844010BF079FC85
:10576000B4F8D8010BF075FC00200BF03CFC0020D5
:105770000BF039FC00200BF036FC94F885010BF09F
:1057800032FC94F892010BF02EFC00200BF02BFC65
:10579000064B0A20DB6CB3F9623093FBF0F080B269
:1057A0000BF057FCA3E300BFFC270020880E00206D
:1057B0000816002021300020742800F00583752889
:1057C00040F088842F200BF041FCBF4CA6E2A028BB
:1057D00000F079830AD8782800F0B6807B2840F062
:1057E00079843C200BF032FC002441E2F12800F0E7
:1057F000E680FE2800F05783F02840F06B84B34C1D
:1058000004200BF023FCE36CB3F866000BF021FCE2
:10581000E36CB3F8640053E303200BF017FC0020A3
:105820000BF0E1FB20460BF0DEFB0D20A6E30BF0B6
:105830000DFC01200BF0D7FB0B200BF0D4FB00205C
:105840009CE306200BF002FC41200BF0CCFB462031
:105850000BF0C9FB4E200BF0C6FB41200BF0C3FB45
:105860009B4B18782CE39B4B185D01340BF0BBFB72
:105870000B2CF8D10024984B185D01340BF0B3FBCE
:10588000082CF8D10024954B185D01340BF0ABFBCC
:10589000072CF8D100F01CBC07200BF0D7FBE72049
:1058A0000BF0A1FB8E4B58790BF09DFB00200BF009
:1058B0009AFB042000F00ABCA3420AD2894A9D5CEC
:1058C000012202FA05F50D421CBF9A401043013334
:1058D000F2E70BF0C7FB824B93F8B0074EE31220C0
:1058E0000BF0B4FB804B00251B88B3F5806F8CBF99
:1058F00008260126754C04F1280333F915000135FB
:1059000090FBF6F080B20BF0A4FB032DF2D1E08DFA
:105910000BF09FFB208E0BF09CFB608E0BF099FB35
:10592000A08E0BF096FBE08E0BF093FB208FC7E26E
:1059300010200BF08BFB00246C4B185D01340BF036
:1059400052FB102CF8D1C3E370200BF07FFB002634
:105950000E2474435D4D0136EB6C2344B3F82501EE
:105960000BF077FBEB6C2344B3F827010BF071FBD2
:10597000EB6C2344B3F829010BF06BFBEB6C234475
:1059800093F82B010BF02FFBEB6C234493F82C01C5
:105990000BF029FBEB6C234493F82D010BF023FB58
:1059A000EB6C234493F82E010BF01DFBEB6C1C44B5
:1059B000D4F82F010BF056FB082EC9D188E37020D4
:1059C0000BF044FB464C04F1700594F8D0000BF04A
:1059D0000AFB94F8D1000BF006FB94F8D2000BF010
:1059E00002FB94F8D3000BF0FEFA94F8D4000BF00D
:1059F000FAFA94F8D5000BF0F6FA073494F8CF00D1
:105A00000BF0F1FAAC42E0D162E3394B185D01349E
:105A10000BF0E9FA102CF8D15AE3364D002428781F
:105A2000400000F0FE000BF011FB2B789C4280F050
:105A30004F83314B33F814000BF00BFB0134F4E7C8
:105A4000224C06200BF002FB206F0BF00BFBB4F88E
:105A5000740035E204200BF0F9FA1C4B986F35E323
:105A60004FF6FF7507200BF0F1FA244B174C1888FE
:105A7000FF28A8BFFF20C0B20BF0B5FA204B186872
:105A8000A842A8BF284620EAE07080B20BF0E1FAF5
:105A9000B4F87C000BF0DDFA114BD4F8800093F8D9
:105AA00085313BB10A235843A842A8BF284620EAC3
:105AB000E07001E000F30F0080B201E202200BF081
:105AC000C5FA104B1888FBE183740108880E00208A
:105AD00025300020339301083F93010817930108F4
:105AE000FC270020950E00200C000020C20E002094
:105AF000D80E0020E42F00203E270020881B002025
:105B0000E01A002010160020C04C0B200BF09EFA6B
:105B1000D4F88430254618780BF065FAD4F8843030
:105B2000002658780BF05FFAD5F88430B74C334430
:105B3000187901360BF057FA032EF5D1D4F88430DA
:105B4000D8790BF050FAD4F8843098780BF04BFAEF
:105B5000D4F88430D8780BF046FAD4F884305889D9
:105B60000BF077FAD4F88430187A07E2A74C1E209D
:105B70000BF06CFAE36C00251B78022B65D1E36C0B
:105B800005F1080253F82200A1490CF071FD10F054
:105B900043F880F30800C0B20BF025FAE36C9D498E
:105BA00003EB8503D86A0CF063FD10F035F880F341
:105BB0000800C0B20BF017FAE36C05F10E0253F8BF
:105BC000220095490CF054FD10F026F880F30800EF
:105BD000C0B201350BF007FA032DD0D1072DE36CCD
:105BE00021D1586C8A490CF043FD10F015F880F370
:105BF0000800C0B20BF0F7F9E36C8549986C0CF023
:105C000037FD10F009F880F30800C0B20BF0EBF993
:105C1000E36C93F84C000CF0D3FC0FF0FDFF80F325
:105C20000800C0B20BE02B4458780BF0DCF9E36CB1
:105C30002B44D87A0BF0D7F9E36C2B44587D01350F
:105C40000BF0D1F90A2DC9D142E2E36C2B4458780C
:105C50000BF0C9F9E36C2B44D87A0BF0C4F9E36C70
:105C60002B44587D01350BF0BEF90A2DEDD12FE202
:105C7000664D04F10802EB6C674953F822000CF002
:105C8000F7FC0FF0C9FF80B20BF0E3F9EB6C62494F
:105C900003EB8403D86A0CF0EBFC0FF0BDFF80B27D
:105CA0000BF0D7F9EB6C04F10E0253F822005A49BD
:105CB0000CF0DEFC0FF0B0FF013480B20BF0C9F93C
:105CC000032CD5D1072CEB6C16D1586C52490CF033
:105CD000CFFC0FF0A1FF80B20BF0BBF9EB6C4E498B
:105CE000986C0CF0C5FC0FF097FF80B20BF0B1F987
:105CF000EB6C93F84C000BE0234458780BF0A9F9B7
:105D0000EB6C2344D87A0BF0A4F9EB6C2344587D58
:105D100001340BF09EF90A2CD4D1D9E114F8010F0B
:105D2000002800F0D5810BF05EF9F7E701200BF0B9
:105D30008DF9364BDB6C187820E150200BF086F99A
:105D40000025324B0C21DC6C344B04EB850494F8B9
:105D50008520013501FB023393F838000BF043F93D
:105D600094F886000BF03FF994F887000BF03BF9AC
:105D700094F888000BF037F9142DE2D1A8E14820FF
:105D80000BF064F90025214BDC6C062303FB054472
:105D900094F8DA000BF027F994F8D5000BF023F90A
:105DA00094F8D6000BF01FF994F8D7000BF01BF90C
:105DB00094F8D8000BF017F9013594F8D9000BF0DE
:105DC00012F90C2DDFD183E14FF0000801260027E6
:105DD0000E4B1A7B974232DA0D33FA5C00240C2307
:105DE00063430E4D05F13001595C914207D12B44BC
:105DF000586B0FF048FD82462EB9B14610E00134D1
:105E00001C2CECD119E0804417E000BF880E002064
:105E1000000020410000C84200007A448474010858
:105E2000D1450ADA0C2303FB04535B6B13F809001A
:105E30000BF0D9F809F10109F2E70137C8E7002EA4
:105E400000F046815FFA88F00BF000F90026BEE70B
:105E5000AE4D0024287B0BF0F9F82B7B9C4280F0A0
:105E60003781AB4B0021E65C0C2202FB01F3A94811
:105E700000F13007DA5DB24205D1034493F83800EF
:105E80000BF0B1F802E001311C29EDD10134E4E757
:105E900008200BF0DBF80124E0B201340BF0A3F88A
:105EA000092CF9D114E108200BF0D0F800200BF0F8
:105EB000D0F800200BF0CDF800200BF0CAF800203D
:105EC0000BF0C7F804E10C200BF0C0F8924B1868F7
:105ED0000BF0C8F8914B18680BF0C4F8904B186899
:105EE000F4E004200BF0B2F88E4B9868EEE094F8E2
:105EF0007A010BF078F894F87E010BF074F894F8BE
:105F00007D010BF070F894F87F0137E0854C072095
:105F10000BF09CF8B4F880010BF09BF8B4F8820108
:105F20000BF097F894F884010BF05DF8B4F8860153
:105F3000C6E701200BF08AF87A4B58791EE07A4CBC
:105F40007A4D2078002600EB4000C0B20BF07EF8BE
:105F5000237802359E4280F0BB8015F8020C0BF0CE
:105F600042F815F8010C013600EB800000EB8000D0
:105F700000F2EE2080B20BF06CF8E9E70BF033F89A
:105F8000A6E008200BF062F80024664B234493F847
:105F9000880101340BF027F8082CF6D198E05B4B10
:105FA000604C93F8880004F12805C0EBC000C0B233
:105FB0000BF04CF894F8F00100235D4AD25C90425B
:105FC00000F08A800C333C2BF7D10834AC42F1D17D
:105FD0007EE040200BF03AF8524C04F14005B4F852
:105FE000A8020BF036F894F8AA020AF0FCFF043479
:105FF00094F8A7020AF0F7FFAC42F0D168E0E02085
:106000000BF024F8474C04F18005B4F82A0204345C
:1060100000F03F000BF01DF8B4F82602C0F3861024
:106020000BF017F894F8240200090AF0DCFF94F84A
:10603000240200F00F000AF0D6FF94F825020AF0BF
:10604000D2FFAC42E1D143E03A4C0D200AF0FEFF12
:1060500000F03AFF0AF0C7FFA0880BF003F82069B0
:106060000BF000F807F0A6FD30E00AF0B3FF05469C
:1060700084200AF0EBFF28460AF0F4FF2D4B1C6940
:1060800005F18003A3428CBF641B802407F04CFE03
:1060900028462246694600F09BFD05460024AC4296
:1060A00016DA1DF804000AF09EFF0134F7E713200A
:1060B0000AF0CCFF0024204B185D01340AF093FF56
:1060C0000B2CF8D100200AF0CDFF00200AF0CAFF07
:1060D000012018E0002016E00AF085FFB4F8F20174
:1060E0000AF0B7FF94F8F4010AF07DFF94F8F50187
:1060F0000AF079FF94F8F7010AF075FF94F8F601B9
:106100000AF071FF61E720B0BDE8F087880E00203B
:10611000950E002084740108E8F7FF1FECF7FF1FBD
:10612000F0F7FF1FFC270020E42F00209C2900200F
:106130002C1600200C000020339301088379DB0724
:1061400048BFB1FA81F1D0F8343148BF49095A68E3
:106150001B8909B1136170475361704710F80A3CFD
:106160000133DBB20A2B84BF10F8131C044A00F879
:106170000A3C82BF002322F8113000F80A3C704725
:10618000001A0020334A70B5136C9068194440F629
:106190008C23081A98429160D060516013463BD915
:1061A000127893F9451010468A420BD1111F082925
:1061B00008D893F84610182901D8013103E083F874
:1061C000442002E0002183F8461093F9444021491D
:1061D000A24219D191F84740B4B10C310024944245
:1061E00006DA51F8046F1C4D25F814600134F6E707
:1061F0000C2805D01849002421F810400130F7E799
:10620000164801780131017083F8452000220121F0
:106210001A7083F8471070BD92F84710C9B140F268
:10622000DA51A0F2EF248C4208D811780B2905D856
:106230000B1D0131117042F8230070BD002283F85C
:106240004720074B03F13002002143F8041F93421B
:10625000FAD170BDEC000020001A00209D0500203E
:10626000F8000020024A136C01331944116470478E
:10627000EC000020024B53F820301B681980704757
:10628000F8170020074BA1F57A7153F820301A68EF
:106290001B8959434FF47A7391FBF3F189B2118052
:1062A000704700BFF817002038B50D4B0D4D9968A9
:1062B0000D4B1A681C465288114203D004F0AAFF05
:1062C000286007E004F0A6FF2B68984282BFC01A3E
:1062D000064B186023685A68054B5A6138BD00BFE9
:1062E000000C0140140F00200807002000000020CF
:1062F0000004014090F83B3210B57BB990F83A3277
:1063000090F83942A34209D2B0F8401201229A40D3
:106310000A430133A0F84022DBB2F3E710BD1FB5FA
:106320000123ADF80830ADF80410002301A9ADF841
:106330000A30ADF80C30ADF8062006F028FB05B0A9
:106340005DF804FB10B5A0F5127494F83C22BAB9BC
:10635000A36A616A994228D0591CA069A162C35CF2
:106360002069DBB25B0043F400738142A4F83E3243
:106370004FF00A0384F83D3228BFA262012312E0E5
:1063800094F93D327BB1B4F83E1220464B08A4F894
:106390003E3201F00101FFF7D1FE94F83D32013B9E
:1063A00084F83D3201E084F83C3294F83832002B16
:1063B0004ED194F839320133DBB2092B84F83932EB
:1063C00003D12046BDE8104094E70A2B40D194F851
:1063D0003B322BB9B4F8403243F00103A4F8403209
:1063E0006379D9071CD5B4F84002820501D4C307EC
:1063F00005D4B4F844320133A4F8443210E0E36A1F
:10640000C0F347000BB198470AE0E3696269D054D2
:10641000E369E1680133B3FBF1F201FB1233E3619D
:10642000012284F8382294F83B220023012A84F8C0
:1064300039320DD1A27984F83B32236B12F0010F6F
:106440001868997A0CBF02220022BDE8104066E766
:1064500010BD1FB50123ADF808300023ADF80C3096
:10646000ADF80A30084BADF804101B7801A9012BD8
:1064700008BF0323ADF8062008BFADF80C3006F0C6
:1064800086FA05B05DF804FBE800002038B510F886
:106490000E2C044650F8043C52B9012200F80E2C90
:1064A00020F80C1C997A18680222BDE83840D0E721
:1064B00030F80C2C20F80A1C891A89B220F8081C24
:1064C000074A10F80F0C002522F8101004F80E5C93
:1064D0001868997A2A46FFF7BCFF04F8065C38BDB5
:1064E000001A0020044B53F820301BB107289CBF32
:1064F0001B681980704700BF14020020D4E6D3E661
:10650000D2E6084A13689B020BD5074B002119708D
:106510004FF6FE730549086803400B604FF4001303
:106520005360704700000240203000206C000240A1
:106530002DE9F047664D6B686649581C0A788E460F
:1065400002F0FF060AB10346F6E737466B60687C47
:10655000EB6895F81080AA7C39B2202900F09C8065
:10656000DFF880C10CEB8103DC789B783CF82110CC
:10657000C3F1FF039BB2002B65D04FF03C0CB1FB85
:10658000FCF9C3F1FF0363431B12B9F1050F5DD89A
:10659000DFE809F0030B1A293A4AE01A4143B1FB3C
:1065A000FCF0DAB21044C0B251E0B1FBFCF00CFBDD
:1065B000101189B2DAB2C1F13C01E31A4B43B3FBCB
:1065C000FCFC204694442CE0B1FBFCF00CFB1011C9
:1065D000E21A89B24A43B2FBFCF25FFA83F8424402
:1065E000D2B2204632E0B1FBFCF90CFB191189B2A2
:1065F000E01AC1F13C014843B0FBFCF05FFA83F8BC
:106600004044C0B2224621E0B1FBFCF80CFB18115B
:10661000D8B289B2E31A01FB03F2B2FBFCFC2246BA
:1066200084445FFA8CF412E0B1FBFCF80CFB181107
:1066300089B2D8B2C1F13C01E31A4B43B3FBFCF27F
:106640000244D2B203E02246204600E044464FEA2C
:10665000042C4CEA004C4CEA020C17234FF00108C2
:1066600008FA03F806F1170118EA0C0FA1EB030171
:10667000DFF8748014BF4FF011094FF0090989B297
:1066800013F1FF3308F80190E8D218360137B6B29B
:10669000BFB2114BA0465FE7EB6001238EF80030DC
:1066A00040F22A33AA740D4A69810D4985F8108099
:1066B00068742E81536000238B840B889BB243F057
:1066C00001030B80136843F001031360BDE8F087FA
:1066D000140F002020300020240F00206C00024006
:1066E00000040040540C00204002002001F003038D
:1066F00001F0FC0101F1804101F5803110B59B00F2
:106700008C680F229A4024EA02028A608A689840C4
:1067100002438A6010BDF0B5B1F800E000234EFAE4
:1067200003F2D50725D58E784FEAD30CF40648BF7F
:10673000CC7806F00F0203F0070748BF2243BF00E2
:1067400050F82C500F24BC4025EA0404BA402243E0
:10675000282E40F82C2005D1C46801229A4024EA52
:10676000020205E0482E04D1C46801229A40224367
:10677000C2600133102BD2D1F0BD2DE9F04F1E467F
:106780004FF414734343554D85B005F1140480460E
:106790009146E718A24610B92B44514A03E001285C
:1067A00005D1504A2B445A641032C3F848214FF4A3
:1067B000147303FB08F34C48EC180AEB030203F5CF
:1067C0009C733432534460612164A262E36200220C
:1067D0004FF480714FF0010BD4F84831032021624F
:1067E000626322636162E263A26384F8502284F8E8
:1067F0004CB284F84D22A4F85622A4F85822C4F8CA
:106800001C906076A67684F85A8258681B8904F535
:10681000A2724FF0020CADF80C3003A910230192C4
:106820008DF80E308DF80FC0CDF800C0FFF773FF64
:10683000636CDDF800C0597B58681B898DF80E1019
:1068400003A9ADF80C308DF80FC0FFF764FF59466F
:106850003846FFF773FC322004F003FD234B019A06
:106860001B68D2F804B01A46B2FBF9F1B1F5803FCB
:1068700003D3012AF8D95208F6E71D4A4FF41474DD
:10688000B3FBF2F204FB08F8584689B2D2B207F023
:106890003BFB05EB0809174B08F512780AEB0804D7
:1068A0000022C9F85C325846214607F075FBD9F83A
:1068B000445016F0010F0CBF022200222868A97A6A
:1068C000FFF72DFD0C4B2846C9F86032211D002230
:1068D00007F062FB384605B0BDE8F08F140F0020CA
:1068E0002492010844920108107601084C0000200F
:1068F00040420F004563000889D200082DE9F743A4
:106900008E460546DFF8A092114699F8B444006817
:10691000164698467246631C89F8B43407F0A0FA0C
:106920002B8901A9ADF8043018238DF8063068686A
:1069300002238DF80730FFF7EEFEAB7A09F5976773
:10694000240127442A6849460C2B00F2F680DFE830
:1069500013F00D00F400F400F4005100F400F40012
:10696000F4008A00F400F400F400C200138CDFF895
:106970003CC223F001031B041B0C1384138CB2F8DC
:1069800004E0108B624520F073004FEA00404FEAAC
:1069900010409BB21FFA8EFE40F0700014D00CF530
:1069A000006C624510D00CF5406C62450CD00CF5C3
:1069B000806C624508D00CF5806C624504D023F0F1
:1069C000020343F0030307E023F00E032EF4407E9E
:1069D00043F003034EF4807EA2F804E01083A2F893
:1069E00034801384138B23F008031B041B0C43F027
:1069F000080336E0138CDFF8B4C123F010031B0446
:106A00001B0C1384138CB2F804E0108B624520F445
:106A1000E6404FEA00404FEA10409BB21FFA8EFE5C
:106A200040F4E04008D00CF5006C624504D023F03F
:106A3000200343F0300307E023F0E0032EF4406E20
:106A400043F030034EF4806EA2F804E01083A2F805
:106A500038801384138B23F400631B041B0C43F452
:106A60000063138369E0138CDFF840C123F4807363
:106A70001B041B0C1384138CB2F804E0908B62454A
:106A800020F073004FEA00404FEA10409BB21FFA1B
:106A90008EFE40F0700008D00CF5006C624504D00A
:106AA00023F4007343F4407307E023F460632EF48F
:106AB000405E43F440734EF4805EA2F804E090839D
:106AC000A2F83C801384938B23F008031B041B0C57
:106AD00043F0080330E0138CDFF8D0C023F4805378
:106AE0001B041B0C1384108CB2F804E0938B20F46D
:106AF000005023F4E6431B0400041B0C000C624509
:106B00001FFA8EFE43F4E04340F4405003D00CF5EE
:106B1000006C624503D12EF4804E4EF4804EA2F8F4
:106B200004E09383A2F840801084938B23F40063E5
:106B30001B041B0C43F4006393832B7B43B1B2F81B
:106B400044306FEA43436FEA53439BB2A2F84430A8
:106B500013889BB243F001031380AB7A0C2B19D836
:106B6000DFE803F0071818180B1818180F18181872
:106B700013000B1902F134000AE00B1902F138007E
:106B800006E00B1902F13C0002E00B1902F1400093
:106B9000C3F8B80438460C44A4F8C064C4F8BC2454
:106BA00003B0BDE8F08300BF140F0020002C0140AB
:106BB000064B70B506461C461D6800F085F918B9ED
:106BC00023685B1BB342F8D970BD00BF9C1B00203B
:106BD000F7B503238DF80430030C8DF805308DF8DC
:106BE0000700030A06200F4614468DF80630FFF70B
:106BF000DFFF78B1084D4FF4805601A904226E6181
:106C000000200AF075FE3846002122460AF070FE88
:106C100020462E6103B0F0BD000C014037B504469C
:106C200003211E2006226B46FEF7FAF870B39DF88A
:106C300001309DF80000164D43EA002000B20BF031
:106C4000C3FC29680BF014FD0BF0D8FE9DF803304F
:106C500020809DF8020043EA002000B20BF0B4FC53
:106C6000A9680BF005FD0BF0C9FE9DF80530A0806A
:106C70009DF8040043EA002000B20BF0A5FC69680F
:106C80000BF0F6FC0BF0BAFE6080012003B030BDC3
:106C90002000002010B5054C2368186905F0BAFFE4
:106CA00018B123681A69024B5A6110BD14160020EE
:106CB000000401402DE9F0437B4A87B013689046F9
:106CC00093B11A681AB17949886902438A619A882E
:106CD0009868ADF8002002228DF80320694604224E
:106CE0008DF80220FFF717FD322004F0BAFA0021D8
:106CF00011221E20FEF738FA012160221E20FEF725
:106D000033FA642004F0ADFA002402A8FFF786FFEE
:106D1000274626460A25022101221E20FEF724FAD4
:106D2000322004F09EFA02A8FFF778FFBDF9082090
:106D3000BDF90A1014448A42A8BF0A46BDF90C30B6
:106D40000F4493421E44A8BF134613F5805F09DD2C
:106D5000574A013DD36883F01003D360DBD14FF075
:106D6000010901E04FF000091E2000211222FEF768
:106D7000FBF90A25022101221E20FEF7F5F9322037
:106D800004F06FFA02A8FFF749FFBDF90820BDF92A
:106D90000A10A41A8A42A8BF0A46BDF90C307F1A0D
:106DA0009342A6EB0306A8BF134613F5805F07DDE9
:106DB0003F4A013DD36883F01003D360DAD101E08C
:106DC0004FF0000920460BF0FFFB014639480BF05D
:106DD00003FD394D20F00040286038460BF0F4FBED
:106DE000014634480BF0F8FC20F000406860304663
:106DF0000BF0EAFB014631480BF0EEFC20F00040BE
:106E0000A860002170221E20FEF7AEF90121202289
:106E10001E20FEF7A9F91E2002210022FEF7A4F988
:106E2000642004F01EFAB9F1000F04D14FF07E5334
:106E30002B606B60AB60D8F800301B4C1A7B002ACB
:106E40002FD01A7D6AB3194900268A69012542F0BC
:106E500001028A61187B197DFFF748FC23681849F5
:106E600093F9150004F0CAFA2368164A1B6904A8AE
:106E7000536104930C238DF815308DF814608DF850
:106E8000165005F097FE236801A85B7D8DF806601B
:106E90008DF8043003238DF805308DF807500AF083
:106EA00009FD07B0BDE8F083141600200010024071
:106EB000000C014000406F462000002001C05E46EB
:106EC000956C0008000401400F4B73B518781C4600
:106ED00098B105230D4D8DF800304FF480560023F6
:106EE0008DF8013001A86E61694602220AF000FDAA
:106EF0002E619DF8050000F0010000F001002070F7
:106F000080F0010002B070BD8D050020000C014032
:106F1000024640213C20FEF727B970B500EB800007
:106F2000094CA0F1A1059C3825440444074B15F8F1
:106F3000010F1E787040FFF7EBFFA542F6D13046F7
:106F4000BDE87040E4E700BF34760108223000203D
:106F500010B5441E14F8010F10B1FFF7DEFFF9E77A
:106F600010BD024680213C20FEF7FEB810B5D420AB
:106F7000FFF7F7FF8020FFF7F4FFA820FFF7F1FFEE
:106F80003F20FFF7EEFFD320FFF7EBFF0020FFF7D6
:106F9000E8FF4020FFF7E5FF8D20FFF7E2FF142018
:106FA000FFF7DFFFA120FFF7DCFFC820FFF7D9FFC5
:106FB000DA20FFF7D6FF1220FFF7D3FF8120FFF77B
:106FC000D0FFCF20FFF7CDFFD920FFF7CAFFF12078
:106FD000FFF7C7FFDB20FFF7C4FF4020FFF7C1FF2B
:106FE000A420FFF7BEFFA620FFF7BBFFAF20FFF7EF
:106FF000B8FFA620FFF7B5FFAE20FFF7B2FF2020B5
:10700000FFF7AFFF0020FFF7ACFFB020FFF7A9FFAD
:107010004020FFF7A6FF0020FFF7A3FF1020FFF797
:10702000A0FF4FF48064013C0020A4B2FFF770FF82
:10703000002CF8D18120FFF794FFC820FFF791FFC3
:10704000AF20FFF78EFF012010BD08B55038C0B249
:10705000FFF787FF0020FFF784FFBDE808401020FE
:107060007FE7012828BF01202DE9F04F0646734F26
:10707000142000FB0671724BD1F8A4421E711C60F3
:10708000704BD1F8B422DD69B1F8AC822A43DA61E1
:10709000A288B1F8AEA222F44072D1F8A85212042C
:1070A00089B0120C4AEA0809A28003A9C5F8109019
:1070B00002228DF80E0028460193ADF80C908DF851
:1070C0000F20FFF728FB019B00971F464FF0080B8E
:1070D000AA6818EA020F03D10A2004F0B7F8F7E70C
:1070E0000A20C5F8148004F0B1F8C5F810800A2011
:1070F00004F0ACF8BBF1010BEAD1C5F814A00A20EA
:1071000004F0A4F8C5F814800A2004F09FF8C5F82C
:1071100010800A2004F09AF80222C5F810A0284630
:1071200003A98DF80F201C228DF80E20ADF80C90CD
:10713000FFF7F1FA444A03A894423A690BBF42F4BC
:10714000001242F480023A613A610BBF3A693A692F
:1071500022F4001222F480023A61A38823F44073DF
:107160001B041B0CA38023889BB243F001032380E4
:10717000A58805F0B1FB0599344B25F03F05B1FB1F
:10718000F3F32D042D0C1D43ADB2A58022880025FC
:1071900022F001021204120C22802D4A03A8B1FB36
:1071A000F2F100298AB208BF012242F400414FF4F3
:1071B000967253434FF47A7293FBF2F301339BB20E
:1071C0002384A1832388009A9BB243F00103238088
:1071D000238823F4816323F002031B041B0C238008
:1071E0004FF480432381142303FB062696F8B13223
:1071F00001248DF80C308DF80D508DF80E508DF85F
:107200000F400AF057FB96F8B0329DF80F208DF82A
:107210000C308DF80D508DF80E501AB103A80AF0FD
:1072200049FB08E05A0903F01F039C4002F12003C8
:10723000084A42F8234009B0BDE8F08F34760108CF
:107240008C140020001002400054004040420F0007
:10725000009F240000E100E0914B70B51A68908A0D
:1072600080B2C1B2CE072ED5118821F40061090485
:10727000090C1180118889B241F4806111800021CC
:107280005971997999B1D97911B9197AFF290ED122
:107290000121D971597A022901BF118889B241F4BB
:1072A00000611180997A41F001011182E2E0997A3E
:1072B00001F0FE0111821A7AFF2A00F0DB80784A81
:1072C000FF215171D6E08D073AD5BFF35F8F587A11
:1072D000C0B2012813D1997989B1D97979B11188CE
:1072E00021F480610904090C1180BFF35F8F118BB9
:1072F0001188D87289B241F4007111801BE0118BA2
:10730000BFF35F8F587A664902280AD1887940B165
:10731000C97931B1118821F480610904090C118007
:10732000A2E0587A5E49032805D1887918B1C97955
:10733000002940F09980918889B241F4806198E0F9
:107340004C0757D50121D9729979002938D0D979BC
:10735000002935D0597A1088022959791ED920F48C
:1073600080600004000C1080148ADD68C8B2E4B2AA
:1073700049B26C541188DC6889B241F40071118003
:107380001968821C5A710A8A0130D2B240B2225462
:107390008A8892B242F480628A8026E080B240F409
:1073A00000701080148ADD68C8B2E4B249B26C542F
:1073B000128A411C49B2D2B203306A54587114E0A7
:1073C000D979374809B9017C41B1118889B241F4B2
:1073D000007111805A7901325A7106E0118889B220
:1073E00041F4807111800122C27119680A88D205A6
:1073F000FCD43FE001F0400101F0FF04E1B1587915
:10740000168ADD68C4B2611C40B2F6B22E54C9B20D
:107410005D7A597149B2C81C854201BF908820F439
:1074200080600004000C08BF90805A7A8A4221D103
:107430001B4A023454711DE006061BD5597948B227
:10744000451C0AD05C690131205CC9B21082587AAF
:10745000597149B288420DD106E0197A5C711182E6
:10746000997909B9597A29B9918821F48061090477
:10747000090C9180597A93F9050001318842084A34
:107480000CD10021D171D17A31B111688A8822F4EE
:1074900040721204120C8A8000221A7670BD00BF5E
:1074A0008C140020344B354A1B68126810B51A60E2
:1074B000334A11685960516892689960DA60314ABC
:1074C000116819615168926859619A612E4A116870
:1074D000D9615168926819625A622C4A11881985DB
:1074E000518859859188D2889985DA85284A1188EA
:1074F00019865188598692889A86264A1188D98693
:10750000518892881987194621F83A2F224A107813
:107510000022824206DA214C34F81240013221F86E
:10752000024FF6E71E4A1288A3F864201D4A12880B
:10753000A3F866201C4A1188A3F86C105188928821
:10754000A3F86E10A3F87020184A3B2112689A66BF
:10755000174A126892FBF1F2B2F5967FC8BF4FF05E
:10756000FF325A67134A1288A3F87820124A5289C8
:10757000A3F85E2010BD00BF902500200830002039
:10758000602300206C230020782300208A1600202E
:10759000B60E0020B00E00207C160020D80E002071
:1075A000FC1A0020540E0020BC0E0020DC06002037
:1075B00000000020040F0020C20E0020A0F17D0377
:1075C000012B70B504460D460A4E05D830687D2162
:1075D00003F035FF84F020043068214603F02FFFCC
:1075E00035B12B881C4404EB142404F0FF042C80D8
:1075F00070BD00BF440C002010B50A4C5E28014647
:10760000206805D15D2103F01AFF20683E2105E0C6
:107610005D2903D103F013FF20683D21BDE8104030
:1076200003F00DBFA81400202DE9F84305460E46CF
:107630000D4B002493E88003B44213DA7B1933F92D
:10764000140008EB050333F9142009EB050333F9A3
:10765000143001341344022293FBF2F3C01A09F0F0
:10766000DDFAE9E7BDE8F8839025002010B5104B5E
:10767000014693F8D837012B12D10E4A0E4C1078E0
:10768000431CDBB213701B0644BF0023137021544C
:1076900006F088FB3F2809D9BDE8104006F060BB22
:1076A000064BBDE81040186803F0C9BE10BD00BF0E
:1076B000FC270020AC240020AE24002074250020EC
:1076C0007FB5264C264E274D2749284A284B20B106
:1076D00028480088B0F5805F32D230881F4E91F87C
:1076E00020101278ADF8040028781B78351D8DF82D
:1076F00006008DF807108DF8082001A829460622FB
:107700008DF809300EF060F830B30198BDF80830FC
:107710007060AB805320FFF7A9FFA08809F06EFAD4
:10772000A07909F06BFAE37901A80193237A029317
:10773000637A039309F0D2F90E4B00221A800BE012
:10774000308891F82010A080127828781B78A071DA
:10775000E17122726372DDE704B070BDA8140020ED
:107760008C0E002064240020A01B0020080D0020A7
:10777000B60D0020382700200A4A138801331380F1
:10778000094A136801331360084A138801339BB216
:10779000202B01BF00231380054A138808BF013343
:1077A00013807047382700201C2700202027002046
:1077B0002227002038B5294B05461B780C46083B8C
:1077C000012B4AD84520FFF751FF2846FFF74EFF0F
:1077D0000E2D33D003D83DB10D2D07D038BD142D5B
:1077E00020D0FF2D32D038BD20682BE06378207880
:1077F0009BB180F08000FFF739FFA568E8B2FFF782
:1078000035FFC5F30720FFF731FFC5F30740FFF74A
:107810002DFF280EFFF72AFF04E0FFF727FF60681F
:1078200009F0FCF92078FFF721FF606809F0F6F90C
:107830002489E0B2FFF71AFF200A0BE0206809F064
:10784000DDF96068BDE8384009F0D8B9044809F0AE
:10785000E9F90020BDE8384008E738BD7025002070
:10786000F19501082DE9F04FBB4B89B01A881C46F1
:10787000BA4F002A40F0A98042F20103B7F8D607B8
:10788000B74EC21A50425041FFF71AFFFFF70AFEE7
:10789000346849202546FFF7E9FEB24B04F11C0984
:1078A000186809F0ABF955F8040B09F0A7F9284658
:1078B0000AF0DDF804F110000AF0D9F84FF01008D2
:1078C000A94D01232A6803FA08F3134203D0D9F81B
:1078D000000009F0A3F908F10108B8F1130F09F14C
:1078E0000409EDD104F128000AF0B1F8B7F84031ED
:1078F000B4F92E00C01A09F081F92B68DB0408D511
:107900009A4BB4F864001B88181AC0F30D0009F0F4
:1079100075F92B68980403D5B4F8660009F06EF980
:107920002B68590503D504F16C000AF090F82B6818
:107930001A0502D5A06E09F071F92B685B0402D517
:10794000606F09F06BF92B68180403D5B4F8780060
:1079500009F054F9A04604F130000AF078F804F177
:1079600036000AF074F8B7F8403138F93C0F0127B7
:10797000C01A09F043F97E4B1B789F4208DA38F9A8
:10798000020FB4F93C300137C01A09F047F9F2E7A9
:107990002B68990505D5B4F95E00A0F2DC5009F01A
:1079A0003DF9326873487260B260121A9110724ADF
:1079B0004A43531C032293FBF2F202EB42029A1A4F
:1079C0007C2303FB020333609BE16C4B6C4A1B6816
:1079D00011688B4206D008A941F8203D00201360B1
:1079E000FFF7E8FE97F8D617238897F8D7070B44D8
:1079F000013BB3FBF0F200FB12338B4280F081813C
:107A0000574C0120FFF75CFEFFF74CFD5020266825
:107A10006568FFF72BFEA268236810681B68626820
:107A200003441068A046A3EB400009F0F7F86A6829
:107A3000736868469B1A0093AA68B36806F11C0B2A
:107A40009B1A0193EA68F36805F11C0A9B1A0293DA
:107A50000AF00DF82A69336968469B1A00936A692F
:107A6000736910279B1A0193B369AA699B1A029341
:107A700009F034F83C4901230A68BB4013428946A7
:107A800006D0DBF80000DAF80030C01A09F0C6F8BA
:107A90000137132F0BF1040B0AF1040AEAD106F1A6
:107AA000260005F12601002330F9022F31F9024F9B
:107AB000121B4DF823200133042BF5D1032200279C
:107AC0005DF82230BF00FFB26BB103F108010F294E
:107AD00002D847F0010706E08033FF2B94BF47F040
:107AE000020747F0030712F1FF32E9D238460024BB
:107AF000FFF7BCFDEB46A24607F00303022B16D0AE
:107B0000032B1DD0012B4ED1BAF1000F05D1DBF8AC
:107B100000409A462401E4B245E0DBF800004FF053
:107B2000000A00F00F002043FFF7A0FD3BE0BAF190
:107B3000000F0CD0DBF80000C0F3031020432CE052
:107B4000BAF1000F1ED19BF80100FFF78FFD9BF8E3
:107B50000000FFF78BFD26E020270020FC270020F7
:107B6000902500201C27002014270020102700202B
:107B70007C1600209C250020DF7BEFBD28270020FD
:107B800024270020DBF80000C0F303302043FFF778
:107B90006DFDDBF80000C0F30710FFF767FDDBF8B1
:107BA00000402401E4B20BF1040B04AB9B454FEA07
:107BB0009707A1D1BAF1010F02D12046FFF756FD78
:107BC000D9F8003013F480541FBFB6F86420B5F81C
:107BD00064100124521A18BF00929A040AD508AA08
:107BE00002EB8401B5F86600B6F866200134121A7B
:107BF00041F8202C5F0512D506F16A0705F16A00ED
:107C00000DEB840E002237F9021F30F902CFCCEBC6
:107C100001014EF822100132032AF4D10334180571
:107C200008D508AA02EB8400A96EB26E0134521A7C
:107C300040F8202C590408D508AA02EB8400696F8B
:107C4000726F0134521A40F8202C1A040BD508AB7D
:107C500003EB8402B5F87810B6F8783001345B1A7B
:107C600042F8203C00E0DCB1012C03D1009808F080
:107C7000D5FF15E0631E00205DF823204000C0B250
:107C80000AB140F00100013BF6D5FFF7EFFC0027F9
:107C90005DF8270008B108F0C1FF0137A742F7DB04
:107CA00030200321FFF7C0FC36200321FFF7BCFC86
:107CB000164B3C201978FFF7B7FCD9F800309B052C
:107CC00006D5B6F95E00B5F95E30C01A08F0A6FF19
:107CD000D8F800200E48D8F80430C8F80420121A4A
:107CE00091100C4AC8F808304A43531C032293FBF6
:107CF000F2F202EB42029A1A7C2303FB0203C8F859
:107D0000003008F0D9FE09B0BDE8F08F7C160020E5
:107D10009C250020DF7BEFBD2DE9F74F0E9FC2EBC6
:107D2000030B4C4C0D9B002914BF4FF006094FF07C
:107D30000409FF1A636882460133164634D122686B
:107D40004A4580F08280DFF82881019158F82200AE
:107D50000DF099FD0B3008F04FFE0199054608B172
:107D6000012073E022683C48032A98BF514658F826
:107D7000222008F0E9FF394A1368181A6368106076
:107D800001336360364B9D720EE00D9A92B103FB96
:107D900007F20D99895C01228A40324909680A423A
:107DA00008D163680133636063680C9A294D93427C
:107DB000EBDB32E003FB0BF5236806EB050A2BB97E
:107DC00070590DF060FD00F1050801E04FF0030867
:107DD000404608F011FE0028C2D1204A204B10680E
:107DE000C8EB000010609A7A1AB12C20FFF73EFC15
:107DF00001E001229A72236843B9705908F012FF1A
:107E00009AF904104B1CCCD0174803E09A44174849
:107E10009AF8041008F098FFC3E710D1012008F089
:107E2000EBFD60B90D4A0A201368013B1360FFF7B0
:107E30001DFC2B6801332B604FF0FF336B60206813
:107E400048452CBF0020012000E0002003B0BDE821
:107E5000F08F00BF30270020FC9501082C27002060
:107E6000A8140020142700200B96010849A101083E
:107E70000079010830B585B004AC002524F8025D16
:107E80000091ADF8060021461020FFF797FB9DF802
:107E900006002146FFF792FB9DF807002146FFF7F9
:107EA0008DFB9DF800002146FFF788FB9DF801003F
:107EB0002146FFF783FB9DF802002146FFF77EFB7A
:107EC0009DF803002146FFF779FB9DF80E00294637
:107ED000C043C0B2FFF772FB05B030BD10B5054C12
:107EE000206803F0A9FA18B1206803F0A2FAF6E7B7
:107EF00010BD00BF1C0C00200028114AB8BF404232
:107F000090FBF2F330B50F4C3C2504FB03006843B3
:107F10000D4D90FBF2F22D682D7B25B903EB830309
:107F200003EB830301E0C3EB031302EB830304FBC6
:107F300002020B804FF47A7392FBF3F24A8030BD59
:107F400080969800806967FFD40B002010B5044626
:107F5000C0B2FFF751FBC4F30720BDE81040FFF7A4
:107F60004BBB024B5E21186803F069BAA8140020CD
:107F700038B50546054C5E21206803F060FA20689C
:107F80002946BDE8384003F05ABA00BFA8140020C3
:107F900038B500240B4D6059254409F0DBF86968B9
:107FA00011B1094801F0EEFFA96811B1074801F0CD
:107FB000E9FF0748103409F0CDF8B4F5E87FE9D1BE
:107FC00038BD00BF187901082F96010835960108C1
:107FD0006CA3010870B5054628460DF054FC064612
:107FE00058B91A4B1A485A791A4BBDE8704003EB3E
:107FF0008203D3F8CC1101F0C5BF2846164932469A
:108000000DF04AFC60B9154809F0A4F8144C54F876
:10801000041F19B1134801F0B5FFF8E7124805E055
:108020000024124B53F8241021B91148BDE87040C8
:1080300009F090B8284632460DF02EFC0134002895
:10804000EFD1024B0B4D5C71C6E700BFFC2700204F
:108050003B96010818790108479601084C960108DB
:10806000E47A01085F9601086CA30108E87A010828
:1080700063960108D6940108F0B585B004460DF06A
:1080800002FC082826D1621EE01D1F4912F8013F9C
:1080900009681944497801F00301022908BF203B0F
:1080A00082421370F1D1254604F1080715F8016BDF
:1080B000164831460DF0D9FB20B1284631460DF067
:1080C000D4FB10B100F024FF1CE0BD42EED12046ED
:1080D00009F048FD0E4809F03DF800230D4A04A9B7
:1080E0001A4492F888210A440849595C0133082B44
:1080F00002F80C1CF2D10023074801A98DF80C30BE
:1081000001F040FF05B0F0BD5000002067AD010850
:1081100072960108FC27002010A201082DE9F04703
:1081200005460DF0B0FB314E0446D6F8088090B9F4
:108130002F4809F00FF82F4B53F8241049B10123B1
:10814000A34013EA080F02D02B4801F01BFF0134B3
:10815000F1E72A4822E02846294922460DF09CFBF7
:1081600058B9284808F0F6FF274C54F8041F002996
:10817000EFD0214801F006FFF7E72B784FF0000918
:108180002D2B03BF013504F1FF344FF0010A4FF0EE
:10819000000A184B53F8297027B91C48BDE8F0476E
:1081A00008F0D8BF2846394622460DF075FBC8B9FD
:1081B000012000FA09F0030601D51548EEE7BAF1EF
:1081C000000F03D002F02AF8124803E040EA08004A
:1081D000B060114808F0BEFF3946BDE8F0470F48CF
:1081E00001F0D0BE09F10109D3E700BFFC27002050
:1081F00078960108507B01085F9601086CA301087E
:1082000047960108829601084C7B01086396010895
:108210008E9601089C960108A59601080FA20108F8
:1082200010B5084808F096FF074B00241C701C632B
:10823000064B1C7003F064FD09F032F9044B1C601E
:1082400010BD00BFAD960108B414002023300020FB
:108250005425002070B5064600240B4BE518AA886B
:1082600016420AD0E158094801F08CFE2846002148
:1082700008F001FF064808F06DFF40F6CC331434D7
:108280009C42EAD170BD00BF88850108D9960108DB
:108290006CA3010808B5084801F074FE05F092FDD2
:1082A000FEF712FE18B9642002F0DBFFF8E703487E
:1082B000BDE8084001F066BEE3960108F0960108AB
:1082C0002DE9FF410A48068885684488B0F8048093
:1082D000C76805F06FFCCDF8008002900197314629
:1082E0002A462346034801F04DFE04B0BDE8F08164
:1082F00010000020F8960108F0B504788BB0054610
:108300000CB1002436E04B4B19680E2303FB04111B
:10831000B1F92951B1F92521B1F92731009591F829
:108320002C5101F59070019591F82D5101F5947142
:10833000029590F90B00039091F906103E480491C4
:108340002146013401F01EFE082CDCD170E02D2BFB
:1083500014D1072C1BDC28460DF0EAFA0AAB661C88
:1083600003EB440424F8100C15F8013F303B092BB3
:10837000FAD934462B78002BE9D104E0A3F130027E
:10838000092A09D8E5E7082CBDF8182009D00BB058
:10839000BDE8F04000F0BCBD202BF8D101352646E9
:1083A000E7E7072AF3D840F2DC55BDF81A00214B65
:1083B000A0F2EE2189B2A9421B68E8D8BDF81C10D2
:1083C000A1F2EE24A4B2AC42E1D8BDF81E6004B222
:1083D00037B2A742DBDB0DB2AF42D8DCA542D6DB19
:1083E000BDF8247007F16404A4B2C82CCFD8BDF83E
:1083F00026E00FFA8EF4112CC9DCBDF82050B42D04
:10840000C5D8BDF82240B42CC1D812B24FF00E0C22
:108410000CFB0233A3F82501A3F82711A3F8296167
:1084200083F82C5183F82D4183F82B7183F82EE1CA
:108430000BB0F0BDD40E002055970108F0B50446EE
:108440008FB020460DF01FFAC5B21DBBAE4808F034
:1084500081FEAE4C94F8D21009B9AD4853E049B250
:1084600094F8D02094F8D130009194F8D310A94812
:10847000019194F9D4100734029194F9CE1003912C
:1084800094F8CF1004912946013501F07BFD102DA1
:10849000E0D1E2E72046A04905220DF0FDF90546AE
:1084A000B8B929469D4870220DF0A9F928469C4B81
:1084B00019680E2303FB001301300022082883F8FB
:1084C0002F2183F8302183F8312183F83221F0D134
:1084D00018E12046934904220DF0DEF905462046B6
:1084E000002D4AD120210DF0C0F9002800F00A81AA
:1084F000461C30460DF0C7F92C4607468A4B53F808
:1085000024502DB989480FB0BDE8F04001F03ABDC4
:1085100030462946FAB20DF0BFF901340028EDD1FA
:108520007A4A164602F17001002382F8D63082F8AA
:10853000D23082F8D13082F8D03007328A42F3D17B
:108540007B4901EBC40191F89022934210DAD1F8F3
:108550009472C3EBC302B0183A44176800F1D0011B
:10856000C0F8D07090880133888092798A71E7E7EB
:108570002946704801F006FD95E06F4907220DF08D
:108580008BF905462046002D49D120210DF06DF9CB
:1085900006460DF078F9C4B26CBB684801F0F2FCF5
:1085A00021466748013401F0EDFC0E2CF8D1584803
:1085B00001F0E8FC00246348214601F0E3FC0025BB
:1085C000574A012311680E2202FB0412D2F82F2110
:1085D000AB4013425C4B5D495D4808BF194601350D
:1085E00001F0D0FC0E2DEBD14948013401F0CAFC5A
:1085F000082CE0D186E0304656490DF09DF92C4616
:10860000002852D0022C55D00DF092F906AB43F859
:108610002400504900200DF08FF90134F0E74D4956
:108620000DF08AF9002460B1082C3ED00DF080F9DD
:1086300006AB43F82400474900200DF07DF90134D2
:10864000F1E7082C31D1069B0F2B2ED8DDF81CE06A
:10865000BEF1070F29D8089F0D2F26D8099E06F1D5
:108660006402C82A21D80A9DFF2D1ED80B986428C1
:108670001BD80C99642918D8884216DA0D9C032C53
:1086800013D8224AC3EBC303134483F8D0E083F822
:10869000D17083F8D26083F8D35083F8D40083F884
:1086A000D51083F8D6402C4CCBE60FB0BDE8F04097
:1086B00000F02EBC069B072B20D807990D291DD84A
:1086C0000278722A0DD06E2A18D1154A0E2012682F
:1086D00000FB032301228A40D3F82F1121EA020272
:1086E00009E00F4A0E20126800FB032301228A4092
:1086F000D3F82F110A43C3F82F2101E000F008FC42
:108700000D4C9EE60FB0F0BD7D970108FC270020C0
:108710006CA30108A8970108C4970108CC28002081
:10872000D40E0020CA970108E87A01086396010870
:1087300018790108CF970108759701083996010843
:10874000DB97010849A1010874A60108D4A5010816
:10875000E0970108E4970108D69401082DE9F74352
:10876000047805468CB9324D95F8AB12B5F8A822BD
:1087700095F8AA322F4800912146013401F002FCFD
:10878000102C05F10405EFD14EE00DF0D1F80F28C3
:10879000044636DC284620210DF067F8264EE4B268
:1087A000D6F83480451CA400002728460DF0C0F8F8
:1087B0005FFA87F9B9F1010F83B208D0B9F1020F5E
:1087C0000BD0B3F5B47F24D2726B13530AE0FF2BA6
:1087D0001FD8736B2344987004E0FF2B19D8736B78
:1087E0002344D87028462C210DF03FF8054608B1E7
:1087F000013502E0B9F1020F0BD10137032FD4D1BB
:1088000012E00E4800210F2203B0BDE8F04300F053
:10881000FCBA08EB0400002104220CF0F0FF03B0C6
:10882000BDE8F04300F074BB03B0BDE8F08300BFC7
:10883000FC270020E6970108B4140020FA970108ED
:108840002DE9F04304788FB00546002C59D17C4BBC
:108850000021142209A807AED3F838800CF0CFFF0E
:108860000722304600210CF0CAFF00231A46A70059
:1088700005A8059308EB070583807249B5F802E067
:1088800031F813C01CEA0E0F0AD00E310DF1380C6E
:10889000595C02F1010E624402F81C1C5FFA8EF270
:1088A0000133072BE9D100210B46674AB5F802E0F6
:1088B00011F802C01CEA0E0F0AD006320DF1380C76
:1088C0008A5C03F1010E634403F8242C5FFA8EF3F3
:1088D00001310629E9D118F807308DE841006A789E
:1088E0005A49029209A81A0903F00F0301F035FB57
:1088F0002146574809AA013401F044FB202CA6D197
:108900009BE00DF015F81F28044600F389802846E7
:108910002021E4B20CF0A9FF1F2C02D900F0F8FAD4
:108920008BE0474B451C9B6B002103EB84042046E6
:1089300004220CF064FF0027464B09AE30460021AC
:108940000A2217F803905FFA87F80CF058FF00230B
:1089500015F8012B32B10A2B04D04A4502D0F2544B
:108960000133F5E74A4561D108F1FF33032B09D8FC
:10897000DFE803F0100502420DF1230037E00DF1AE
:1089800023011FE030460CF0D3FF2378C0B243EA46
:10899000001006E030460CF0CBFF237800F00F000B
:1089A0001843207034E00133062B0BD02A4800F224
:1089B0007B369E5D9642F6D1034493F87523638817
:1089C0001343638011F8012F12B30023EEE7013344
:1089D000072B0CD0204A02F26E369E5D8E42F6D1F5
:1089E00002EB4303B3F8602363881343638010F8FA
:1089F000011F69B10023EDE730460CF099FF0F2805
:108A000004DC30460CF094FF607001E000236370DA
:108A10000137052F90D1012404F044FF6CB97DE7A4
:108A20000E4800211F2200F0F0F906E02046002148
:108A300004220CF0E4FE0024EEE70FB0BDE8F08362
:108A4000B4140020787C01088D7C0108009801088E
:108A50000F980108997C010818790108FA97010814
:108A60002DE9F04FAC498BB004460CF0D1FEAB4978
:108A7000002820460CBF012507250CF0C9FEA84997
:108A80000028204608BF02250CF0C2FE002808BFBF
:108A90000425E90740F1E780A24808F05BFB0020CD
:108AA00008F064F9A04CA14808F054FBA04808F075
:108AB00051FB62799F4BA04803EB8203D3F8CC11A2
:108AC00001F060FA9D4801F05DFA26460027D6F8CD
:108AD00010800021404609F05FFF20B1984801F066
:108AE00051FA002669E039469648D6F814B0D6F80F
:108AF00018A0D6F81C9001F045FA4046002109F074
:108B000055FF10B1202008F01DFB06A9404601F0DA
:108B1000BFF801468C4801F035FA5846002109F0AB
:108B200045FF10B1202008F00DFB06A9584601F0C2
:108B3000AFF80146844801F025FA5046002109F0BB
:108B400035FF10B1202008F0FDFA06A9504601F0CB
:108B50009FF801467C4801F015FA4846002109F0CB
:108B600025FF10B1202008F0EDFA06A9484601F0D3
:108B70008FF801370146754801F004FA0C2F06F111
:108B80001006A4D1AAE749B294F8D02094F8D130C5
:108B9000009194F8D3106E48019194F9D4100734E1
:108BA000029194F9CE10039194F8CF1004913146BC
:108BB000013601F0E7F9102E03D094F8D210002905
:108BC000E1D1644808F0C6FA574B634C9F6854F8EB
:108BD000041F19B1614801F0D5F9F8E70E46604B62
:108BE00053F826404CB10123B3403B4203D05D48CB
:108BF000214601F0C7F90136F1E75B4808F0AAFA0F
:108C00002146494B0AAA0B4493F888311344574A2A
:108C10008A5C0131082903F8102CF2D1002306A93F
:108C200053488DF8203001F0ADF9524808F092FA1F
:108C3000514800F051FD514808F08CFA4E48FFF7BA
:108C4000FFFD4F4808F086FA4B48FFF787FD4D4877
:108C500001F098F94020FFF7FDFA4B4808F07AFA46
:108C6000454800F073FBAA0739D5484808F072FA66
:108C7000474808F06FFA404808F0B8F8454808F04F
:108C800069FA3D4800F0CEF8434808F063FA3A48E4
:108C900000F0AEFA414801F075F9374800F03EF9AE
:108CA0003F4808F057FA3448FFF726FB00260E2706
:108CB000774300243B4A0123D26BA3403A44D2F8C5
:108CC0000A2013421ED101340E2CF3D10136082E96
:108CD000EDD12C4801F056F98020FFF7BBFA6B0765
:108CE00016D5314808F036FA304808F033FA2248F1
:108CF00008F056F8234801F045F94FF48070FFF76B
:108D0000A9FA05E031462246294801F03BF9DAE7A5
:108D10000BB0BDE8F08F00BF1B9801086A9C0108EA
:108D20002298010828980108FC270020369801089D
:108D30004898010818790108549801085F980108BB
:108D40006C980108799801083896010810A201086A
:108D500091980108819801084C7B0108B09801089E
:108D6000507B0108BE980108CB98010867AD010847
:108D7000D7980108E0980108D6940108EF980108F7
:108D8000FB9801086CA301080999010816990108CC
:108D9000299901083799010841990108509901085A
:108DA0005E990108B41400206A9901087B990108B2
:108DB0008D990108F8B504460E4617460025204651
:108DC00020210CF052FD0446D0B1013420460CF0B5
:108DD000AFFDB0F5617F05DB40F634039842A8BFD4
:108DE000184601E04FF46170A0F56170192390FB03
:108DF000F3F00DB9307000E070703B7801333B70D8
:108E00000DB90125DBE72046F8BD30B505460C4617
:108E1000134629462246BDE83040014801F0B2B869
:108E2000749F01087FB504780646E4B9354B1921D3
:108E3000186800EB840090F8875090F885204D4327
:108E400005F5617590F88630009590F888004143EB
:108E500001F5617101912C482146013401F092F82D
:108E6000142CE3D14BE00CF063FD1328054641DCE4
:108E7000244B701C1C68202100238DF80F300CF04F
:108E8000F4FC2035064670B1013630460CF050FD3A
:108E90001A289FBF04EB850358719DF80F300133EA
:108EA00098BF8DF80F30304620210CF0DEFC0646CE
:108EB00070B1013630460CF03BFD0D289FBF04EB2E
:108EC000850398719DF80F30013398BF8DF80F30EE
:108ED00004EB85043046E11D0DF10F02FFF76AFF38
:108EE0009DF80F30042B0AD0601D002104220CF0E5
:108EF00086FC04E0054800211322FFF786FF04B03A
:108F000070BD00BFD40E0020939F0108FA9701089E
:108F1000014808F01FB900BFA89F0108F8B5047800
:108F2000064674B9304D2146B5F8C421B5F8C631AE
:108F30002E48013401F026F8042C05F10405F2D185
:108F4000F8BD2B490CF064FCA8B9274B4FF47A719B
:108F50004FF4FA62A3F8C411A3F8C621A3F8C8110C
:108F6000A3F8CA21A3F8CC11A3F8CE21A3F8D011FD
:108F7000A3F8D221F8BD30460CF0DAFC03280546F0
:108F80002BD8304620210CF070FC044630B101345F
:108F900020460CF0CDFC0126074600E006462046A0
:108FA00020210CF062FC10B9BDE8F840B0E70130B8
:108FB0000CF0BEFC012EF7D140F2DC53A7F2EE22FA
:108FC0009A42F1D8A0F2EE229A42EDD8064B7035C3
:108FD00003EB85039F80D880F8BD0648002103225B
:108FE000BDE8F84011E700BFFC270020B69F01084C
:108FF000C49701088CA401082DE9FF4104780546B7
:10900000002C34D16D4808F0A5F86D4D2869002179
:1090100009F0C2FC002840F0CE802146694800F0EB
:10902000B1FF2869694600F033FE0146664800F04A
:10903000A9FF6869694600F02BFE0146624800F00E
:10904000A1FFA869694600F023FE01465E4800F0D2
:1090500099FFE869694600F01BFE013401465B4850
:1090600000F090FF0C2C05F11005CFD1A3E058497A
:1090700005220CF011FC38B9514B0022034410308A
:10908000C0281A61F8D196E02846524904220CF013
:1090900003FC04462846002C3FD120210CF0E5FBC0
:1090A000002800F08880451C28460CF0ECFB0746A1
:1090B000494B53F824601EB9484808F04BF87AE051
:1090C00028463146FAB20CF0E7FB01340028EFD114
:1090D0003B4B0021C2181030C02811619E46F7D1C9
:1090E0003F4B03EBC402D2F804C09846BCF1000F1A
:1090F00004D131463B4800F045FF53E0002718F803
:1091000034309F42F5DA3B010EEB03051035634422
:109110000FCB013785E80F00F1E70CF009FC0B28B5
:10912000064643DC284620210CF09FFB054648B14B
:109130000135284600F016FD214B012403EB0613F0
:10914000186100E00446284620210CF08EFB0546FD
:1091500040B10135284600F005FD194B013403EB01
:1091600006135861284620210CF07FFB054640B1CC
:109170000135284600F0F6FC114B013403EB0613D1
:109180009861284620210CF070FB10B9FFF7C0FE53
:1091900011E0013000F0E6FC094B032C03EB06164E
:1091A000F061F3D11048FFF727FF04E00F480121D9
:1091B0000C22FFF72AFE04B0BDE8F081C99F010828
:1091C000FC270020E49F0108EA9F010810A2010883
:1091D000C4970108CA970108E87A01086396010854
:1091E000A49E0108CF970108D6940108FA970108B8
:1091F000F0B5047887B0064614BB514B19201968A6
:10920000062303FB041191F8D65091F8DA20454368
:1092100005F5617591F8D530009591F8D750D031AA
:10922000684300F561700190087A0290497A4548D8
:1092300003912146013400F0A5FE0C2CDDD17CE029
:109240000CF076FB0B28044672DC3D4B701C1D684D
:10925000202100238DF817300CF007FB064680B163
:10926000013630460CF064FB03289FBF062303FB46
:10927000045383F8DA009DF817309CBF01338DF852
:109280001730304620210CF0F0FA074680B1013744
:1092900038460CF04DFB0D289FBF062303FB0453FB
:1092A00083F8D5009DF817309CBF01338DF8173037
:1092B00006266643A9193846D6310DF11702FFF785
:1092C00079FD20210CF0D1FA074670B101373846FC
:1092D0000CF02EFB14289FBF9DF817307619013330
:1092E00086F8D80098BF8DF81730384620210CF04A
:1092F000BCFA78B101300CF01BFB0D289FBF062390
:1093000003FB045383F8D9009DF817309CBF013349
:109310008DF817309DF81730062B0ED0062202FB71
:1093200004500021D5300CF06AFAFFF7F1FD04E09B
:10933000054800210B22FFF768FD07B0F0BD00BF14
:10934000D40E0020EE9F0108FA9701082DE9F3479B
:10935000047807464CB9204601A908F067FB0134A0
:10936000FFF7F4FF122CF6D178E00CF0E1FAC5B269
:10937000112D6ED8781C20210CF077FA394C05F1AC
:10938000D00614F816800346374F30B9A8F1020210
:10939000D2F1000848EB020843E000F1010A5978D5
:1093A00038460CF062FA60B1032D8CBF0323002312
:1093B000C01BC0B23B44184490F80490B9F1030FAD
:1093C00002D1FFF7A5FD49E0A9F10203D3F100089E
:1093D00050464FF0200148EB03080CF046FAD8B194
:1093E000B8F1000FEDD001300CF0A2FA40F2ED23FD
:1093F00080B2984205DD40F6CA039842A8BF1846DD
:1094000001E040F2EE20A0F2EE20192290FBF2F0F3
:1094100004EB4603587002E0B8F1000FD1D104F814
:10942000169014F81630FA5CB8F1000F0CD00D4B02
:109430000E4803EB4606717819234B43294603F285
:10944000EE2300F09FFD09E02946094800F09AFD4F
:1094500004E0084800211122FFF7D7FC02B0BDE864
:10946000F08700BFFC2700205C7D01080EA00108EA
:1094700020A001088CA4010807B50123ADF8041051
:1094800001A98DF806208DF80730FDF744F903B0E7
:109490005DF804FB2DE9F843054672B6424C4FF4E3
:1094A00080614FF400776161204648226761FFF7D1
:1094B000E3FF204639461022FFF7DEFF3B4B03EB6C
:1094C000C502506853F835604FEAD00E384B06EBB2
:1094D0008E021A6056F82E2000F007015A608900AB
:1094E0009A600F228A40D24399469D6815409D603C
:1094F0005D682A405A609D6808228A402A439A6023
:109500005A68012505FA01F10A435A605A688540F4
:1095100046F82E2035612761A3685805FCD440F633
:109520000557D9F80420D9F800301A604FF40073B9
:10953000756163611F4B08221A6110225A61A3688A
:10954000DFF86480590503D4002FF8D0013FF6E717
:10955000482235613046A9B2FFF78EFF154A102325
:10956000136187B1A268104B5205D8D5B2684FF489
:10957000007015420F4A4FF0080115BF186158617D
:1095800011615161EEE74FF400710823C8F8101023
:10959000404613611822FFF76FFF62B6BDE8F8433B
:1095A0000A2001F05EBE00BF0008014050A0010883
:1095B000F4140020000C014030B5094900220B785A
:1095C000084C1557854202BFFF25155503F1FF339F
:1095D00002F10C0208BFDBB23C2AF1D10B7030BDA6
:1095E000100F00202C160020002208490C2303FB3A
:1095F00002135968814204D10022C2621A725A6071
:1096000070470132052AF0D1704700BF2C160020A8
:109610002DE9F743064689469DF8288011461A46EB
:109620009DF82C3000250C2068431D4FC419C057ED
:10963000B04202D1207A20B12DE00135052DF2D1C2
:1096400029E0022E0FD005DC56B1012E23D1009364
:1096500014480AE01E2E0ED01F2E1CD101200AE055
:109660000093114801E011480093434603F0BEFE09
:10967000044638B90FE0FDF780F8036841469B695E
:10968000044698470C2303FB05752671204685F890
:1096900008906C6000E0002003B0BDE8F08300BFDC
:1096A0002C160020004400400038014000480040D3
:1096B00010B5084B0022196801EBC20393F9024070
:1096C000844201D1981C10BD0132052AF4D100203A
:1096D00010BD00BF28160020F0B5027887B08AB907
:1096E0004A4C04F1280694F8F0210023484950B26E
:1096F000595681426ED00C333C2BF7D10834B4421A
:10970000F1D181E0002204920592451C0CF010F981
:10971000C4B260B2FFF7CCFF074618B18DF8104015
:10972000012400E00446284620210CF09EF805465E
:1097300038B1013528460CF0FBF80134ADF81200C1
:10974000E4B20026284620210CF08FF8B0B3451C67
:1097500028460CF0EDF800222E495FFA82FE51F8FF
:109760002230834204D00132082AF5D1002300E0E0
:10977000734651F82320824220D1022E0FD0032EAF
:1097800012D05A1E012ED2B204D0042A13D88DF85A
:1097900014300EE0042A0ED88DF8153009E0052BA0
:1097A00009D88DF8173004E09A1E052A03D88DF8E1
:1097B00016300134E4B20136042EC3D1052C04D88E
:1097C00007B0BDE8F040FFF7A3BB04AB03CB3860A4
:1097D000796019E094F8F5010E4B94F8F45153F8C0
:1097E0002000B4F8F221009094F8F70153F820001B
:1097F000019094F8F60153F8200053F825300290B8
:10980000054800F0BFFB79E707B0F0BDFC2700205A
:109810002C160020B09101082FA0010838B1438810
:1098200011EA030003D08B420CBF012002207047D5
:1098300030B50A4B0A491C680A7B042A0AD8134629
:10984000551C04EBC303EAB29D882842F5D00A7385
:10985000981C30BD0A73002030BD00BF28160020C0
:10986000F4140020014B00221A73E1E7F4140020E5
:109870002DE9F047877890F803C0BBB2C7F1640EBA
:1098800003EB83065C42C3F178001C4D5FFA8EFE49
:109890007600CCF16408A4B280B2A3B20FFA83F9C7
:1098A000B9F1000F04DC002B14BF3B46012300E09C
:1098B000734609FB09F25B4302FB0CF292FBF3F3E4
:1098C000434403FB09F30A2293FBF2F333449BB2B4
:1098D00025F8023FB1F800904A880A34C9EB020A21
:1098E0001AB202FB0AF24FF47A7392FBF3F3A4B2BA
:1098F0004B4484422B80D0D1BDE8F0870015002076
:1099000010B544780078002240F6C41102FB02F33F
:10991000193B634303F6C4135343434393FBF1F3EF
:10992000034921F812300132072AEDD110BD00BFE2
:109930001A150020104B043033F91000B0F5617F88
:1099400005DB40F633039842A8BF184601E04FF408
:1099500061700A7819235A4302F28332824208DA8C
:109960004A78534303F283338342B4BF002001207B
:1099700070470020704700BF3E27002010B500F15F
:10998000500302788A4203D18478C278944204D387
:1099900004309842F5D1002010BD012010BD0B4BC2
:1099A0001B6813F4805F0A4BB3F9063005D0C089F9
:1099B000421A934207DD084400E0008A8342B4BFA4
:1099C0000020012070470120704700BF901B00203D
:1099D0003E2700201FB5084B1B681B0309D58DF8D7
:1099E0000400039101230D2001A98DF80530FDF736
:1099F000E1FE05B05DF804FB901B0020F0B50124EA
:109A0000B0FBF4F58D4201D34C43F9E70026D4B105
:109A1000B0FBF4F504FB1500B4FBF1F41EB9002D06
:109A200001DC002CF3D1092D03F1010EEFB204DDAE
:109A3000002A14BF3725572500E030253D441D700E
:109A400001367346E3E71C70F0BDF0B50124B0FBAE
:109A5000F4F58D4201D34C43F9E70026D4B1B0FBB5
:109A6000F4F504FB1500B4FBF1F41EB9002D01DC84
:109A7000002CF3D1092D03F1010EEFB204DD002A11
:109A800014BF3725572500E030253D441D700136B1
:109A90007346E3E71C70F0BD03685A1C026019703E
:109AA00070472DE9F843089E002B07468846144668
:109AB000334614BF4FF030094FF0200913F8012B43
:109AC0000AB9254603E0002CFBDD013CF6E7002D3A
:109AD00004DD38464946C047013DF8E7354624EAEB
:109AE000E474A01B284415F8011B11B13846C04787
:109AF000F7E7BDE8F883024B186801F0A0BC00BF8F
:109B0000600E0020F8B507460C464868002115464F
:109B10001E4608F041FF58B1284608F055FD10498F
:109B200008F0A6FD01464FF07E5008F055FE60603B
:109B30006168304608F094FC0146304608F04CFE5F
:109B4000256806462946384608F088FC0146304616
:109B500008F08EFD0146284608F082FC2060F8BD22
:109B6000DB0FC9402DE9F04102780346202A00F1BD
:109B70000100F9D0092AF7D02D2A02D10346414D20
:109B800004E02B2A08BF03464FF07E551C460026F2
:109B9000234614F8012BA2F13007F9B209290DD898
:109BA0003949304608F064FD0646384608F00CFD99
:109BB0000146304608F054FC0646E9E72E2A17D144
:109BC000314F234614F8010B3038C2B2092A0FD89E
:109BD00008F0FAFC394608F0FFFD0146304608F06F
:109BE0003FFC29490646384608F042FD0746E8E7AB
:109BF0001A7802F0DF02452A39D15A782D2A02D18B
:109C00000233012704E02B2A14BF0133023300275B
:109C1000013B002413F8012F303AD1B2092903D8AF
:109C20000A2101FB0424F5E7B4F59A7F28BF4FF41D
:109C30009A74A0464FF07E53B8F1070F07D9184623
:109C4000124908F015FDA8F108080346F4E704F0EE
:109C5000070434B118460C4908F00AFD013C0346DC
:109C6000F7E719462FB1304608F0B6FD04E04FF093
:109C70007E51304608F0FCFC0146284608F0F8FC0E
:109C8000BDE8F081000080BF0000204120BCBE4C38
:109C900030B5054687B00C4603A800210C220BF016
:109CA000AEFD2846002108F09FFE20B12846284935
:109CB00008F0D6FB03E02846254908F0CFFB2549EC
:109CC00008F0D6FC08F09AFE054680EAE070694686
:109CD000A0EBE57007F0AAFE002DACBF20232D23DA
:109CE00068468DF80C300BF0CEFD012807D13023EB
:109CF0008DF80D308DF80E308DF80F300CE0022805
:109D000005D130238DF80D308DF80E3004E0032896
:109D100004BF30238DF80D30694603A80BF096FD83
:109D200003A80BF0B0FD0338C5B22A4603A92046AC
:109D30000BF0D4FD00236355204607490BF086FD48
:109D400003AB204659190BF081FD204607B030BD0A
:109D50006F12033A00007A4480A0010870B50646ED
:109D6000B6FBF2F40846154614B12046FFF7F6FF9D
:109D700005FB1464024B1B5D00F8013B70BD00BF86
:109D800082A001082DE9F04F81468A4616461C46FE
:109D900089B000253178002900F0DB80252902D028
:109DA0000136484674E072784FF00008302A0CBF44
:109DB000B278B71CA2F1300312BF4FF0000BF71CB2
:109DC0004FF0010B092B19D8A2F13003D9B20929A0
:109DD00005D80A2202FB083817F8012BF4E7A2F194
:109DE0006103052B02D8A2F1570305E0A2F141035C
:109DF000052B03D8A2F137030A2BEADD6C2A30D1F8
:109E00003A787E1C642A00F083800BD8252A3DD046
:109E100003D8002A00F09D80BCE7582A0CD0632AA2
:109E200019D0B7E7732A22D002D86E2A37D0B1E70B
:109E3000752A5CD0782AADD1271D2068A2F158047C
:109E400062424FF01001624155E02CD9582A32D0BD
:109E5000632A2AD13E4648462178271DD04701353E
:109E60000FE0642A63D00ED9732A14D13E462368CA
:109E700048460093514642460023FFF712FE271D35
:109E800005443C4686E7252ADFD13E464846252143
:109E9000D04701357EE70AD86E2A06D13E462368B0
:109EA00004341D6076E7002A53D03E4672E7752AD7
:109EB00026D0782AF9D1A2F1580304F1040C5A42B1
:109EC0002068CDF80CC04FF010015A4105ABFFF7E8
:109ED00095FDDDF80CC03E46644605AB0093484650
:109EE000514642465B46FFF7DCFD054452E72068D9
:109EF000271D0A21002205ABFFF7A7FD3C46ECE732
:109F000004F1040CCDF80CC020680A210022DDE722
:109F10002068271D002808DA2D238DF814304042D0
:109F20000DF115030A210022E6E705ABFAE72068E8
:109F300004F1040C00280ADA2D238DF81430404275
:109F40000DF11503CDF80CC00A210022BFE705ABC7
:109F5000F8E7284609B0BDE8F08F0EB40FB505ABA1
:109F600053F8042B0190064901A80393FFF70AFF59
:109F7000019B00221A7004B05DF804EB03B0704737
:109F8000999A00080FB413B50B4904AB08680B4944
:109F900053F8042B09680193FFF7F4FE0446084BBD
:109FA000186801F043FA0028F9D0204602B0BDE855
:109FB000104004B0704700BFC4000020C000002063
:109FC000600E002080EAE073A3EBE0738B4206DBB7
:109FD000002801DD401A704702D008447047002075
:109FE00070472DE9F84321F0004520F00046074670
:109FF00088462846314608F0F7FC08B9344600E0A8
:10A000002C462046002108F0C7FC60B9284631469E
:10A0100008F0CCFC08B9304600E02846214608F09C
:10A02000DBFB044600E000242046254908F020FB25
:10A03000244908F013FA214608F01AFB224908F0D7
:10A040000DFA214608F014FB204908F007FA2146D2
:10A0500008F00EFB1E4908F001FA1E4900F1004904
:10A06000204608F005FB1C4908F0FAF9214608F0E3
:10A07000FFFA4FF07E5108F0F3F90146484608F028
:10A08000ABFB29460446304608F0AEFC20B1214621
:10A09000124808F0E3F904464046002108F086FC27
:10A0A00020B121460E4808F0D9F90446384600216F
:10A0B00008F07CFC08B104F100442046BDE8F883B8
:10A0C00039094E3DE3B59E3E88FA163E45FE7F3F78
:10A0D000A7DFA83499FB243F69A2163EDB0FC93FD6
:10A0E000DB0F494070B5044608F088FC203040285A
:10A0F00057D820462C4908F077FC28B120462B4938
:10A1000008F0ACF90446F4E72046294908F04EFC73
:10A1100028B12046254908F0A3F90446F4E7204673
:10A12000244908F061FC30B12249204608F096F934
:10A13000014620480AE020461F4908F037FC40B19C
:10A140001C49204608F08CF901461B4808F086F9A6
:10A1500004462146204608F08BFA0546204629464B
:10A1600008F086FA00210646284608F081FA1349CD
:10A1700008F074F90146284608F07AFA104908F008
:10A180006FF90146284608F073FA0E4908F066F99F
:10A190000146304608F06CFA0146204608F060F9A6
:10A1A00070BD002070BD00BFDB0F4940DB0FC94010
:10A1B000DB0F49C0DB0FC93FDB0FC9BF92E7413955
:10A1C0009730083C15A82A3E08B5034908F048F91D
:10A1D000BDE8084086E700BFDB0FC93F064B10B55E
:10A1E0001A881C4622EA00009042188002D0012002
:10A1F00001F0A2F8208810BD8C0E0020064B10B58F
:10A200001A881C4610439042188002D0012001F0A9
:10A2100093F8208810BD00BF8C0E0020024A93687E
:10A2200023EA000090607047FC27002008B5104B1F
:10A230001A780023D9B2914207D20E49002051F872
:10A240002310013309680880F4E7322001F009F88F
:10A25000094B1B685A0309D5084B9B685B0305D45F
:10A26000BDE8084040F2DC5000F0FBBF08BD00BF75
:10A270007C160020F8170020901B0020FC270020EF
:10A280002DE9F34102F094FE4B4A6F23137040F224
:10A29000E4735380BE231371EF2382F8E037002369
:10A2A0001946164682F8E137F25C0133514040F21C
:10A2B000E4729342F8D1404B404A83F8E117404B97
:10A2C00004275A6002F188325A600020013F17F0DB
:10A2D000FF075ED03A4B34223A4CDA6004F17848FA
:10A2E000A8F5FC38C8F3090353B100234FF400501C
:10A2F00056F80880019302F039FB0428E6D11CE0EF
:10A300004FF4302002F032FB0428DFD12C4D4FF403
:10A3100030202B6943F002032B616C612B6943F001
:10A3200040032B6102F022FB41F6FD732A690428E9
:10A3300003EA02032B61D8D0C8E7214D4FF4005047
:10A340002B6943F001032B611FFA88F3238002F08D
:10A350000DFB042813D1A31C0193019B4FEA18485D
:10A36000A3F800804FF4005002F000FB41F6FE73AA
:10A370002A69042803EA02032B6106D0A6E741F606
:10A38000FE732A6913402B61A0E70F4B04349C42F3
:10A39000A4D10B4A0428136943F08003136102D14E
:10A3A00006F0CDF810B9052000F0DEFF02F0ECFD5C
:10A3B00002B0BDE8F08100BFFC2700202301674503
:10A3C0000020024000F80108E4FF010810B50E4C1F
:10A3D0002068FFF795FA20680022047A02FB02F356
:10A3E000193B634303F6C4135343192193FBF1F361
:10A3F000064921F812300132072AEFD1BDE810409A
:10A400000349FFF735BA00BF0C0F0020300E0020C3
:10A410003C2900202DE9F04106F091F810B9042004
:10A4200000F0A2FFBC4C02F0C3FDBC4940F2E47254
:10A4300020460BF0D9F994F8B0374FF4CC71022BC9
:10A4400084BF002384F8B03794F8B027B44D01FBE3
:10A4500002F303F53A7020442344286093F848033C
:10A4600001FB0242022884BF002083F8480392F8CF
:10A470004833AC4A13700C2202FB0343AA4A03F28E
:10A48000B273136046F20902A3681A401AB9A24ACD
:10A4900043F400539360A368DF0703D54FF40050E3
:10A4A000FFF7BCFEA3685E0409D50820FFF7B6FEDF
:10A4B0004FF40050FFF7B2FE0120FFF7AFFEA36894
:10A4C000180706D54FF40050FFF7A8FE0120FFF74C
:10A4D000A5FEA368990413D54FF40040FFF79EFE34
:10A4E0008D4B93F88431012B03D14FF40060FFF7BB
:10A4F00095FE4FF48030FFF791FE4020FFF78EFE6F
:10A50000A3685A0603D54FF48030FFF787FEA3688F
:10A5100003F40852B2F5085F0AD11B0508D57E4B3B
:10A5200093F88431012B03D14FF40060FFF776FEDE
:10A5300094F8DE21784B2AB193F8E22112B100227F
:10A5400083F8E2214FF0000C6746784E784B1E608E
:10A5500004EB0C03B3F8F2E14FEA5E0101F077314E
:10A560004FEA9E0303F03333C1EB0E00C11A4FEAEA
:10A57000DE0303F01133CB1A03EB231303F00F3286
:10A58000FF2392FBF3F31EF00108C3EB032318BF74
:10A590000137A2EB030318BFFFB2012B0ADD022B28
:10A5A00040F0B780B8F1000F00F0B3801EF0BC0F90
:10A5B00000F0AF800CF1080CBCF1280FC8D1013FAE
:10A5C000012F00F2A680FFF701FF30220021594839
:10A5D0000BF015F9584F594BD5F800801F60584BB8
:10A5E000002108F18500C3F80080FFF7C7F9554B3B
:10A5F00080F001001870544B07F128021A60534B89
:10A6000007F1D8021A6098F8000005F075FB504B6E
:10A6100094F8D61107F196021A6064224A434D4B12
:10A62000C8325A6000229A60DA601A615A619A61EF
:10A63000DA6183F8202083F82120474B2D6807F149
:10A640002E021A60454B05F225121A60444B05F2A2
:10A6500095121A60434B07F108021A60424BDFF86B
:10A660003C811F60414B07F1A2021A6007F1AC0365
:10A67000C8F800303E4BB4F864011E6007F0A0FF3C
:10A68000C8F80800B4F8660107F09AFF95F868303A
:10A6900008F1040288F8043095F88430C8F80C00FA
:10A6A00088F8053094F8E131E86E88F81030314BC5
:10A6B000C8F814501A6005F17003C8F818302E4914
:10A6C00007F0D6FF01464FF07C5008F085F8B5F84A
:10A6D0002241C8F81C00204607F076FF01462748B3
:10A6E00008F07AF8264907F0C3FF264A264B156082
:10A6F000264A186005F174031360254A05F21D15FA
:10A700001560244A1760244ABDE8F041136002F046
:10A710003BBC07F0F9F956E7FC27002000F80108D8
:10A72000D40E0020302500200C0F002084290020AA
:10A730008C1B0020EC0D00203C290020200E002066
:10A74000240E00200A000020842300206C05002035
:10A75000F82F0020A01B0020EC230020F014002084
:10A76000F41700205C1700205417002080160020EA
:10A770005817002068240020DB0F49400000614486
:10A780004C3D0F440007002084070020F406002001
:10A79000740700207C070020EC050020281500200D
:10A7A00008B5FFF76DFDFFF735FEBDE80840012055
:10A7B00000F0C2BD2DE9F04F8DB00091814600211F
:10A7C0001546AB480C229846AA4F0BF018F800210A
:10A7D0001422A9480BF013F8A84B97F800B003F126
:10A7E0001802BBF1010F94BF1E461646A04C4FF055
:10A7F000000A51460C2284F820A084F821A004F11C
:10A8000024000AF0FCFF2320266300F02AFD7520B7
:10A8100001210DF10F02FAF7E5FBA0B1984B50466C
:10A82000A362984B0121E36204AA432384F82430F5
:10A83000FAF7D8FB9DF8103003F07E038DF8103046
:10A84000002844D14CE094F8343063BB8E4A8F4EDC
:10A8500093694FF4805B43F00803936110238DF8F4
:10A860001A303046032306A98DF81B30ADF818B016
:10A87000FBF751FF864AC6F810B0138823F0400357
:10A880001B041B0C1380138823F038031B041B0CC0
:10A8900043F00803138013889BB243F040031380F6
:10A8A000012384F834307520012106AAFAF75EF9F5
:10A8B0009DF81830702B56D1052384F8203043239F
:10A8C00084F82430734BA362734BE3624BE0682B34
:10A8D00006D1012384F820301D2384F8243042E07F
:10A8E0009DF80F3003F07E03682B8DF80F3035D1C3
:10A8F0000223062084F820300146A36A06AA98475E
:10A900009DF81D1001F001029DF81B1001F00101DE
:10A910004B0043EA82019DF8192002F001030B432A
:10A920000AD05BB2012B01D1002302E0022B0ED131
:10A93000012384F8213016E04D4B0C209B6A012145
:10A9400005AA98479DF8143013F00F0303D1032094
:10A9500000F00AFD07E0042BEAD1E5E7702B04BF05
:10A96000042384F8203094F820200020022A404B51
:10A9700084F835000BD14949D960494919614949E1
:10A9800099614949D961012183F835101FE0012AF5
:10A990000DD1464983F83520D96041490422196117
:10A9A000434959613F4999613F49D9610FE0043AF0
:10A9B000012A00F25C833F4ADA60394A1A61394A57
:10A9C0009A61394ADA61012283F8352007223A492F
:10A9D000D4F8C0308B4643F001030A70C4F8C0308D
:10A9E000364B00221A709A46B9F1080F00F2B48073
:10A9F000DFE809F00DB20D296E8C29A2A200B9F191
:10AA0000010F40F2B7804FF000098AF800903B78C0
:10AA1000012B18D800260CAB03F8186D53203146D3
:10AA20000122FAF7FDF970B19DF81830E52B0AD133
:10AA3000234B84F836602360224B636004238AF83A
:10AA4000003002238EE094F82020094B022A3FD1E7
:10AA50001D4A1A601D4A5A6093F82130002B0CBF22
:10AA60006F236E23237201238AF80030032379E0D9
:10AA700048150020253000205415002028820108A8
:10AA8000E54F00087152000800100240000C014020
:10AA9000003800406D4B0008994B0008894D0008B4
:10AAA000914900087549000890C1793DB94B0008EB
:10AAB0003D490008B94C0008400000202430002027
:10AAC0003153000899500008F54D0008D949000895
:10AAD0003B78012B1AD800220CAB03F8182D1C2050
:10AAE0000D210122FAF79CF980B19DF818302A2B2C
:10AAF00001D01A2B0AD1CF4A84F837302260CE4ACF
:10AB000002238AF80030626004232BE000210CABA2
:10AB100003F8181D18200122FAF782F960B19DF898
:10AB20001830FB2B08D1C54B2360C54B6360012354
:10AB30008AF80030052315E094F82030C14A043B20
:10AB4000012B3FF65CAFC04B1360C04B5360012339
:10AB50008AF80030082305E0B9F1010F0AD94FF057
:10AB600000093DE78BF80130D4F8C03043F0020310
:10AB7000C4F8C0303B78012B05D106F015FFB44B6B
:10AB80004FF400525A61042D00F2CC81DFE815F039
:10AB90000500D4016600050093010A2000F061FB66
:10ABA0007720A021012205ABFAF73AF9002855D009
:10ABB0001E2101227720FAF7D7FA4FF42F6000F018
:10ABC00045FB0025A5F160014FF00009C9B2022242
:10ABD00006AB77208DF818908DF81990FAF720F9C8
:10ABE0009DF819309DF8182043EA0222954B03F195
:10ABF00038016A520235102DE4D1B3F846104A46A6
:10AC000001F00F0E01F47F41A3F846104B460125D9
:10AC100022F001002044008F002818BF0025D6072D
:10AC200003D5C0B24340082002E083EA1023FAE7CC
:10AC30001E0448BF83F4C05301384FEA4303F7D1E1
:10AC40000132102AE4D141EA0E017E4AA4F84610EE
:10AC500025B9C3F303339E4500F0E88194F848908A
:10AC6000784DB9F1000F40F0FB81DFF8E4A106F068
:10AC70009BFE4FF4804B2826504605A9ADF814B032
:10AC80008DF81660FBF747FD4FF40052CAF810200C
:10AC90003046704900F0B2FB0E210220FBF726FD82
:10ACA0000822CDF818B006A84FF0010B8DF81D2032
:10ACB0008DF81C908DF81EB001F07CFF4FF0030C56
:10ACC00004A88DF811C0CDF804C08DF810608DF87F
:10ACD00012908DF813B006F0EDFD142000F0C1FACB
:10ACE000D02177205A4605ABFAF79AF8514600284A
:10ACF00000F0BE809DF81430DDF804C0552B85F8B7
:10AD00006330A5F86CC040F0B380D1215A4605AB42
:10AD10007720FAF785F89DF81430772003F00F02BA
:10AD20001B0985F8642085F86530162206ABAA2138
:10AD3000FAF776F89DF818209DF8193043EA0223B7
:10AD4000A5F84C309DF81A209DF81B3043EA0223E9
:10AD5000A5F84E309DF81C209DF81D3043EA0223D3
:10AD6000A5F850309DF81E209DF81F3043EA0223BD
:10AD7000A5F852309DF820209DF8213043EA0223A7
:10AD8000A5F854309DF822209DF8233043EA022391
:10AD9000A5F856309DF824209DF8253043EA02237B
:10ADA000A5F858309DF826209DF8273043EA022365
:10ADB000A5F85A309DF828209DF8293043EA02234F
:10ADC000A5F85C309DF82A209DF82B3043EA022339
:10ADD000A5F85E309DF82C209DF82D3043EA022323
:10ADE000A5F8603041F27073A5F8703046F678131C
:10ADF000A5F87230184B6B67184BAB67184BEB67B5
:10AE0000184BC5F88030184BC5F8843095F8483099
:10AE10004BB9FAF723FA42F6E06000F017FADAF8D5
:10AE20000830C3F38039114B83F80090012384F874
:10AE3000483015E17B520008F94F00080D53000817
:10AE40005350000848150020754D0008D9490008E6
:10AE500000100140194B00085D520008B14F000876
:10AE600039520008654F0008614800082C00002096
:10AE7000804A136823F48043136000237E48DA007D
:10AE800000F1880505EB020EDEF804C0DFF838E2B9
:10AE9000F4450AD115F93350282D06D18318002224
:10AEA000C3F88C2083F8882002E00133032BE5D11E
:10AEB0004FF400534B6194F8A0906F4DB9F1000F1F
:10AEC00040F0C880142000F0CCF905F1A1037620F1
:10AED000D0210122F9F7A4FF95F8A130582B2BD1EE
:10AEE00005F1A403882118227620F9F799FF76202E
:10AEF000F4213122FAF738F9012385F8A0305F4BAD
:10AF0000A5F87090AB675E4B6B6745F6D813A5F854
:10AF100072305C4BEB675C4BC5F880305B4BC5F81F
:10AF2000843097E0012D07D0594B9D70D4F8C03084
:10AF300043F00403C4F8C030D4F8C0309A0702D5F7
:10AF40004D4B1B689847002384F8C4304FF47A7344
:10AF5000C4F8C830BC20E36898474E4B97F800907F
:10AF600003F11802B9F1010F94BF99469146009E72
:10AF7000494F00233B700EB1022E6DD100250CAB62
:10AF800003F8185D1E200A210122DFF8ECA0C4F8A6
:10AF9000CC90F9F745FFA8B19DF81830482B61D146
:10AFA0003E4B0222CAF8D0303D4BCAF8D4300323BE
:10AFB0003B70374BDA70D4F8C03043F00803C4F864
:10AFC000C03001E005464DE0364B93F855210AB1FB
:10AFD00084F8352093F856210AB133490A7093F862
:10AFE000573103B13B70D4F8C030234D1B0718D53F
:10AFF000642698FBF6F4204607F0E6FA074606FBBF
:10B00000148000B207F0E0FA284907F031FB01464E
:10B01000384607F025FA264907F02AFBC5F8D8007C
:10B0200002E00023C5F8D830012020E042F210737E
:10B03000A2F87030A2F872301E4B032553671E4BE6
:10B0400093671E4BD3671E4BC2F880301D4BC2F86E
:10B05000843069E7042567E7012EB5D91E4687E7E6
:10B06000022561E7012EAFD900263D7086E70DB0BD
:10B07000BDE8F08F00040140481500205D4800083D
:10B080005F48000831520008194F00089D4600082B
:10B09000400000205882010826300020B56C0008CE
:10B0A0001D6C0008FC270020243000208988883C83
:10B0B0000000204129520008094F000821520008D1
:10B0C000F94E0008E1440008194B00080120002156
:10B0D00005F09EBF174AF0B5164692F8DC30D2F85C
:10B0E000E0E0042B10D85C1C0EEBC3039D1CE4B203
:10B0F00008D09A88D10705D5104203D008E0013165
:10B10000052907D12346ECE786F8DC300020F0BDA6
:10B110009F7800210C2202FB01F3064D05F1E40C9F
:10B120001CF803209742EAD12B4485F8DC40D3F881
:10B13000E800F0BD481500200023036043608360F1
:10B14000C360036143618361C361036243628362DD
:10B1500070478A6810B50C6A036814430A6923F4BF
:10B16000FF4314434A6923F0700314438A6914436C
:10B17000CA6914434A6A14438A6A22431343036028
:10B18000CB6843600B6883604B68C36010BD00BF31
:10B19000034B4FF4805208B11A6170475A617047EF
:10B1A00000080140034B4FF4805208B15A617047C8
:10B1B0001A61704700080140094B1A680E2303FB0F
:10B1C0000020437AFF2B07D0064A12789A4203D90F
:10B1D000054A32F8130000E0808800B2704700BFD3
:10B1E000F0140020E42F00203E2700201FB5084B5C
:10B1F0001B681B0309D58DF80400029100230D2064
:10B2000001A98DF80530FCF7D5FA05B05DF804FB0F
:10B21000901B002010B50A4A0A4B11689B6800BFBA
:10B2200012689142F7D1084A4FF47A70146800FB13
:10B2300004F2D31AB3FBF4F300FB013010BD00BFDE
:10B240009C1B002010E000E06816002038B5044682
:10B25000FFF7E0FF0546FFF7DDFF401BA042FAD3F2
:10B2600038BD10B504462CB14FF47A70FFF7EEFFED
:10B27000013CF8E710BD024A1368013313607047C0
:10B280009C1B002010B50024054AA3185B681BB165
:10B29000A256282A00D198470834182CF4D110BDA2
:10B2A000D0150020014B1B68184700BF0C30002050
:10B2B00010B50020FFF7F6FF054B00241C7001F0CD
:10B2C0008DFE044B1C719C609C811C6110BD00BFF5
:10B2D000C41B00206816002010B5E0B1124B1B689B
:10B2E00013F0020304D0114B1B78012B13D9002358
:10B2F0000C225A430E4C1119125D824203D00133C5
:10B30000102BF5D110BD0B4B186938B14A78407835
:10B31000824203D310BDBDE81040C9E70022196185
:10B320009A819A6010BD00BF901B00204800002049
:10B33000E88301086816002010B540001428A8BF53
:10B3400014200023074A022199540B44991814240D
:10B35000834201F8014CF5DBFF21D1540F20BDE8F9
:10B360001040B9E7592500202DE9F84381460B2606
:10B37000013E37D01E4B10225A6108221A6109F192
:10B3800001074FF032080525194C0120E36883F0CE
:10B390001003E360E36883F00803E360FFF782FFD4
:10B3A0004046FFF75EFFE368002083F01003E36090
:10B3B000E36883F00803E360FFF774FF4046FFF79C
:10B3C00050FF45B1013DDFD14FF4FA70FFF749FF5F
:10B3D0004FF0FA08D8E7013FD6D14FF47A70FFF763
:10B3E00040FFC5E7034A044BDA60BDE8F88300BFBD
:10B3F000000C01400400FA0500ED00E00A4B10B516
:10B400005A6832B1DA681AB15A6942B9022200E0C8
:10B41000012203EBC204616003F8320010BD00207A
:10B42000BDE81040A0E700BFD015002003685B69AD
:10B4300018470368DB68184703685B6818470368A8
:10B440001B681847B0F902302DE9F74F93421CBF33
:10B450000023037090F800A004460E469146BAF10E
:10B46000000F40F0B480104607F0AEF88A4907F0AC
:10B47000FFF88A4907F0FCF84FF07C5107F0F8F824
:10B480000746FEF72FFE05463846FEF79DFE0146AD
:10B49000284607F0A1F90146054607F0E9F880497A
:10B4A0008346284607F0E4F80346584619460193B8
:10B4B00006F0D6FF4FF07E5106F0D2FF01464FF066
:10B4C0007E5007F089F92946804607F0D1F82946D1
:10B4D00007F0CEF807460146606006F0C1FFE7605E
:10B4E0004FF07E572946A0602761284606F0B8FF36
:10B4F000294607F0BDF84FF0804106F0AFFF014646
:10B50000404607F0B5F8019B60611946584606F0C1
:10B51000A5FF394606F0A4FF0146404607F0A8F80B
:10B5200040F2DC53A0462746554663651023A4F835
:10B5300052301823A061A4F850304FF09741D8F84A
:10B54000100007F095F80021824607F02FFA28B185
:10B5500050464FF07C5106F081FF04E050464FF01A
:10B560007C5106F07DFF07F0ABFAC7E90E014FF002
:10B570009741D8F8040007F07BF80021824607F0D5
:10B5800015FA28B150464FF07C5106F067FF04E0F1
:10B5900050464FF07C5106F063FF07F091FA0135F9
:10B5A000032DC7E9080108F1040807F10807C4D111
:10B5B000A6F2DC531B042367E3676367C4F880309B
:10B5C000A367C4F884300123A4F802902370D4F850
:10B5D0005490B4F95280C9EB0606636A06FA08F67D
:10B5E0007343276A4FEAE67B206F07FB0B3326671E
:10B5F000A7FB0667E26F1F44636CD4F840C0534357
:10B600004FEAE27B0CFB0B3ED4F88010C4F880209C
:10B61000ACFB02237344B61A67EB0307E36AA26A22
:10B6200043434FEAE07B02FB0B3EA2FB0023734443
:10B63000B6185F41E36C656F4B436067A06C4FEADF
:10B64000E17B00FB0B33C4F88410A0FB010119441B
:10B65000636B361A05FB03F3206B4FEAE57B00FBB7
:10B660000B3367EB0107A0FB0501801919447941F1
:10B67000B4F95020A56706F0D7FC08F1FF3201238A
:10B680009340E067C01841EBE371424606F0CCFC02
:10B69000484403B0BDE8F08F6F12833ADB0F494096
:10B6A000F404B53F2DE9F04F904C8DB0257D032D6E
:10B6B00014D9A3695888B0F5FA7F0FD2B4F92610CF
:10B6C000B4F920600029B8BF49424242531A9E4251
:10B6D00003DB4318B342A8BF33462384A369B4F8FD
:10B6E00028A0B4F81E80B4F81C90B4F920B0804EA5
:10B6F00001930027AF4206F110063CD20FFA8AF000
:10B7000006F062FF56F8181C06F0B2FF02900FFA1E
:10B7100088F006F059FF56F8101C06F0A9FF029AAF
:10B720000146104606F09CFE02900FFA89F006F0E2
:10B730004BFF56F8141C06F09BFF029A0146104678
:10B7400006F08EFE019B029093F9010040420BFB34
:10B7500000F006F039FF56F80C1C06F089FF029A3B
:10B760000146104606F07CFE07F048F9614A22F8CF
:10B7700017000137BEE7604B1A7802F0040202F0AE
:10B78000FF03002A00F091805C4B0120DB780293DC
:10B79000584B1A88A84216B207D233F9102001304C
:10B7A0009642B8BF1646B2B2F4E7D4F8EC00D4F82B
:10B7B00018904188D4F8F0C08E42C6BF511A8AB2A0
:10B7C000002201924E4A4F4E1268B6F9066002F40A
:10B7D000805A02F010020392D4F8F470454A03EB49
:10B7E000450E724557D0138801995B1A9BB222F817
:10B7F000023BBAF1000F25D099F800504DB9BCF8C2
:10B800000E80FD88C5EB080B5E4502DD4544AE4267
:10B8100013DBBCF80E501BB2AE42CBBF7D888588CF
:10B82000B0F80280B7F80080AB4203DB4345A8BF05
:10B8300043461D4622F8025CD3E74645CCBF7B88D1
:10B840003B8825E0029945881BB251B1B0F80480CD
:10B85000434503DBAB42A8BF2B46984622F8028C37
:10B86000BFE7B0F80080434503DBAB42A8BF2B46DF
:10B87000984622F8028CBCF810309E42B1DA039B45
:10B880000BB1838804E099F80030002BA9D103881C
:10B8900022F8023CA5E794F8F830144A013BDBB2E9
:10B8A000182B194F00F23A8109E0AB42F3D2174A44
:10B8B00032F813100F4A22F813100133F5E7012173
:10B8C0009940134B0B40002B00F02881114B1B8833
:10B8D00013F4807F0B4B1FD0518CADF81410918C5A
:10B8E000D28CADF81610ADF818202CE068160020A8
:10B8F0009C160020D80E002021300020A01B002024
:10B90000901B00203E270020C20E00203225002080
:10B91000992098018C0E0020918BB548ADF8141039
:10B92000D18B0068ADF81610118CC004ADF818105A
:10B9300009D5D2F8F020B3F90600D2899042BCBFF5
:10B940004942ADF81810AB4D4FF47A71B5F90220A9
:10B950004FF4616002F5E1624A4392FBF0F2A2F516
:10B96000FA72ADF82C20B5F9002002F5E1625143DE
:10B9700091FBF0F1A04AA1F5FA711288ADF82E10F2
:10B98000A2F2DC52ADF81A20D4F8F0201988D2893E
:10B99000891AADF81C105988891AADF81E109988BB
:10B9A000891AADF82010D988891AADF822101989A2
:10B9B000891AADF824105989891AADF82610998989
:10B9C000DB89891A9A1AADF82810ADF82A200023CD
:10B9D000002227F813200133082BF9D1874B884820
:10B9E0001B6800F126010193864B1B68029394F8B3
:10B9F0008A31C3EBC303034403F1260A514574D0D3
:10BA00000B7833B103F1150201239340019A1340DF
:10BA100067D0029B11F806CC4FF00E0E0EFB0C3EC9
:10BA2000BEF90020BEF9023064249B1A11F9022CE1
:10BA30009BB25A4392FBF4F211F805BC4FEA53094A
:10BA400011F8035CC9EB02024FEA4B060CAC92B250
:10BA500011F8018C264415B936F81C4C0CE0B0F9ED
:10BA6000004036F91C6CB44208DA2544A54203DBD9
:10BA7000AE423446A8BF2C46048008E007DD651BB3
:10BA8000B54203DBA542A8BF25462E460680DEF858
:10BA90000A50012404FA0BF42C42B0F9006011F9A9
:10BAA000044C12B204FB06F44FF0640694FBF6F467
:10BAB00014BF4FF0FF35012594420ADB4FFA88F29C
:10BAC0005A4392FBF6F2C9EB020212B2A242A8BF9D
:10BAD00022464D4B33F81C9002FB059523F81C5071
:10BAE00000E003800230073188E7464B474ED3F829
:10BAF000008000250E2303FB058393F9064036F9E9
:10BB0000023FE8B26343642493FBF4F43480FFF70C
:10BB100053FB01352044082D3080EBD1344B394D97
:10BB20001B6813F0200F32D00020FFF745FB388050
:10BB300006460120FFF740FB304B334C1B687880F2
:10BB40001B0624D5324B2B4AD3F88C311B78012BA2
:10BB500020D1D5F800C0B2F900309CF91410B2F928
:10BB6000022059439CF906304FF0320E5B4253439A
:10BB700091FBFEF16FF0310293FBF2F293FBFEF3C7
:10BB800089B20A4432440B442280184460802D68F4
:10BB9000002315E0D5F800E0B2F902309EF9061056
:10BBA0005943322391FBF3F1314421809EF9146013
:10BBB000B2F9001001FB06F292FBF3F21044E5E744
:10BBC0000E2101FB035137F91300B1F900205C008D
:10BBD0009042B1F9021003DB0AB28242A8BF0246CA
:10BBE0000133082B3A53EBD10DB0BDE8F08F00BF05
:10BBF000901B0020F00E0020D80E0020900E002098
:10BC000062170020F0140020C20E0020C00E002099
:10BC1000681600202DE9F8430024244BE0B21E7D75
:10BC2000B0420DD203EB8003214AD3F8903132F8B1
:10BC300010101BB10B2801D8DB6898470134ECE7E2
:10BC40001C4B1B685B032FD500242346E2B2B24293
:10BC50002AD2DFF858904FEA840809F5C87757F8D8
:10BC6000242055689D4217D0284602F077F9EFF35B
:10BC70001283502282F312882821AA8C01FB0090A3
:10BC800092B20132C0F8E421AA8ADBB292B242F049
:10BC90000102AA8283F3118857F8083000221B683A
:10BCA00001341A802B46D1E7BDE8F88368160020DE
:10BCB000D80E0020901B002008B50E4B1B6813F413
:10BCC000805F0D4B14BFD3F8F420D3F8EC20197D1E
:10BCD00092880023D8B2884204D2084820F8132062
:10BCE0000133F7E7FFF796FFBDE808403220FFF782
:10BCF000B8BA00BF901B002068160020D80E0020A4
:10BD00000A4B30B51A680A4B02F48052D3F8F4405B
:10BD1000D3F8EC5000230AB1A18800E0A9880548B7
:10BD200020F8131001330C2BF5D130BD901B0020EF
:10BD3000681600203225002070B5124D00242146DF
:10BD400005F58D70702285F88A4109F058FD21466D
:10BD5000D5F860320B4A0B4493F9020088B11E6893
:10BD600002F58D740E5108199C88073184809B79E7
:10BD70007029837192F88A3103F1010382F88A31C4
:10BD8000E6D170BD681600202DE9F84F4668D1F85D
:10BD900008A0D0F808904F680D68D0F80080514690
:10BDA0003046144606F064FC39468346484606F0A1
:10BDB0005FFC0146584606F051FB29462060484684
:10BDC00006F056FC51468146404606F051FC0146BD
:10BDD000484606F043FB39466060404606F048FCA2
:10BDE00029460746304606F043FC0146384606F031
:10BDF00035FBA060BDE8F88F2DE9F04106460D4601
:10BE000040684968144606F02BFBA9688046B06874
:10BE100006F026FB29680746306806F021FBC4F8C7
:10BE200004802060A760BDE8F0812DE9F04106465E
:10BE30000D4608467168144606F01AFCB168804643
:10BE4000284606F015FC29460746306806F010FC27
:10BE5000C4F804802060A760BDE8F08108B50748F9
:10BE600009F011FDC0B21428044B04D8421C202153
:10BE70001954D0B2F7E700221A5408BD95240020C7
:10BE80002DE9F74FFFF7C6F9A64C8046266865688E
:10BE9000A768861BF643451BC71BED43FF43F60F00
:10BEA000ED0FFF0F2EB93FB9002D00F08782B94684
:10BEB0002CE04FF0000929E0B14627E003EB8A0BA4
:10BEC000BBF802301A050ED413F4805F1DBF964AEA
:10BED0009BF801101268954A954B14BF52F8212027
:10BEE000126843F82A20BBF80230D80516D4990509
:10BEF0000AD5904B1B7813F0040F0CBF8E4A8F4A63
:10BF00008B4B126843F82A2009F10109207B5FFA64
:10BF100089FA8B4982450B68D0D326E0894A50467E
:10BF2000594601F04FFC884B1B885A0603D55046F2
:10BF30005946864A16E0580703D550465946844A62
:10BF400010E0190703D550465946824A0AE09A077D
:10BF500003D550465946804A04E0DB07D4D5504605
:10BF600059467E4A01F02EFCCEE7DFF808E2009346
:10BF7000BEF906307822A3F57A7353434FF47A72F0
:10BF800093FBF2F3F34603F22B13019300225FFAC3
:10BF900082FE864517D2009B03EB820EBEF802E0BC
:10BFA0001EF4806F0DD040F2671ADFF88491019B78
:10BFB00039F822E09E449EFBFAFC0AFB1CEE29F8AD
:10BFC00022E00132E3E74DB308F5C333A0336360E9
:10BFD000637B544A13BB9373614B1B6813F0020FCE
:10BFE0000AD0DFF894E19EF800E0BEF1000F03D024
:10BFF0004FF0010E82F80EE0DA0506D5594BDB78DA
:10C000001BB1A37B43F00203A3734A4B1B7813F0CD
:10C01000050F02BFA37B43F00403A37394F80EE063
:10C02000BEF1000F03D13F4B5B7B002B4FD094F848
:10C030000DC01CF0010FACF10C031DD1BCF1030FBE
:10C0400007D8DFF8E8901EF0040F3B4A08BF4A46C5
:10C0500000E0364AACF1040CBCF1070F05D8DFF85C
:10C060001CC11EF0010F18BF6246DBB2032B0ED8B5
:10C070001EF0020F3C4B06E0DBB2032B06D82F4B21
:10C080002A4A1EF0020F18BF1A4600E0274A4FF056
:10C09000000C5FFA8CF383420DD20B6803EB8C0328
:10C0A0005B881B0642BFD2F80090214B43F82C90CE
:10C0B0000CF1010CEDE785B1BEF1000F08D0637BF8
:10C0C000184A0133DBB2142B06D1002304E025B15A
:10C0D000637B002BF3D100E05373002E52D0234A30
:10C0E0003223B2F90250B2F90020002DB8BF6D42E0
:10C0F000002AB8BF524295FBF3F592FBF3F2EDB282
:10C10000D3B2AB4238BF2B46194A13B192FBF3F3BB
:10C1100000E0134643442360E37B024A83BB0123D0
:10C120002FE000BFCC180020E8140020C4920108C2
:10C13000540C002021300020D4830108C48301085E
:10C14000EC140020888201088C0E00208E820108E9
:10C15000948201089A820108A0820108A68201083F
:10C16000901B0020A01B0020DC8301088A16002001
:10C17000400D03003E27002058250020E4830108DD
:10C180000023D3738F4D904B2D78E27BADB9002FF8
:10C1900000F00F818D4B267B1A788D4B02F0040244
:10C1A00093F800C08B4BD2B2D3F800E00B680021AB
:10C1B000894D03EB86060F46B5E01AB9874A1A6126
:10C1C000002508E0864AFAE70A68AB00D6187688A8
:10C1D000760604D40135EBB28342F5D3D7E7814E1E
:10C1E000B6F90060192E25DD12F803E094F814C0AA
:10C1F0000EF00F09E14526690CDCDFF8CCC19CF894
:10C2000015C0BCEB1E1FDEBFD6F800C0DFF8D8E1BA
:10C2100043F80EC012F803E094F816C00EF00F09B0
:10C22000E14533DBDFF8A0C19CF815C0BCEB1E1F55
:10C230002CDC26E0193629DA12F803E094F814C051
:10C240000EF00F09E14526690CDCDFF87CC19CF893
:10C2500017C0BCEB1E1FA2BFD6F800C0DFF888E1F4
:10C2600043F80EC012F803E094F816C00EF00F0960
:10C27000E1450BDBDFF850C19CF817C0BCEB1E1F7B
:10C2800004DBD6F800E0584E43F806E0554EB6F908
:10C290000260192E1BDD12F803C094F814E00CF0B4
:10C2A0000F09F14526690CDCDFF81C9199F815900F
:10C2B000B9EB1C1FDEBFD6F80090DFF82CC143F8A5
:10C2C0000C90D25C02F00F0CF4451EDD82E71936AB
:10C2D00080DA12F803C094F816E00CF00F09F1456B
:10C2E00026690CDBDFF8E09099F81590B9EB1C1F7C
:10C2F000DEBFD6F80090DFF8F0C043F80C90D25CB7
:10C3000002F00F0CF445FFF665AF94F817E0BEEBB2
:10C31000121FA2BF3668344A9E505BE7588800055A
:10C3200004D404330435B342F8D122E04AB101EB1E
:10C330000C0A06209AFBF0F900FB19A001280DDC7D
:10C3400001E057B9012793F801900EEB89003EF800
:10C3500029A090F80290C07803E01746002081469B
:10C360008246013125F802AC85F800906870C9B2A8
:10C37000D7E7174A1378013B13F0FF0308BF0623E2
:10C380001370124B1B785B0741BFBBF906304FF4AB
:10C390007A72A3F57A7303EBC30348BF93FBF2F3FE
:10C3A000124A46BF0133DBB2012392FBF3F343444D
:10C3B000A36003B0BDE8F04FFAF7BAB803B0BDE828
:10C3C000F08F00BF080D0020CC1800202130002085
:10C3D0002D000020E8140020560C0020E083010806
:10C3E000C49201088A160020540C0020400D03005E
:10C3F000084BDA68D10709D4DA68520708D4DB6839
:10C4000013F0100F14BF0320042070470120704761
:10C41000022070470020024003788B4286BF024B07
:10C4200033F8110000207047E8180020002213465E
:10C4300070B5234914180C44247E83EA042308248D
:10C4400013F4004F4FEA430318BF83F4815304F100
:10C45000FF3418BF83F0010314F0FF049BB2EFD147
:10C460000132192AE5D100F1190200F11A050A4436
:10C470000D44167E2A7E02EB062292B29A421ED10B
:10C480000F4B93F83950E2B2AA4215D2431C03EB8A
:10C490004203DBB2CA1801330B44127E1B7E03EB4E
:10C4A00002239BB24FF4AF6253431B1303F548734F
:10C4B00021F814300134E6E7012381F83A3070BDE9
:10C4C000E818002003788B420BD9074B89001A78B3
:10C4D000064B1944C86B02B1400800F5777080B272
:10C4E00070470020704700BFE82F0020E8180020A8
:10C4F00007299DBF034B03EB8101B1F86C000020BD
:10C50000704700BFE8180020034B03EB4101B1F86E
:10C510008C00C008704700BFE818002008B5084B21
:10C5200003EB8101D1F8AC0006F04AF8054906F0AA
:10C530009FF8054905F094FF06F086FA80B208BD21
:10C54000E81800200000203F00005C44024B03EB91
:10C550004101B1F8F4007047E8180020024B03EBEA
:10C560004101B1F818017047E8180020024B03EBB5
:10C570004101B1F818017047E81800200020704709
:10C5800070B50546FEF746FE314CD4F83031C4F89C
:10C590003001C31AB3F5FA5FC4F8343182BF002307
:10C5A00084F8383184F8393194F838312BB9A12D19
:10C5B00002BF274A012182F8391194F83911244A1F
:10C5C00029B1D118EDB201330D7682F8383194F8E3
:10C5D000385194F83A31AB4239D11D4B93F83B3185
:10C5E000052B02D0062B03D02CE00020FFF71EFF06
:10C5F000637E1E2B26D100200246C1B26B1E9942DB
:10C6000019DA21440B7E0821DBB283EA0206F60721
:10C6100044BF83F01803C3F3460301F1FF3154BF55
:10C620005B0843F0800311F0FF01C2F34702ECD135
:10C6300001301A46E1E723441B7E9A4202D10320CF
:10C64000FFF7F4FE002384F8393184F8383170BDE7
:10C65000E818002010B50446FEF7DCFD41F28831F1
:10C660000E4BE4B2D3F83C21C3F83C01821A8A4253
:10C67000C3F8402184BF002283F8442193F8442169
:10C6800006490F2A134418BF013283F8454112BFEF
:10C6900081F84421012381F8553110BDE8180020AC
:10C6A00010B50446FEF7B6FD41F288310E4BD3F8C3
:10C6B0005821C3F85801821A8A42C3F85C2184BF0A
:10C6C000002283F8602193F860210749142A13445B
:10C6D00018BF013283F8614112BF81F86021012344
:10C6E00081F8763110BD00BFE818002038B5044647
:10C6F000FEF790FD274A2749D2F87831C2F8780131
:10C70000C31AB3F57A6F84BF002382F87C3192F8A4
:10C710007C3133B9A82C3BD181F87D31A1F87E3131
:10C7200006E0022B02D181F8804101E0242B02D8DF
:10C73000D11881F8814192F8801101330231DBB2C6
:10C7400049008B42134D82F87C3118DAB5F87E31FE
:10C75000E0B283EA0020082310F4004F4FEA4000C3
:10C7600018BF80F4815003F1FF3318BF80F001003F
:10C7700013F0FF0380B2EFD1A2F87E0138BD013182
:10C780008B4201BF002385F87C31012385F87D3180
:10C7900038BD00BFE818002010B50446FEF73AFD8A
:10C7A00040F6AC510F4AD2F8A831C31A8B42C4BF2D
:10C7B000002382F8AC3192F8AC31D11881F8AD4148
:10C7C00023B90F2C0DD10749C1F8A8010133DBB201
:10C7D000192B044982F8AC310CBF0123002381F8E6
:10C7E000C63110BDE81800204FF6FE7302681340F2
:10C7F00003600023036043608360C360284B98425A
:10C8000001D1284A27E0284B984201D1254A2AE045
:10C81000264B984201D1234A2DE0254B984201D165
:10C82000204A30E0234B984201D11E4A33E0224B8C
:10C83000984204D11B4A536843F470032EE01F4B07
:10C84000984204D1174A536843F0706326E01C4BAA
:10C85000984204D11B4A536843F00F031EE01A4B61
:10C86000984204D1174A536843F0F00316E0174B7F
:10C87000984204D1134A536843F470630EE0144B9A
:10C88000984204D10F4A536843F4704306E0114BB9
:10C89000984204D10B4A536843F4702353607047A5
:10C8A00008000240000002401C000240300002402C
:10C8B00044000240580002406C00024080000240E8
:10C8C00008040240000402401C04024030040240FC
:10C8D00044040240580402401F4A10B5536803F054
:10C8E0000C03042B03D0082B04D01C4B14E01C4B6E
:10C8F0001B6811E053685168C3F38343C90303F114
:10C90000020301D4174906E0516811F4003F1449AD
:10C91000096818BF49084B43036053681249C3F3C1
:10C920000313CC5C0368E34043605468C4F30224FF
:10C930000C5D23FA04F484605468C4F3C2240C5DD3
:10C94000E340C3605268C2F381320A44127CB3FBF5
:10C95000F2F3036110BD00BF0010024000127A0024
:10C960003000002000093D00AC82010810B50446EB
:10C97000FFF73EFD012806D11CB1FFF739FD013C50
:10C98000F8E7052010BD002C08BF052010BD0A885F
:10C99000F0B54B888E88B1F808E0CC88002A3AD1EF
:10C9A000028C43F0010322F001021204120C0284F3
:10C9B000058B078CADB225F0F30545EA0E1189B25F
:10C9C00041EA06027A49BFB2884212D001F50061FD
:10C9D00088420ED0B0F1804F0BD0A1F5983188423B
:10C9E00007D001F58061884203D001F5806188425B
:10C9F00002D127F0020701E027F00A071F43028354
:10CA00000784038B23F00C031B041B0C0383038B91
:10CA10009BB21C4344E0042A44D1028C22F0100251
:10CA20001204120C0284018B058C21F44072120551
:10CA3000120D42EA0E325E4992B242EA0622884262
:10CA4000ADB292B212D001F5006188420ED0B0F1C1
:10CA5000804F0BD0A1F59831884207D001F5806155
:10CA6000884203D001F58061884207D125F020017A
:10CA700041EA03139BB243F0100304E025F0A00148
:10CA800043F010030B4302830384038B23F44063BE
:10CA90001B041B0C0383038B9BB243EA0424A4B244
:10CAA0000483F0BD082A028C3ED122F48072120465
:10CAB000120C0284828B3E4D92B222F0F307018C5D
:10CAC00047EA0E1292B2A84289B242EA060212D096
:10CAD00005F50065A8420ED0B0F1804F0BD0A5F54A
:10CAE0009835A84207D005F58065A84203D005F522
:10CAF0008065A84207D121F4007141EA03239BB26B
:10CB000043F4807304E021F4206143F480730B4309
:10CB100082830384838B23F00C031B041B0C83830D
:10CB2000838B9BB21C4341E022F480521204120C0E
:10CB30000284858B018C25F440752D052D0D45EA69
:10CB4000062545EA0E321A4D89B2A84292B212D099
:10CB500005F50065A8420ED0B0F1804F0BD0A5F5C9
:10CB60009835A84207D005F58065A84203D005F5A1
:10CB70008065A84207D121F4005141EA03339BB2FA
:10CB800043F4805305E047F6FF5543F480530D40CE
:10CB90002B4382830384838B23F440631B041B0C8D
:10CBA0008383838B9BB243EA0424A4B28483F0BDC5
:10CBB000002C0140016830B5CD43154B1C682C405A
:10CBC0001C605A682A405A60027902F1804202F5DC
:10CBD000823214682143116002689C68D5432C405E
:10CBE0009C60D9682940D9604179102909BF9968AA
:10CBF00001F180431143996015BF03F58233D96871
:10CC000019680A4316BF0A43DA601A6030BD00BFD4
:10CC100000040140054B1A685B69034004D01042D0
:10CC200014BF0120002070471846704700040140DF
:10CC3000CA78F0B5D40648BF8C780D8802F00F038F
:10CC400048BF234315F0FF0F1DD0016800240126C3
:10CC5000A64006EA0507B74211D14FEA840E0F2617
:10CC600006FA0EF621EA0601282A03FA0EF641EA30
:10CC7000060101D1476102E0482A08BF076101347B
:10CC8000082CE4D10160FF2D1FD94168002404F174
:10CC900008070126BE4006EA0507B74211D14FEA50
:10CCA000840E0F2606FA0EF621EA0601282A03FA58
:10CCB0000EF641EA060101D1476102E0482A08BFA9
:10CCC00007610134082CE2D14160F0BD0F4B1A68B6
:10CCD00042F001021A6059680D4A0A405A601A6807
:10CCE00022F0847222F480321A601A6822F48022C0
:10CCF0001A605A6822F4FE025A604FF41F029A60CA
:10CD0000044B4FF000629A60704700BF0010024071
:10CD10000000FFF800ED00E02DE9F8435B4C0368EC
:10CD2000023AC4F8C83183880D46A4F8CC31062AEB
:10CD300005D8DFE802F00A101822292F3500B4F8D0
:10CD4000C8310B80B4F8CA3113E0B4F8CA310B8093
:10CD5000B4F8C83105E0B4F8C8315B420B80B4F8D0
:10CD6000CA315B4205E0B4F8CA315B420B80B4F8CB
:10CD7000C8316B80B4F8CC311DE0B4F8C8315B42E7
:10CD80000B80B4F8CA3112E0B4F8CA310B80B4F8A1
:10CD9000C8310CE0B4F8C8310B80B4F8CA3105E0F2
:10CDA000B4F8CA315B420B80B4F8C8315B426B8087
:10CDB000B4F8CC315B42AB80354B1B79002B62D190
:10CDC000B5F9000005F000FC8046B5F9020005F059
:10CDD000FBFB0746B5F9040005F0F6FBD4F8D011CB
:10CDE0000646404605F044FCD4F8DC11814638463E
:10CDF00005F03EFC0146484605F032FBD4F8E81148
:10CE00008146304605F034FC0146484605F028FBD3
:10CE100008F002FFD4F8D4112880404605F028FC21
:10CE2000D4F8E0118146384605F022FC0146484618
:10CE300005F016FBD4F8EC118146304605F018FCDD
:10CE40000146484605F00CFB08F0E6FED4F8D81180
:10CE50006880404605F00CFCD4F8E4118046384662
:10CE600005F006FC0146404605F0FAFAD4F8F01148
:10CE70000746304605F0FCFB0146384605F0F0FA5F
:10CE800008F0CAFEA880BDE8F88300BFE8180020BB
:10CE90003000002038B50F4BD3F8F421D3F8F80157
:10CEA000948980F31000201A05F08EFB0A4905F0E2
:10CEB000DFFB0546204605F087FB0146284605F0C6
:10CEC0008BFC05F09BFD6428A8BF642020EAE0707D
:10CED000C0B238BDE81800200000C84244F6FB711B
:10CEE000084BD3F8F421137803EB431300FB03132F
:10CEF0005078C0EB0030B3FBF0F39078B3FBF0F068
:10CF000080B27047E818002010B50A4C0A2294F845
:10CF1000FD3104F5067004EB4303B3F80C1289B23B
:10CF2000A4F81412FEF78EFA80B2FFF7D7FFA4F828
:10CF3000A00210BDE818002010B51149D1F8A432A4
:10CF400003EB4002147E14B1022C10D00BE0022837
:10CF500005D9032807D1D1F8A822D20401D5D88950
:10CF600010BD988A10BD074B33F8100010BD507EDD
:10CF700000EB800000EB800000F2EE2080B210BDDC
:10CF8000E81800203E27002008B5FEF743F9074BBC
:10CF9000022283F8B022D3F8B422C3F8AC02C3F85B
:10CFA000C022012283F8D92208BD00BFE818002062
:10CFB00008B5FEF72FF9084B022283F8B022D3F808
:10CFC000C02200F5B71000F5587002F2DC52C3F829
:10CFD000AC02C3F8C02208BDE81800200F4B10B502
:10CFE00093F8DC221C46012A0CD007D3022A0CD16C
:10CFF0000B4AD36883F00803D36006E0084B08228D
:10D000001A6102E0064B08225A61FEF703F900F5A7
:10D01000F42000F59070C4F8E00210BDE81800207C
:10D02000000C0140026B0346C16810B5406942B173
:10D030001A6C8C1A013A08BF0A46005D1A64C0B225
:10D0400010BD1A6A805C01328A4228BF0022C0B239
:10D050001A6210BD436B13B190F844007047836AA5
:10D06000406A1B1A584258417047426A816A0369F4
:10D070008A4238BFD218521A416B21B149680A441A
:10D08000591E8A4203D2013B981AC0B27047002051
:10D090007047036B13B15B68016C01E0C369016AFF
:10D0A0008B423CBFC2689B18581AC0B27047426A94
:10D0B000806A131A5842584170474171704743794A
:10D0C0009B070AD5436A8269D154436A01690133D7
:10D0D000B3FBF1F201FB123343627047427902F075
:10D0E000020202F0FF0342B10369426A806A013B17
:10D0F000DBB2101A23EA00007047184670474379E4
:10D1000013F001031FBFC36803F1FF32C369006A54
:10D110001DBF181A1040C0B218467047437910B5A9
:10D1200013F0010304460DD0FFF7E9FF58B1236A5D
:10D130006269E168D05C0133B3FBF1F201FB1233A9
:10D14000236210BD184610BDF0B5046D8279A38925
:10D15000467923F4005312F0020F4FEA03434FEADB
:10D1600013430CBF00214FF4005112F0040FA381B0
:10D1700014BF4FF4806E4FF0000E16F0010F876859
:10D18000054614BF04200020B307238A48BF40F09F
:10D1900008029BB223F4405343EA01032382A1898E
:10D1A00048BF90B289B221F4B05121F00C014EEA8F
:10D1B000010140EA0102A281A38A87B023F44073EF
:10D1C0001B041B0CA38201A8FFF786FB039B049E94
:10D1D000254A944218BF1E46A389192272431BB2E6
:10D1E000002BB4BF7E00BE00B2FBF6F66427B6FB90
:10D1F000F7F00001010907FB1163A28912B2002AAE
:10D20000B7BFD9001A013231B1FBF7F2A7BF3232F2
:10D21000B2FBF7F302F007021043A8BF03F00F03BD
:10D22000AA79A8BF184380B212F0010F20812B6D9C
:10D2300006D00E498B4202BF042001F54841086127
:10D2400012F0080F9A8A0BBF22F0080292B2120461
:10D2500042F0080208BF120C9A829A8992B242F4F4
:10D2600000529A8107B0F0BD0038014000440040F0
:10D27000417169E7816067E703460A4690F8460214
:10D28000D96A9B79F9F779BA38B5A0F5137463793F
:10D29000A579DB0746D594F8383205F00105F3B1DE
:10D2A000226B1068838DC3F34E03838494F83C3261
:10D2B00023B1B4F842320133A4F84232917A6A00C1
:10D2C000F9F72DF8012384F83B32002384F8393232
:10D2D00084F83A3284F83832A4F8403238BD94F8F1
:10D2E0003B322046012B04BF94F8393284F83A329D
:10D2F000F9F700F894F83B22236B3AB9012284F83D
:10D300003B221868997A05FA02F207E0002284F8B5
:10D310003B2295421868997A08BF0222BDE838403E
:10D32000F8F7FDBF38BD026D70B515880446ADB283
:10D33000A90613D5036B8BB9C36A1BB1908880B261
:10D3400098470BE0E169928840694E1CD2B2E661D1
:10D350004254E169E268914228BFE3612B0613D58C
:10D36000636AA26A9A42236D0AD0511CA069A16225
:10D37000825C9A802369994206D30023A36270BD20
:10D38000DA6822F08002DA6070BD836A8169426BDC
:10D390001944D160416A994297BF0169CB1ACB1AEF
:10D3A000536096BF0023536083624FF0000380F800
:10D3B0004430136888BF816243F0010313607047F3
:10D3C000436A8269D154436A02690133934228BF98
:10D3D00000234362436B1BB11B68DB0705D4D4E712
:10D3E000026DD36843F08003D36070472DE9F043AA
:10D3F0001D469D4B8DB09842894690469DF85070D1
:10D4000052D19A4B9A4A9B491A609B4AC3F80880AA
:10D410005A6102F580729A614FF48072DA601A6183
:10D42000964A18651A63A2F54842543ADA649A6437
:10D430005963934B3C079A6942F480429A615A6956
:10D4400042F001025A614FF002038DF803304FF4AD
:10D450000073ADF8003001D51C230FE0A80706D5F6
:10D460001823884869468DF80230F9F754F9E9071E
:10D470000AD54FF48063ADF80030482381486946EF
:10D480008DF80230F9F747F90E238DF804300022A9
:10D49000012301A88DF805308DF806208DF807309E
:10D4A000724C04F007FA9DE0774B98424AD1774BD3
:10D4B0006F4AC3F808801A604FF48072DA601A610C
:10D4C000734A18655A6102F580729A61714A9A64CA
:10D4D000DA646B4BDA6942F40032DA615A6942F07D
:10D4E00001025A6102238DF803303A074FF004031A
:10D4F000ADF8003001D51C230EE0AB0706D518238C
:10D50000604869468DF80230F9F705F9EE0709D54C
:10D510000823ADF8003048235A4869468DF8023098
:10D52000F9F7F9F826238DF804300022012301A829
:10D530008DF805308DF806208DF80730534C04F037
:10D54000B9F94FE0544B984240F0F380534B484AAE
:10D55000C3F808801A60524A18655A6102F5807251
:10D560009A614FF48072DA601A614E4A3C079A64FD
:10D57000DA64434BDA6942F48022DA619A6942F054
:10D5800008029A614FF002038DF803304FF4806374
:10D59000ADF8003001D51C230FE0A80706D51823ED
:10D5A000414869468DF80230F9F7B5F8E9070AD520
:10D5B0004FF40063ADF8003048233B4869468DF8CE
:10D5C0000230F9F7A8F827238DF804300022012350
:10D5D00001A88DF805308DF806208DF8073004F08D
:10D5E00069F92E4C0026012384F844302662E66156
:10D5F000A6626662C4F82C906571C4F80880A771B1
:10D600002046FFF7A1FDEA0758D5236B002B4DD02C
:10D6100001A8FDF791FDE36C206B01934FF480535B
:10D620000A9380230693E3680B96049320230993BF
:10D63000636905960293079608960396FFF7D4F858
:10D6400001A9206BFDF785FD226B216D136843F066
:10D65000010313608B8A9BB243F040038B825368B3
:10D660009BB223642AE000BF0038014088220020DA
:10D67000C082010844000240D01B00205800024034
:10D680000010024000080140004400403422002005
:10D69000D01D00200444004000480040E02100204C
:10D6A000D01F002004480040000C01404FF6DF72FC
:10D6B000236D1A80DA6842F02002DA60AB0730D5B9
:10D6C000636B002B28D001A8FDF736FDA36C002565
:10D6D00001934FF480530A93802306932369606B70
:10D6E0000493102303930B950595079508950995C9
:10D6F000FFF77AF8606B01A9FDF72BFD636B1A68E1
:10D7000042F002021A60226D5D605D60938A9BB2F6
:10D7100043F08003938204E0226DD36843F08003DA
:10D72000D360226D204693899BB243F400539381CA
:10D7300000E000200DB0BDE8F08300BF2DE9F0410E
:10D7400005460E46078A83899BB21F40002F37D0BB
:10D75000B7FA87F24FF00043D340DB4399B21F4042
:10D76000A2F11B032982042BF0D8DFE803F0221F6B
:10D770001C190300746A24B1013C0023A4B2736233
:10D7800001E0AC8DA4B2D6F82080B8F1000FDDD056
:10D79000D8F80030404621469847D8F80480F4E78E
:10D7A0003068A98E08E07068298F05E0B068A98FFD
:10D7B00002E0F068B5F84010036889B29847C5E701
:10D7C000BDE8F08110B54B88DC0641BF2F4B1479C2
:10D7D0001B6853F8244044BF2D4B43F820404B882E
:10D7E0009B0641BF294B54791B6853F8244044BF22
:10D7F000274B43F820404B881C070ED5254B0C784F
:10D800001B78B3EB141FA1BF204BD4781B6853F8CF
:10D810002440A4BF1E4B43F820404B889B070ED5E5
:10D820001D4B0C781B78B3EB141FDFBF174B5478DC
:10D830001B6853F82440DCBF154B43F820404B884D
:10D84000DC070FD5154C0B78247803F00F03A342A7
:10D85000DFBF0E4B14781B6853F82440DCBF0C4B21
:10D8600043F820404B885B070FD50B780C4903F039
:10D870000F0309788B42A1BF044B92781B6853F8C1
:10D880002220A4BF024B43F8202010BDE814002042
:10D89000540C0020E3180020E1180020E0180020BC
:10D8A000E2180020254A0023F0B515681C461A46E8
:10D8B0002348244903700B702E1976884EB92F5DCA
:10D8C0003FB9037000230A704B7007781C461A4654
:10D8D0000CE0360548BF013204F1040403F10103F2
:10D8E00048BFD2B2802CDBB2E6D1EAE7E0B2B84260
:10D8F0000CD215F82400013406099E4200F00F00F6
:10D90000A8BF731C9042A8BF421CEFE78A704B70FF
:10D91000C2F3470102F001020A444C1E0A490B48B7
:10D920000A70C3F3470203F001031344047008496B
:10D93000501E084A08701370F0BD00BFEC140020A0
:10D94000D8180020D0210020E2180020E018002084
:10D95000E3180020E11800202DE9FF476F4B044633
:10D9600033F910306E492BB902280CD06D4B1B884F
:10D97000980708D06C4B002223F814206B4B1B88AF
:10D9800021F81430C7E031F814301BB9684A02EBB3
:10D990008402536001339BB221F814301BB2002B78
:10D9A00018DD022C624A634809D1B0F90400202531
:10D9B00090FBF5F5D06800EB4510D0600AE030F937
:10D9C0001400802590FBF5F502EB8402506800EB13
:10D9D000C5105060584F386890F85E20934240F070
:10D9E0009A80534A00EB040C02EB84025568022C27
:10D9F00095FBF3F39CF857E0536008BF5E424FF08D
:10DA0000000221F8142007BFB6B214219EB20A21E9
:10DA1000454DBEF1000F7CD0002E7AD035F8142091
:10DA2000002A76D00FFA86F90FFA82F8C14570D035
:10DA300089EAE97288EAE87AA2EBE972AAEBE87A65
:10DA4000CAEB0202B9F1000F12B209B2DFF8F89086
:10DA500003DDB8F1000F03DC20E0B8F1000F1DDAA0
:10DA60008A420BDD022C90F85A2002D102F5807216
:10DA70000EE039F8141040320A4419E049428A4253
:10DA800018DA022C11D190F85A20C2F57F42C03228
:10DA9000B9F804100A44A9F804200BE0002AB8BF22
:10DAA00052428A4206DD022C04D039F81420203A72
:10DAB00029F8142039F914209CF854809211424519
:10DAC00003DB7245A8BF724690461C4A1FFA88F9CC
:10DAD0001268120308D5142001A98DF8044002939E
:10DAE000ADF80C90F9F766FE154B1B786BB10FFA89
:10DAF00089F004F069FD134904F06EFED7F8008048
:10DB000004F1080748F8270003E03B68234483F842
:10DB1000018025F8146004B0BDE8F0878A16002063
:10DB20006C0700208C0E0020660700205E07002096
:10DB3000D0210020B60E002058070020901B0020A6
:10DB40005C0700200000204160070020094A13788C
:10DB500018441346C0B210F0800F18BF8038107000
:10DB6000054A19781378994201BF00231370014ABE
:10DB700013707047AD240020AC24002010B50A4B70
:10DB80000A4A1B7842609C18094A046012789A423B
:10DB900025BFD31A0B60C3F1800300232EBF4B6057
:10DBA0000B604A6010BD00BFAD240020AE240020F1
:10DBB000AC2400201FB5684602A9FFF7DFFF044B25
:10DBC00002981B6803440398184405B05DF804FBF1
:10DBD000900500202DE9F04F89B001930023824683
:10DBE000994602910392039A934205DA029A52F8F7
:10DBF000232001339144F6E7019B4D46002B56D17B
:10DC0000F9F762F9002852D101987DE00222404ED6
:10DC10008DF81C201A0C4FF480578DF81D2006201B
:10DC20001A0A8DF81E208DF81F30F8F7C1FF7761B2
:10DC3000062003F093FE374B01223761D0461A705D
:10DC400077612646002007A9042203F051FE029FB7
:10DC50004FF0000B039B9B451EDABC4657F8042B84
:10DC60004FEA8B03002A48D0B24236D332465AF8E4
:10DC700003100020CDF814C0049303F039FE049B78
:10DC8000DDF814C05AF8032032444AF80320DCF8C7
:10DC900000309E1BCCF800601D4B4FF480521A617F
:10DCA0001D4A2D1B13681C44019B146053B34DB3D4
:10DCB000194B1B68DCB22A19B2F5807F174A88BF5E
:10DCC000C4F58074D26898BF2C4693429ED3144A00
:10DCD00000231370134A137014E00020D8F80010CA
:10DCE00003F006FE57F8043CD8F80020F61A134457
:10DCF000C8F80030002347F8043C0BF1010B08F191
:10DD00000408A7E7C5EB090009B0BDE8F08F00BF24
:10DD1000000C01408D05002090050020100000201F
:10DD2000AC240020AD24002030B50B4C0B4D2278E4
:10DD30002B7885B09A420CD0684602A9FFF71EFFE7
:10DD40000123684602A90222FFF744FF00232B703B
:10DD5000237005B030BD00BFAD240020AC240020EE
:10DD600030B50E4D0E4C2A78237885B09A4211D0EA
:10DD7000684602A9FFF702FF002302A902226846B3
:10DD8000FFF728FFFFF7E2FE20782B781B1A584296
:10DD9000584100E0012005B030BD00BFAD24002097
:10DDA000AC240020054A064B10781B7883422EBF16
:10DDB000181AC0F18000C018704700BFAD240020C1
:10DDC000AC24002038B50E4C4FF4805545F20820A5
:10DDD000F8F7EEFE6561062003F0C0FD094B012255
:10DDE0002561C7201A70656103F0B8FD064A00235B
:10DDF00025611370054A1370054A136038BD00BFD2
:10DE0000000C01408D050020AC240020AD24002032
:10DE1000900500200148024990E400BF000800403E
:10DE2000A01800200148024988E400BF0004004017
:10DE3000781800204FF0804000497FE450180020FF
:10DE4000014802497AE400BF002C01402818002054
:10DE50000148024972E400BF002C0140281800204C
:10DE6000254B10B55A43254B254C1B680139B3FB94
:10DE7000F2F20388013AA04289B292B29BB212D068
:10DE800004F50064A0420ED0B0F1804F0BD0A4F591
:10DE90009834A04207D004F58064A04203D004F572
:10DEA0008064A04202D123F070039BB2154CA042C3
:10DEB00006D004F58064A0421CBF23F440739BB2DB
:10DEC00003800F4B8185984202850FD003F50063D4
:10DED00098420BD003F54063984207D003F5806366
:10DEE000984203D003F58063984201D10023038652
:10DEF0000123838210BD00BF40420F004C00002070
:10DF0000002C01400010004073B505460068FFF783
:10DF1000A7FF2A680124138800269BB243F001035F
:10DF20001380EB7A01A88DF804308DF805408DF848
:10DF300006608DF8074003F0BDFCEB7A1B2B0BD17C
:10DF4000192301A88DF804308DF805408DF806607E
:10DF50008DF8074003F0AEFC02B070BD0C4B800A98
:10DF600098420CD004D8B0F5801F0CD10120704726
:10DF7000084B984205D04933984206D003E002206E
:10DF8000704703207047FE2070470020704700BF95
:10DF900001001000020010002DE9F8430468074654
:10DFA000204688469146FFF7D9FF03284BD8BA7A16
:10DFB0009108B8F1000F06D1A589AEB202258D40B7
:10DFC00026EA0505A5810A2303FB00131F4A42F830
:10DFD0002380043342F82390B8F1000F07D0BD7AB4
:10DFE000A189AD080223AB400B439BB2A381282338
:10DFF000434303F120011144EFF31286502585F3CA
:10E00000128803F10C051C331544134455F8047FA2
:10E0100017B10F60296804319D42F7D100230B60CE
:10E02000F3B283F31188282303FB0020036A23B192
:10E03000A3899BB243F0010304E0A38923F0010309
:10E040001B041B0CA381BDE8F88300BF2818002027
:10E050000148FFF768B900BFE02100200148FFF741
:10E0600062B900BF342200200148FFF75CB900BF4D
:10E07000882200200C4B4FF400525A604FF6FE737A
:10E080000A48D0F8EC2011680B401360D0F8DC206F
:10E09000D0F8E0309A4202D0B830FFF776B90123C9
:10E0A00080F8FC30704700BF00000240D021002003
:10E0B0002DE9F04F054690F850008DB00A91069278
:10E0C0000B9350B13228A8BF322004F07DFA0146EC
:10E0D0009B4804F081FB044600E09A4C9A4B188858
:10E0E000002808BF012004F06FFA9849079004F057
:10E0F000BFFA00900099204604F0B2F9014600985A
:10E1000004F06AFB924B08901B88980724D591492C
:10E11000B1F90030B1F9020083EAE37280EAE071FC
:10E12000A2EBE372A1EBE07191420C46B8BF14463A
:10E13000B4F5E17F12DA914203DD0028D8BF4042F6
:10E1400003E0002BCCBF1846584204F03DFA824948
:10E1500004F042FB074603E0002701E04FF07E5742
:10E160004FF0000B03950024CDF804B0E3B20993FF
:10E1700063000593794B33F8146030B204F024FA4D
:10E18000774904F075FA04F039FC04F01DFA75497A
:10E1900004F06EFA6F4B029033F9140004F014FA95
:10E1A0006B4B80461B889907049362D0014604F0AC
:10E1B00057F904F023FC069B5B42984203DB069B65
:10E1C0008342A8BF03460599674A885E0B9A1B1ACB
:10E1D00032F91400184404F0F7F98246287F04F05D
:10E1E000EFF9624904F044FA8346287A04F0E8F92A
:10E1F0000146504604F03CFA5D4904F039FA04F057
:10E20000FDFB81460BF1004004F0F8FB814505DB86
:10E21000584604F0F3FB4845A8BF484604F0D4F93B
:10E22000DFF8709101900099504604F021FA59F8F6
:10E23000241004F015F94F494FEA840B824604F08C
:10E24000B5FB38B950464C4904F0CEFB20B1DFF89D
:10E2500028A101E0DFF81CA149F80BA0A87C04F07C
:10E26000AFF90146504604F003FA444904F000FABD
:10E270008346049BDA0700F18F8036B2002EB8BFC8
:10E280007642B6F5206FDFF804914FEA840603DD8D
:10E29000002349F8243028E03949404604F0E8F9E1
:10E2A000039B8246587804F08BF90146504604F0EF
:10E2B00093FA029904F0D2F8009904F0D9F959F8C8
:10E2C000241004F0CDF82F49814604F06FFB38B9D3
:10E2D00048462D4904F088FB20B1DFF8AC9001E0FE
:10E2E000DFF8A090294B43F80690039BD87A04F0FE
:10E2F00067F9264B53F8241004F0BAF9244904F0C6
:10E30000B7F9049B06469B0749D54046019904F09E
:10E31000A5F80146384604F0ABF90146019804F02F
:10E320009FF859468046304604F098F80146384632
:10E3300004F09EF90146584604F092F806462EE095
:10E3400083F9223EAF4C593C880E0020BD378635FC
:10E350008C0E00208A1600200000E143B60E00203B
:10E360000000A03ECDCC4C40F00E00200000A040AC
:10E370006F12033C0000F0C10000F0410AD7A33D3A
:10E380000000A043000040C300004043E4220020FE
:10E390000AD7233CDC2200205E46DDF80480DFF84B
:10E3A0006C9219F8040004F00FF90146029804F089
:10E3B0005FF98B4904F05CF90146404604F04EF8E1
:10E3C00009F1040A5AF82410A30080460298049325
:10E3D00004F044F8009904F0FFF9029B4AF8243055
:10E3E00009F10C0353F824A00293514604F036F8C7
:10E3F0000146089804F03CF90146504604F030F814
:10E40000029B09F1140943F82400824619F804001C
:10E4100004F0DAF80146504604F02AF9714904F094
:10E4200027F982463146404604F01AF8514604F076
:10E4300015F807F0F1FB6C4B059A98526B4B1B8853
:10E44000180506D56A4B1B78590702D50998FFF7BE
:10E4500083FA404604F0D2FADFF8B491049BDFF867
:10E46000B48149F80300304604F0C8FA049B48F828
:10E470000300604B0AF10040029304F0BFFA049BD2
:10E480001A46029BCDF808809850039A9A460132AA
:10E4900003920CB9012469E6079804F0AFFA20F062
:10E4A000030004F091F8544904F096F90A9B95F89A
:10E4B00053200746514CDFF860B193F806E0DFF8CF
:10E4C0005C81002A6CD0B4F904104D4A0029B8BF11
:10E4D000494201FB0EF191FBF2F2E87864324243CB
:10E4E000642092FBF0F004F06FF80190BBF9040097
:10E4F00004F06AF84FF07A5104F0BAF807F08CFB98
:10E50000A2888346009204F05FF8DDF804C06146FB
:10E5100004F0AEF83B4904F05FF90446009A12B2E9
:10E520001046009204F050F8214603F097FF8BEA62
:10E53000EB71A1EBEB71B1F5207F0446009A05DC8D
:10E5400082EAE271A1EBE271642903DD0022C8F8DE
:10E550000820AEE050205043EA7890FBF2F0CBEB7D
:10E56000000004F031F8394604F082F804F046FA6D
:10E57000D8F808207D231044B0F57A5F224AA8BF5E
:10E580004FF47A509042B8BF1046C8F8080090FB8C
:10E59000F3F06B7B5843801104F016F8064688E0D0
:10E5A0004FEA4E01B4F904402831BBF9040000924F
:10E5B0004C4304F009F84FF07A5104F059F807F091
:10E5C0002BFB6411201A03F0FFFF002CB8BF64423C
:10E5D000322C834624DD009AC8F808203AE000BFB8
:10E5E000A69B443BF7CC9238841600208C0E00206A
:10E5F000213000207823002000803B458A1600202F
:10E600000CFEFFFF0000A04280C1FFFFF0220020AF
:10E61000602300206C230020B60E00203023002051
:10E62000687B03F0CDFF0146584604F021F83946D7
:10E6300004F01EF804F0E2F9D8F808201044324A39
:10E640009042A8BF1046314A9042ACBFC8F80800BB
:10E65000C8F80820D8F808306FF0FF005B13B3F556
:10E66000807FA8BF4FF480739842B8BF184603F06C
:10E67000ABFF0646584604F0C1F9EB7858438011C9
:10E6800003F0A2FF224B04461B78032B11D9B5F8E7
:10E690004E50B5F5FA7F0CD204F0B0F96B429842B7
:10E6A00003DBA8420346A8BF2B46184603F08CFFA5
:10E6B00004463146204603F0D3FE04F09FF9154D81
:10E6C00080B2A88000B203F07FFF07F0A5FA124BDA
:10E6D000A8801B881A0506D5104B1B785B0702D54E
:10E6E0000220FFF739F9204604F088F9C9F808003C
:10E6F000304604F083F9029B98600023CAF8083082
:10E700000DB0BDE8F08F00BFFEFFFF0F020000F06C
:10E710007C160020841600208C0E00202130002062
:10E720002DE9F04F89B00693B54B0026B3F902707E
:10E73000B3F90030002FB8BF7F42002BB8BF5B4257
:10E740009F42B8BF1F468046B346B2463446B7F52F
:10E75000FA7F05910392A8BF4FF4FA7701900296D1
:10E76000A84B198811F003053DD0A54B600033F983
:10E770001420039B52005B429A4203DB039B9342AB
:10E78000A8BF1346A04A6FF0040A805E069A1B1ABF
:10E7900032F914006422184498F80830434393FB7C
:10E7A000F2F398F81C200AFB02FA534504DB02EB53
:10E7B000820A9A45A8BF9A46944A52F824301844CF
:10E7C00042F210739842A8BF1846914B9842B8BFC6
:10E7D000184698F8123042F824005843012D4FEAA9
:10E7E0002033029337D0864B8A4833F914B0019B0B
:10E7F000A60093F801C0884B50F824E033F9145078
:10E8000085EAE573A3EBE573B3F5206F16DC5023BF
:10E8100003FB0BF292FBFCF3042295FBF2F55D1B6C
:10E82000AE44BEF57A5F7D4BA8BF4FF47A5E9E453D
:10E83000ACBF40F824E040F8243002E0002340F868
:10E84000243083597D2693FBF6F6019BDB7A7343D4
:10E85000402693FBF6F6880711D507FB06F507FB64
:10E860000BF90298C7F5FA7303FB0A9903FB0053EF
:10E870004FF4FA7199FBF1F293FBF1F505E0CA0749
:10E8800059BF35465A465246029D63000493624B77
:10E89000042033F814C062490FFA8CF393FBF0FEA6
:10E8A00014F80190203109FB0EFE6FF04F099EFB1A
:10E8B000F9F9914431F9142021F814C09B1A98F801
:10E8C000502093FBF0F062B1079203F07DFE5549B2
:10E8D000554B01EBC401079A1B68FBF713F904F0D1
:10E8E0008DF8524B00EB40001A5D514950432022F5
:10E8F00090FBF2F209EB050304989B1A4352414B3B
:10E900001B881B0508D54B4B1B78580704D52046A0
:10E910000492FFF721F8049A47495042019A474B65
:10E9200041F82450464D013243F8249045F8240024
:10E93000019289460CB9012412E7314A0424B2F944
:10E940000410059A334E927998F80D000F32520058
:10E950004A4331495211B1F90410002A91FBF4F1F4
:10E96000A2EB0101B8BF5242322AB4680BDC00FBB3
:10E970000140344A8242A8BF024633488242ACBFBB
:10E98000B260B06001E00022B26098F803402F4A04
:10E990004C431278A411032A0CD9B8F84E20B2F5D2
:10E9A000FA7F07D251428C4203DB9442A8BF14463F
:10E9B00000E00C46B6686FF0FF0246F34F36B6F53E
:10E9C000807FA8BF4FF480769642B8BF1646184A9B
:10E9D000A11991800B4A1288110508D5154A1278A1
:10E9E000520704D502200193FEF7B6FF019B9C60FD
:10E9F0000023C9F80860AB6009B0BDE8F08F00BF24
:10EA00008A1600208C0E0020F00E00200823002023
:10EA1000F0D8FFFF30230020B60E002080C1FFFF9A
:10EA2000F0220020482300202C2300200423002073
:10EA300084160020213000206C2300206023002059
:10EA400078230020FEFFFF0F020000F07C1600205C
:10EA50002DE9F04F87B00493A64B80461C880391A4
:10EA600004F00204A4B2934694B1A34BB3F902405C
:10EA7000B3F90030002CB8BF6442002BB8BF5B4232
:10EA80009C42B8BF1C46B4F5007FA8BF4FF4007489
:10EA9000C2460025984B042633F91510974B984829
:10EAA00033F815304FEA450C0193BDF904304900A5
:10EAB00093FBF6F2029283EAE372A2EBE372B2F501
:10EAC000206F4FEA850950F825600FDC029A8A1AF8
:10EAD0003244B2F57A5F8B4EA8BF4FF47A52B242FD
:10EAE000ACBF40F8252040F8256002E0002240F845
:10EAF000252050F809709AF801609AF80B204E43CF
:10EB0000FF117C4857430088B21186074FEAA717C8
:10EB10003CD0CBF10000814203DB5945A8BF5946E8
:10EB2000084642F2107E7849784E3CF90110401AAE
:10EB3000049931F91510084459F80610014471453B
:10EB4000A8BF7146DFF8F8E17145B8BF714649F8D2
:10EB5000061098F80860704398F81C60C01106EB26
:10EB60008606C6F1000E704503DBB042A8BF3046F2
:10EB7000864698F81200CEEB0206414309137F1A2D
:10EB80006743664301EB67270EEB662260490298F4
:10EB90004E5D243146433CF90100A2EBA6161B1A38
:10EBA000042093FBF0F098F85020BDF804302CF8C6
:10EBB000013082B1CDF808C0019203F005FD55493E
:10EBC000554B01EBC501019A1B68FAF79BFF03F057
:10EBD00015FFDDF808C0514B00EB40005B5D50496C
:10EBE0005843F2194311D21A2CF80120414A1088D7
:10EBF000944610F4006F0DD04A480078400709D5BC
:10EC00002846059101930292FEF7A6FE0599DDF8CC
:10EC100008C0019B44485B4249F80060434E0AF13A
:10EC2000010A49F80670424F49F8073081460DB98C
:10EC300001252FE7304B0425B3F90400039B98F816
:10EC40000D409B790F335B0043432C485B11B0F9B7
:10EC50000400002B90FBF5F52948A3EB0505B8BF90
:10EC60005B42322B82680BDC04FB0524314BA34250
:10EC7000A8BF2346304CA342ACBF8360846001E050
:10EC80000023836098F803305D432C4BAD111B7853
:10EC9000032B0CD9B8F84E30B3F5FA7F07D25C429B
:10ECA000A54203DB9D42A8BF1D4600E025468468BF
:10ECB0006FF0FF0344F34F34B4F5807FA8BF4FF4E7
:10ECC00080749C42B8BF1C462B198B80BCF8003066
:10ECD0001A0506D5134B1B785B0702D50220FEF7F9
:10ECE0003BFE0023C9F80850B460BB6007B0BDE824
:10ECF000F08F00BF8C0E00208A160020B60E002078
:10ED00003023002080C1FFFFF00E002008230020E8
:10ED1000F0220020482300202C2300200423002080
:10ED20008416002021300020602300206C23002066
:10ED300078230020FEFFFF0F020000F07C16002069
:10ED4000F0D8FFFF2DE9F04F87B00393984B0026D2
:10ED5000B3F90280B3F90030B8F1000FB8BFC8F1C1
:10ED60000008002BB8BF5B429845B8BF9846834661
:10ED7000B246B1463446B8F5FA7F0292A8BF4FF4C6
:10ED8000FA78009001968B4B198811F0030040D05F
:10ED9000022C3ED0864B650033F91420029B5200B2
:10EDA0005B429A4203DB029B9342A8BF1346824A0E
:10EDB0006FF00409AD5E039A5B1B32F914506422B4
:10EDC0001D449BF808306B4393FBF2F39BF81C2027
:10EDD00009FB02F94B4504DB02EB82099945A8BF08
:10EDE0009946764A52F824302B4442F21075AB42D1
:10EDF000A8BF2B46724DAB42B8BF2B4642F8243019
:10EE00009BF81220012802FB03F34FEA23330193FE
:10EE10003DD0674B6B4D33F914A0009BA00093F8D5
:10EE200001E0694B55F8247033F9146086EAE67303
:10EE3000A3EBE673B3F5206F1CDC022C14D0502337
:10EE400003FB0AF292FBFEF3042296FBF2F69E1BF2
:10EE50003744B7F57A5F5D4BA8BF4FF47A579F42AE
:10EE6000ACBF2F502B5007E08AEAEA73A3EBEA739A
:10EE7000642BE4DD00232B50524B7D26C35893FBBB
:10EE8000F6F6009BDB7A7343402693FBF6F68D077C
:10EE900013D5022C11D008FB06F508FB0AF70198E0
:10EEA000C8F5FA7303FB097703FB00534FF4FA72BA
:10EEB00097FBF2F193FBF2F508E0C80704D5022CAA
:10EEC00002D0019D494601E0354651463E4B04279C
:10EED00033F914303E4A93FBF7F3A25C6FF04F070F
:10EEE000534393FBF7F3022C4FEA440C01EB030767
:10EEF0000FD13846CDF810C003F066FB354B3649CC
:10EF00001E221B68FAF7FEFD03F078FD0746DDF8C8
:10EF100010C02D4B314A3CF803103CF902000BB2F3
:10EF20002CF802109BF85020181A042390FBF3F0E1
:10EF300082B1CDF814C0049203F046FB2849254B5A
:10EF400001EBC401049A1B68FAF7DCFD03F056FDDF
:10EF5000DDF814C0234B00EB40001B5D22495843F1
:10EF6000202390FBF3F37A19D21A2CF80120114ACE
:10EF70001288110508D51D4A1278520704D5E0B24F
:10EF80000493FEF7E9FC049B194A5B4242F82470A3
:10EF9000184A42F82450184A42F82430009B0134A1
:10EFA0000133032C00937FF4EEAE07B0BDE8F08F81
:10EFB0008A1600208C0E0020F00E0020082300206E
:10EFC000F0D8FFFF30230020B60E002080C1FFFFE5
:10EFD000F02200202C2300202423002018230020CE
:10EFE0004823002004230020841600202130002024
:10EFF000602300206C230020782300202DE9F04FAF
:10F0000087B00493874B81461B8803929D0737D5B1
:10F0100040F2E632109B8448DC89B0F900301B1BBB
:10F0200003F2F315954203D8002BB8BF5B4201E011
:10F030004FF4FA73B0F9022040F2E630121B02F2EC
:10F04000F314844203D8002AB8BF524201E04FF4BF
:10F05000FA729342B8BF13460522C3F5FA7393FBC5
:10F06000F2F30A22643B534399F81C20D210534315
:10F07000642293FBF2F3134423EAE373DBB200E070
:10F080006423C8460093CB1C02930025029B022DEB
:10F0900013F8011F654802934FEA450B06D1B0F9FA
:10F0A000040001F11B04444363112DE030F91520E5
:10F0B000039B50005B42984203DB039B8342A8BF43
:10F0C00003465B4830F90B4004981B1B30F91500D0
:10F0D0001844544B1E88F40712D401F11B035A4301
:10F0E000B1074FEA22130FD599F812409DF900108D
:10F0F00044434C43642294FBF2F203EB221303E0FB
:10F1000099F8083043431B114A4A042432F90B2072
:10F1100098F8017092FBF4F41C1B474E6743AB5DFB
:10F12000022D03FB07F701934FF0640397FBF3F7FE
:10F130004FEAE7170AD1384603F046FA311D1E227E
:10F14000F368FAF7DFFC03F059FC07463B4A3A4BF9
:10F15000118803F1100E01FB04F298F80B605EF8C1
:10F160002500D21206FB0206354AB6F5001FA8BFDD
:10F170004FF400169642B8BF164603F11C0252F82F
:10F18000250042F825404FF6FF720909B2FBF1F164
:10F19000201A484399F850404EF825604FEA850AF6
:10F1A000761380116CB1059303F00EFA059B22468D
:10F1B00003F1280101EBC501DB68FAF7A3FC03F0BA
:10F1C0001DFC98F8153000EB40005843019B1D4A88
:10F1D00043431846642390FBF3F0BB190412234405
:10F1E00022F80B300F4B1B881A0506D5164B1B78DF
:10F1F0005B0702D5E8B2FEF7AFFB144B01354AF8C6
:10F20000037003F10C02032D03F118034AF80260A6
:10F210004AF8034008F101087FF438AF07B0BDE8B1
:10F22000F08F00BF8C0E00203E2700208A160020A1
:10F23000F00E0020B60E0020202300201016002023
:10F240000000E0FF84160020213000206023002011
:10F250002DE9F04F11F0FD0499B00190039106D013
:10F26000AD4B1B689A0700F1BE8000F02FBDAB4B81
:10F27000AB485B689847AA4D0028F1D0A94B2846B7
:10F280001A782946FDF748FDA74B1B88002B00F094
:10F290008280A64B5A6E03F16806127803F1740857
:10F2A0000292A14A35F9140017884FEA440AB7F5CB
:10F2B0007A7F02BF00223260C8F810203268024410
:10F2C000326003F081F9D8F8101001F1010BBBF1A5
:10F2D000010FC8F810B007D10022C8F80400C8F820
:10F2E0000000C8F808202BE0D8F800C0059061465F
:10F2F000CDF810C003F0B2F88146584603F064F927
:10F300000146484603F068FADDF810C00146604641
:10F3100003F0A6F88346059AC8F80400594610463B
:10F3200003F09CF80146484603F0A2F9D8F808100B
:10F3300003F096F8C8F800B0C8F80C00C8F8080048
:10F34000DFF8ECB10022012F25F80A202AF80B2063
:10F35000DFF8D4912AD1D8F81000012808DD01384F
:10F3600003F032F90146D8F80C0003F035FA00E05A
:10F37000002006F06BFE029B7BB10490184603F060
:10F3800023F9049A0146104603F02EFB28B14FF4EE
:10F390007A73A9F80030002319E032684FF47A71CB
:10F3A00002F5FA7292FBF1F22BF80A200134032CD9
:10F3B00006F1040608F114087FF473AF012F02D19F
:10F3C0003846FBF789FFB9F80030013BE1E75849BF
:10F3D00035F8132031F81310521A25F81320013391
:10F3E000032BF4D13CE7039B002B00F06F844F4CC0
:10F3F00094F8B670254647B1012F40F05E84D4F8EA
:10F40000F870D4F8FC60002424E1FBF703FF064603
:10F41000C4F8B800D4F8C000301A03F0D1F8454958
:10F4200003F026F9444BC4F8BC005B6804F1C40047
:10F43000C4F8C060984704F1C406002800F0FD80BD
:10F440003E4B30461A783146FDF766FCB4F8CA30B8
:10F45000002B42D03B46D4F8CC00B5F8CA2038493E
:10F46000B2F5C87F04BF002241F823204FEA830C85
:10F4700036F913E051F80C202C4F724441F80C205F
:10F48000002126F8131020F813100133032BE4D1C8
:10F49000B7F8CA30012B1BD1D7F8D0304FF4C87E53
:10F4A000C83393FBFEF20280D7F8D420C83292FB17
:10F4B000FEF24280D7F8D830224AC83393FBFEF3DD
:10F4C00012889B1A8380019B19805980FBF768F989
:10F4D000B4F8CA30013BA4F8CA301B4B1B685B0769
:10F4E00040F19780B4F8DC20104B322A2ED1D3F8AB
:10F4F000CC201188A3F8DE1051889288A3F8E01080
:10F50000A3F8E220019A1288A3F8E420019A528815
:10F51000A3F8E6201CE000BF0816002054150020C8
:10F52000B60E00207D1500201E3000202023002074
:10F53000D0230020BD378635481500202430002018
:10F54000F02300200C000020901B0020002A3FD058
:10F55000D4F8CC100020B5F8DC304FEA800E322B06
:10F56000394B04BF002243F8202036F910C053F86D
:10F570000E20364F624443F80E20002326F8103048
:10F5800021F81030013003281A46E4D1B7F8DC30F6
:10F59000012B18D10C2087F8F42087F8F530FBF701
:10F5A0009BFED7F8CC30B7F8DE201A80B7F8E02001
:10F5B0005A80B7F8E2209A80B7F8E430019A1380B5
:10F5C000B7F8E6305380B4F8DC30013BA4F8DC3007
:10F5D00094F8F6301D4AE3B1D2F8E830322193FBBB
:10F5E000F1F3D2F8CC50002082F8F6002B80D2F84C
:10F5F000EC3093FBF1F36B80D2F8F030144A93FBBC
:10F60000F1F312889B1AAB80019B18805880FBF79E
:10F61000C7F8D4F8CC20B4F8C43011885B1AA4F829
:10F62000C4305188B4F8C6305B1AA4F8C63092884A
:10F63000B4F8C8309B1AA4F8C83094F8B630013337
:10F6400084F8B630D3E600BF082400202023002031
:10F650000C000020DFF8D8B20BF1C40232F814001D
:10F66000B04A0BF5807522F8140000B202F0ACFF2E
:10F67000394602F0FDFFAC4A45F8240032F9140087
:10F6800002F0A2FF314602F0F3FF0BF5867545F854
:10F6900024000134032CDDD128462A460BF58C7159
:10F6A000FCF7AAFB28460BF5927106AAFCF7A4FB0F
:10F6B00006A80246DBF8BC10FCF7B7FB06984FF033
:10F6C0007C5102F0D5FF4FF07C510646079802F0BE
:10F6D000CFFF4FF07C510546089802F0C9FF314634
:10F6E0000446304602F0C4FF29460746284602F089
:10F6F000BFFF0146384602F0B3FE214607462046CA
:10F7000002F0B6FF0146384602F0AAFE4FF07C51E7
:10F7100002F0AEFF01464FF07E5002F09FFEDBF894
:10F7200034910290494602F0A3FFDBF83881039040
:10F730004146204602F09CFF039A0146104602F023
:10F740008FFEDBF83C7103903946284602F090FFAB
:10F75000039A0146104602F081FEDBF830A10390C7
:10F760005146304602F084FF039A0146104602F0EB
:10F7700077FE41460590029802F07AFF39460390E1
:10F78000304602F075FF039A0146104602F068FE0B
:10F7900051460390284602F06BFF039A014610463B
:10F7A00002F05EFE49460390204602F061FF039A94
:10F7B0000146104602F052FE49460490284602F0E7
:10F7C00057FF41460390304602F052FF039A01462C
:10F7D000104602F043FE39460390029802F048FFBB
:10F7E000039A0146104602F03BFE51460390204624
:10F7F00002F03EFF039A0146104602F031FE5146E8
:10F800000390029802F034FF49468246304602F0E7
:10F810002FFF0146504602F021FE4146064628468B
:10F8200002F026FF0146304602F018FE3946054632
:10F83000204602F01DFF0146284602F00FFE059B00
:10F84000DDF810C0039A03F10041CBF83001CBF88A
:10F8500038C109A80CF1004CCBF83C2102F1004260
:10F86000CBF834310991CDF828C001460B920CAA8F
:10F87000FCF7C2FA2D48DBF8301112AAFCF7D5FAD2
:10F880000FAE09A8294915AAFCF77EFA15A812A9F6
:10F890003246FCF7B1FA0CA8314615AAFCF774FA07
:10F8A0003246224815A9FCF7A7FA1198DBF8401157
:10F8B00003F09AF89BF8442110B142F0080201E0ED
:10F8C00022F008021A4C8BF84421D4F8483104F590
:10F8D000A8771B7873B3D4F84C913846494612AADE
:10F8E000FCF7A3FAD4F85C8104F58070414615AAB0
:10F8F000FCF79BFA12A815A93A46FCF77DFA04F525
:10F90000B070494612AAFCF790FA3046414615AA53
:10F91000FCF78BFA12A815A904F5B072FCF76CFA83
:10F9200014E000BFB00E0020B60E0020E4820108F3
:10F930002023002004F5807304F5B07593E80700D8
:10F9400087E8070096E8070085E80700D4F800017B
:10F95000D4F80481014602F08BFE4146054640463C
:10F9600002F086FE0146284602F07AFDD4F80871BE
:10F9700005463946384602F07BFE0146284602F02D
:10F980006FFD9A49074603F02FF8994E002520B9DC
:10F990003846984903F00AF830B1C4F82451C4F845
:10F9A0002851C4F82C5112E006F5927206F5A870A1
:10F9B00006F5B071FCF7E8F9D6F8BC108E4802F0F5
:10F9C0000BFF014606F592700246FCF72EFAB4F8DA
:10F9D0006C31874D01339BB2B3F57A7FA4F86C315B
:10F9E0004ED1D5F83001D5F83491014602F040FEF1
:10F9F00049460646484602F03BFE0146304602F0C4
:10FA00002FFDD5F8388106464146404602F030FECB
:10FA10000146304602F024FDD5F83C7106463946D1
:10FA2000384602F025FE0146304602F019FD06F088
:10FA30000DFB01464FF07E5002F0CEFED5F834119A
:10FA4000064602F015FED5F838118146304602F020
:10FA50000FFED5F83C118046304602F009FE3146D3
:10FA60000746D5F8300102F003FE0023C5F8300147
:10FA7000C5F83491C5F83881C5F83C71A5F86C31EA
:10FA8000D4F83081D4F838614046314602F0F0FDB8
:10FA9000D4F83471D4F83C5139460446284602F073
:10FAA000E7FD0146204602F0D9FC014602F0D8FCF1
:10FAB0004FF07E51044602F097FF50B920464F495F
:10FAC00002F074FFE0B920464FF07E5102F08CFF47
:10FAD00008B14FF07E54204602F018FC06F0D8F82A
:10FAE00002F068FC0021044602F07EFF48B1444960
:10FAF000204602F0B3FC002102F076FF88B923E033
:10FB0000404C04F100493E49484602F0A7FC002160
:10FB1000824602F069FF90B12046002102F064FFA6
:10FB200030B12046364902F099FC4FF0010902E05D
:10FB30004FF001095046344902F038FF0FE02046EB
:10FB4000002102F051FF08B1204600E048462C4950
:10FB500002F084FC2D494FF0010902F045FF00B985
:10FB600081465FFA89F353B128464146FAF739FADC
:10FB7000014602F075FC4FF0000A05467DE039466B
:10FB8000404602F075FD29468146304602F070FD80
:10FB90000146484602F064FC014602F061FC314631
:10FBA0008346304602F064FD81463946384602F00D
:10FBB0005FFD494602F054FC014602F051FC01464B
:10FBC0004FF07E5002F04AFC00218246584602F077
:10FBD000E3FE20B15046002102F0DEFEC0B95146DE
:10FBE0005846FAF7FEF9824614E000BFB81E8D3F72
:10FBF000202300203D0A673F6F12833A000080BF38
:10FC0000DB0FC93FDB0FC9BF35FA0E3C35FA0EBC1E
:10FC10004FF0000A2946404602F02AFD3146804650
:10FC2000384602F025FD0146404602F019FC014627
:10FC300002F016FC29460646284602F019FD014648
:10FC4000484602F00DFC014602F00AFC01464FF066
:10FC50007E5002F003FC00210546304602F09CFE77
:10FC600020B12846002102F097FE28B929463046E7
:10FC7000FAF7B7F9054600E000251A49504602F0A8
:10FC8000F7FC05F0C9FF184E16493080204602F0F7
:10FC9000EFFC05F0C1FF1549708005F1004002F04E
:10FCA000E7FC02F0ABFE80B2114B10F4004F18BF1E
:10FCB00000F5B4701880002300E001230D4A0021F4
:10FCC00082F8B610002B7FF492AB07E0094B0022BC
:10FCD000A3F8C420A3F8C620A3F8C82019B0BDE833
:10FCE000F08F00BF4D3D0F44F00E0020E12E654225
:10FCF000F40E00202023002001380A4B042804D8E9
:10FD0000DFE800F00507090B0D00074A08E0074A85
:10FD100006E0074A04E0074A02E0074A00E0074A13
:10FD20001A6070474400002045ED0008FDEF000810
:10FD3000251C010851EA000821E70008B1E000088D
:10FD4000022803D0431E584258417047064B1B6897
:10FD50001B7823B1054B1868C0F3C0407047044BB3
:10FD60001878C0F3800070476C050020900E0020CA
:10FD700021300020674B73B51878FFF7E1FF664D1F
:10FD800004462B78834220D0C8B1644B1B68E3B192
:10FD900093F9000002230093614B04211B680022A9
:10FDA0005B78003318BF012301934FF41653F9F722
:10FDB0002FFC5C4B186040B101232B7005E0594EBD
:10FDC0003068F9F711FC34602C70574B574D187898
:10FDD000FFF7B6FF2B780446834218D088B1544B06
:10FDE0001B68A3B10022012493F9000008214FF4FD
:10FDF000964300940192F9F70BFC4E4B186028B91A
:10FE000005E04C4E3068F9F7EFFB34602C704A4B3C
:10FE10004A4D1878FFF794FF2B78044683422E460C
:10FE200043D0002838D0464B1A68002A3DD0D379F9
:10FE300092F90000002B4FF00202424C08BF02234F
:10FE40000092002254F8233001921021F9F7E0FBD0
:10FE50003D4B0546186040B33C4C94F84A30022BA9
:10FE60000BD094F89620022A01D14C3405E023B13E
:10FE7000002A04F14C0418BF0024354B1C6044B127
:10FE8000204600214C2205F0BAFC0223256084F8AC
:10FE90004A300123337008E02B4E306801F066F8D9
:10FEA0003068F9F7A1FB34602C702A4B2A4D187882
:10FEB000FFF746FF2B780446834229D000B3274B37
:10FEC0001B682BB3264A93F900001268032352786B
:10FED0002021002A0CBF08220922009301924FF42E
:10FEE00061430022F9F794FB1E4B186080B11E4A53
:10FEF000012313702B701D4B1A681D4B1A6007E00D
:10FF0000184E3068F9F770FB174B34601C702C707A
:10FF100002B070BD74050020C90B002070050020E0
:10FF2000D40B0020A814002075050020D80B002059
:10FF30002C0C00201C0C002080050020320C00201E
:10FF40007C050020B0910108340C002064270020BB
:10FF5000380C00208C050020400C00208805002073
:10FF600084050020440C0020480C00209C1B00202D
:10FF70004C0C0020642928BF6421F8B501FB00F572
:10FF8000642495FBF4F40646E4B20027FBB2A342D6
:10FF900004D29F20F6F7C1FF0137F7E7B4420BD236
:10FFA000142195FBF1F5C4EB8410663DC4EB800091
:10FFB0002844C0B2F6F7B1FF0134E4B2B44201D232
:10FFC0009A20F7E7F8BD2DE9F743FBF723F98F4DAA
:10FFD0002B68C31A002BC0F27F8200F5433303F570
:10FFE000A0732B608A4B1E782B79C6F38006F31A18
:10FFF00018BF01232E714EB1002B00F06D82854B8E
:020000040801F1
:100000005A789A7001225A701A7025E0814A2BB1F1
:10001000D37843F00203D37093785370D47804F00C
:10002000020101F0FF0339B97A498968411A0029B0
:1000300003DB04F0010300E0012303F0010775492D
:1000400017704BB1E70707D50B79734A013303F0FB
:1000500003030B71D35C4B706E4CDFF8088223787E
:100060007BB3E37823F00203E3706C4B0344AE20D0
:10007000A360F6F776FF08B1F6F778FF88F800007E
:10008000002800F02982B020F6F76BFF4020F6F739
:1000900068FF0020F6F765FF1020F6F762FF4FF4C7
:1000A0008067013F0020BFB2F6F732FF002FF8D182
:1000B0003846F6F7CAFF6278594B53F82200F6F734
:1000C00047FF98F80030002B00F006826378052B7C
:1000D00000F2C281DFE813F00600C00117007700CC
:1000E000650180014F49504A504B5148F9F735FF9F
:1000F0000120F6F7AAFF4E48F6F72AFF0220F6F78E
:10010000A4FF4C48A6E14C4F3B689C0735D5DFF86F
:1001100058810A23B8F80010DFF85091B1FBF3F2D0
:1001200003FB121399F8001092B29BB20091404861
:100130004249F9F712FFFBF791FE0120F6F785FF20
:100140003B48F6F705FF3E4B99F800201868B8F8D1
:100150000030047902FB143164234B43C178022040
:100160000C1B5443B3FBF4F4E4B2F6F76EFF2146E4
:100170001520FFF7FFFE032400E001243B6818056B
:1001800040F16A812F4B30491F68642397FBF3F2DB
:10019000096803FB1273009125482C49F9F7DDFE2D
:1001A000FBF75CFE2046F6F750FF2148F6F7D0FE3D
:1001B000FCF770FE0746601CF6F747FF152039462E
:1001C000FFF7D8FE48E10120214FF6F73EFF214816
:1001D000F6F7BEFE3B6899074AD51F4A1448B2F9A4
:1001E0000210B2F900300091B2F904201B490192CB
:1001F0001B4AF9F7B2FEFBF731FE0220F6F725FFA6
:100200000B48F6F7A5FE032433E000BF902400203E
:1002100021300020E00D0020A7A00108404B4C0039
:10022000F0820108ABA00108B4A0010817930108EF
:1002300095240020BBA00108901B0020C0A001084D
:10024000DC1A0020080F0020E01A0020D8A00108C6
:1002500008160020EDA00108B00E002003A101083F
:1002600012A1010835020020881B00204800002050
:1002700002243B68DA071AD5994A9A48B2F9021063
:10028000B2F900300091B2F9042097490192974ADF
:10029000F9F763FE04F10108FBF7E0FD2046F6F7ED
:1002A000D4FE5FFA88F88F48F6F752FE44463B6862
:1002B0001B0718D58E4A8B48B2F90210B2F90030EC
:1002C0000091B2F90420884901928A4AF9F745FE63
:1002D000671CFBF7C3FD2046F6F7B7FEFFB2814867
:1002E000F6F736FE3C46844A7F49B2F90030B2F94F
:1002F00002207C480092814A814FB2F90020B94621
:100300000192804AF9F729FEFBF7A8FD2046F6F78F
:100310009CFE7448F6F71CFE72493868F9F7B8FC81
:10032000704805F0B0FA04F101085FFA88F8C1B22C
:10033000092909D84B1CDBB2294420224A7100212B
:10034000EA1891711946F3E7664FD9F80400394469
:10035000F9F79EFCFBF782FD4046F6F776FE38463D
:10036000F6F7F6FD3946D9F80800F9F791FC38465A
:1003700005F089FA0234E4B2C1B2092909D84A1C4D
:100380006B18D2B2202159710021AB189971114616
:10039000F3E739440020F9F77BFCFBF75FFD2046CB
:1003A00055E00024584F3B78A34255D90E2C53D02A
:1003B00060080130F6F749FE204601F011FB3B785A
:1003C000A34206D92020F6F7A8FD601CC0B201F0B8
:1003D00007FB0234E4B2E5E74C4C4D4994F8B027F2
:1003E0004048F9F7BAFD0120F6F72FFE3D48F6F731
:1003F000AFFD484B48491F783A483A46F9F7ADFDFA
:100400000220F6F722FE3748F6F7A2FD0C2303FB85
:100410000744424994F8B32794F8B2373148F9F7C2
:100420009CFDFBF71BFD0320F6F70FFE2D48F6F7AA
:100430008FFD94F8B81794F8B62794F8B737294881
:1004400000913749F9F789FDFBF708FD0420F6F71D
:10045000FCFD2448F6F77CFD002E3DD1314BB02049
:1004600093F82030052B97BF2F4A3F249B181C7E02
:10047000F6F777FD0C20F6F774FD1620F6F771FD00
:100480002046F6F74AFDB020F6F76BFD0220F6F79E
:1004900068FD1720F6F765FD244B1B78002B244BD5
:1004A00018BF72201B7808BF2120002B18BF5220D4
:1004B000F6F733FDB020F6F754FD0820F6F751FDAE
:1004C0001720F6F74EFDEC7E1A4B185D013404F050
:1004D0000304F6F722FDEC7603B0BDE8F08300BF1D
:1004E000B60E00209524002003A1010816A10108E2
:1004F000BC0E00205EAD0108F00E0020F40E0020BE
:10050000D40C00201AA10108E42F0020FC270020B1
:100510001EA10108302500202AA101083BA10108E5
:100520004CA10108A01B0020F0820108080D00204A
:10053000B60D00205EA101080846F7F797B80F4BEB
:100540001A786F2A16D140F2E4725988914211D17B
:100550001A79BE2A0ED193F8E0270020EF2A0BD19A
:1005600013F8012B5040064A9342F9D1B0FA80F0BB
:100570004009704700207047704700BF00F801082D
:10058000E4FF01082DE9F74FE94C002140F2E47245
:10059000204605F034F9E74B04F53A721A60E64B51
:1005A00000221A70E54B04F2B27119606F232370B8
:1005B000032363714FF48173A3604FF41673A4F89F
:1005C0006431FA23A4F866314FF4FA73A4F86C315D
:1005D000012384F85E3184F8693184F86A3184F843
:1005E0007C3184F88431052384F8273240F2DC53CF
:1005F000A4F8963140F24C43A4F8983140F26C7361
:10060000A4F89A3140F27533A4F89C3140F64303C4
:10061000A4F89E312346202184F868116E2184F8C5
:100620007A110A2184F87B112B2184F87D11212174
:1006300084F87E11232184F87F114FF4C871A4F847
:100640008011032ACCBF0121002102F1010283F8AD
:10065000A01114BF1E210521122A83F8A11103F154
:100660000203EED140F27E42A4F8402140F23A72F9
:10067000A4F8422140F2DC52A4F8462140F27E5216
:10068000A4F8482140F2EA52A4F84A2140F2B452B8
:100690004FF4FA63A4F8C631A4F8CA31A4F8CE31F5
:1006A000A4F8D231052384F8E031C82301264FF4A1
:1006B0007A7AA4F8E431A4F84C214FF4C8733222BA
:1006C000DFF870B21E274FF01909A4F8E831A4F83A
:1006D0004E21A4F8C4A1A4F8C8A1A4F8CCA1A4F800
:1006E000D0A184F8E26184F8E36184F8E661A4F8BB
:1006F00044A184F8937184F8E191A4F85031A4F8EE
:10070000522184F8DF6184F8EC61019201F0FCF978
:10071000DBF8003000255F212573D9700F21597156
:10072000222199710E21197435219976212159744C
:100730005321D9765A211972782199722D21197570
:100740004FF4FA71019AA3F84E107D494FF0280832
:100750001420DF721F7383F807900A274FF0640993
:100760004FF07F5C587598755A731A711E7083F834
:10077000018083F80280DF759D731D76DD735D76E1
:100780009F7483F81C9083F809809E7783F85080CB
:10079000C3F820C09963C3F824C0D963DFF8C0C18F
:1007A0006849DFF8C0E19962C3F848C066494FF074
:1007B0004B0CC3F82CE0C3F830E083F84CC0DFF8F2
:1007C000A8E14FF4E17C5963A3F85CC000214FF02D
:1007D000100C196483F85EC0C3F844E083F85350EA
:1007E00083F8547083F8557083F8567083F85790E7
:1007F00083F8589083F8599083F85A5084F8B427B6
:1008000040F2DC524FF0460CA4F8BC2704220191C0
:1008100084F8B3C784F8BA0784F8B29784F8B55758
:1008200084F8B95784F8B65784F8B75784F8B8579E
:10083000A3F8645083F86820152283F87420434A93
:10084000A3F866509A67424AA3F86250DA67414AB1
:10085000C3F86CE0C3F8802083F8708083F871805F
:1008600083F884603C4801F07DF9DBF800204FF408
:10087000487382F81D5182F81E5182F81F8182F858
:10088000206182F82451A2F8223184F8D67184F8CC
:10089000D771A4F8D8A184F8DA51A4F8DC911446F1
:1008A00001990E2303FB05236FF0170683F82561DA
:1008B000032683F826616FF02F0683F82761072649
:1008C00083F828616FF0230683F82961052683F8F1
:1008D0002A61642384F82B3101355A2384F82C31A2
:1008E00084F82D31082D4FF0FF0384F82E314FF09E
:1008F000000004F10E04D4D1034682F895010C4D9A
:100900005A191033C02B1161F9D105F52A70002155
:10091000402204F074FF0023104EEA189959043362
:100920000868382B024CC2F8A802F5D11EE000BFBF
:10093000FC270020D40E0020302500200C0F0020C2
:100940008FC2F53C000060406666663F9A99193F89
:10095000F6287C3F3D0A773F90A1010810830108EB
:1009600000004040CDCCCC3E0000A04004F50A7011
:100970000021802204F043FF06F13801702204F5C3
:100980000A7004F031FFFCF78DFFDBF800600023F4
:100990000125314604F590604FF4CC7284F8D837C5
:1009A00084F8D65784F8D75704F01EFF04F5C360C7
:1009B00031464FF4CC7204F017FF0E4B1B681A68D7
:1009C000C4F8BE275A68C4F8C2279A68C4F8C62774
:1009D0001A68C4F8CA275A68C4F8CE279A6802234E
:1009E000C4F8D22784F8E05484F8783603B0BDE820
:1009F000F08F00BF0C0F002038B5144B05461B6864
:100A000098421ADD124B93F8D84714B1012C09D043
:100A100017E0104B1B68186988B1A842CCBF0120B1
:100A2000022038BD7F280CDCFDF7BCF9C0F17F0047
:100A3000854208DDFDF794F905E0002038BD01206E
:100A400038BD022038BD204638BD00BF2C2700200D
:100A5000FC27002074250020074B93F8D837012B82
:100A600008D1064A064BD0681B68834234BF002079
:100A70000120704700207047FC2700201000002054
:100A80009005002038B5094B93F8D85765B9084C44
:100A90002068F8F7A9FD074B25601B78022B03D1CE
:100AA000BDE8384000F0F0BF38BD00BFFC27002093
:100AB0007425002071250020064B93F8D8371BB110
:100AC000012B05D1FDF74CB9034B1868FAF7AEBC02
:100AD00000207047FC27002074250020F8B5011F76
:100AE00006460023083051F8042F02F120043F2C61
:100AF0003BD802F108040F2C06D80232032A04D98D
:100B0000002B08BF012300E002238142EBD1012B1F
:100B100030680ED0022B1AD0736800F0030003F087
:100B200003039B0043EA0010B36803F00303184378
:100B300017E000F00F0040F04000F6F797FDB068B6
:100B4000736800F00F0040EA0310C0B209E000F043
:100B50003F0040F08000F6F789FD3079F6F786FD1A
:100B6000307ABDE8F840F6F781BD06F10C0734464F
:100B70003A46002552F8043DAD0003F18001FF29FB
:100B800010D903F50041B1F5803F02D245F00105CF
:100B900008E003F50003B3F1807F34BF45F00205A0
:100BA00045F00305B242E5D165F03F00C0B2F6F76B
:100BB0005DFD05F00303022B207807D0032B0CD03A
:100BC000012B13D1F6F752FD60780FE0F6F74EFDDA
:100BD0006078F6F74BFDA07808E0F6F747FD6078FF
:100BE000F6F744FDA078F6F741FDE0780434F6F717
:100BF0003DFDBC424FEAA505DBD1F8BD10B504466A
:100C00007F2C06D964F07F00C0B2F6F72FFDE4090F
:100C1000F6E7E0B2BDE81040F6F728BD430083EAEE
:100C2000E070EBE72DE9F047304B86B093F8D8370A
:100C30000746012B01D004464AE004F024FE054695
:100C4000064603A96846FCF799FF039B049A02979E
:100C500013442B443F2B059519D90023684603A95B
:100C60000322FCF7B7FF039B3BB9049B2BB9204A37
:100C700013705370059BABB301E0FCF767FF039B58
:100C8000049A059E134433447F2B2BD8029FDFF830
:100C900060903946CA461AF8024BC4F18008B04544
:100CA00028BFB0460AEB04004444E4B2424604F0D4
:100CB0009BFD802C89F8004014D1C8EB06065046F5
:100CC00007EB0801324604F08FFD89F8006009E067
:100CD000254614F8011B21B1064B1868FAF7AFFB43
:100CE000F6E7ED1B284606B0BDE8F087FC2700209C
:100CF000AC240020742500200FB437B506AC54F89E
:100D0000045B4820F6F7B2FC2020F6F7AFFC2A4639
:100D100023460B4900200194F9F734F804460A20D1
:100D2000F6F7A4FC074BC4F1FF241A6804F57F040E
:100D3000FD3414441C6003B0BDE8304004B070477B
:100D4000390501082C2700200FB407B504AB53F870
:100D5000042B054900200193F9F714F803B05DF85E
:100D600004EB04B0704700BF3905010807B5064B16
:100D700006490093064B074A01930748074BF9F7CA
:100D800001F903B05DF804FB3F930108BBA0010823
:100D900017930108B4A0010899A101083393010831
:100DA00008B5037833B90C4B0C481978BDE80840F6
:100DB000F9F7E8B804F0BCFD02280CD8064B0C2269
:100DC0001870074B02FB0030064B02301860F9F731
:100DD000FDFA0548E5E708BD30250020BFA1010860
:100DE000AC2F00200C0F0020D694010808B5037822
:100DF0003BB90B4B0B4893F8B017BDE80840F9F727
:100E0000C1B804F095FD022808D8054B83F8B00757
:100E1000F9F736FAF9F7FEFA0348E8E708BD00BF2C
:100E2000FC270020C3A10108D694010838B5037837
:100E300003BB214B1B6801330F2B07D81F490C2222
:100E400002FB031295681C462DBB00E01C460134D2
:100E50000F2C01DD002400E005D818490C2202FB0C
:100E600004129568BDB99C42F1D11548BDE83840DF
:100E7000F9F788B804F05CFD0F28044605D80F4A3E
:100E80000C2303FB00239D682DB92146BDE83840A3
:100E90000C48F9F777B8084B1C60FAF709FA2146B5
:100EA0002A460948F9F76EF80C235C43034B185D9A
:100EB000BDE83840FAF710BA38000020E88301088E
:100EC000D0A10108E6A10108FEA1010873B50378CD
:100ED00013B9F8F71DF83DE01F4901AA04F089FD98
:100EE000002401462646254699B134B1012C08D18B
:100EF000084604F01DFD064603E0084604F018FD10
:100F000005461549002001AA04F073FD013401468D
:100F1000EAE70B2D02D911480C220BE0022C10D16C
:100F2000A6F57A73B3F57A7F07D90D484FF47A7135
:100F30004FF4FA62F7F769FF0CE00A4B03EB450345
:100F40005E80084B084803EB45032946B3F90220AD
:100F5000F9F718F802B070BDE4970108FA97010894
:100F6000B59B01083025002015A2010838B50D4CAD
:100F700005462368834206D1F8F736FB2046002158
:100F80004C2204F03CFCE36CAB4209D12846F8F754
:100F90002BFBBDE83840044800214C2204F02FBC54
:100FA00038BD00BF64270020B0270020034BDA695A
:100FB000D379591C1344D171187A70473025002019
:100FC00010B5FFF7F3FF84B2FFF7F0FF04EB00204A
:100FD00080B210BD10B5FFF7F3FF0446FFF7F0FF36
:100FE00004EB004010BD38B50446054D2146286A83
:100FF000FAF725FAEB6998796040987138BD00BF1F
:1010000030250020014BDB699879ECE73025002082
:1010100038B504460D462420FFF7E5FF4D20FFF7C5
:10102000E2FF002C084C14BF21203E20FFF7DBFF1D
:10103000E369002228469A71FFF7D5FFE36993F828
:101040004900BDE83840CEE73025002001460020A9
:10105000DEE710B50446C0B2FFF7C5FF200ABDE8C1
:101060001040C0E710B5044680B2FFF7F2FF200C35
:10107000BDE81040EDE737B5828883680446100666
:101080000D4641BF29494FF4CC7091F8B01700FBD1
:101090000133D10542BF26490C20097802F03F02F6
:1010A00048BF00FB0133042A12D006D8012A0DD014
:1010B000022A2FD193F900102DE0102A0AD0202AFD
:1010C0000AD0082A26D1B3F9001024E0197822E0CA
:1010D000198820E019681EE069461868F8F7D8FDFD
:1010E00001461448F8F74EFFF5B1E06801F06CFADC
:1010F0006946F8F7CDFD01460F48F8F743FF206930
:1011000001F062FA6946F8F7C3FD01460A48F8F7AC
:1011100039FF09E000210948F8F734FF25B10848F4
:10112000E1682269F8F72EFF03B030BDFC270020EC
:1011300030250020389601083196010849A10108A0
:1011400024A20108024B0146586AFAF778B900BF99
:101150003025002010B5441E14F8011F21B1034BA7
:10116000586AFAF76CF9F7E710BD00BF3025002088
:1011700010B503781BB9BDE810400948EAE704F050
:10118000D7FB0446062899BF214606480648062193
:10119000F8F7F8FE601EC0B2BDE81040F8F77AB963
:1011A0002BA2010872A201089EA20108F7B52A49E4
:1011B0002A4B91F828002A4D1C682A4B05EB800029
:1011C0001A88D0F8C010284B28481B7800914FF49B
:1011D0007A71B4FBF1F1F8F7D5FE254B2548196873
:1011E000254B0026B1FBF3F1F8F7CCFE234B1F682B
:1011F000F3B205EB8302D2F8D010E1B101249C4098
:101200003C4216D0220714D01D4A0B20D25C00FBB2
:101210000323134A1B4802EB8303D3F8F020F8F7AB
:10122000B1FE022C05D1184B197A11B11748F8F705
:10123000A9FE0136DCE71648FFF78CFF154B164870
:101240001A88164B92B2198840F2E47303B0BDE8D5
:10125000F040F8F797BE00BF302500209C1B00200F
:10126000E8830108881B002048000020C9A201086B
:101270004C0000200CA3010840420F00081600207B
:10128000400000201CA301084815002024A30108E9
:101290006CA301088A0E002028A30108880E0020F4
:1012A0002DE9F0410024804625460F4E4146A759BE
:1012B000384604F025FB58B139460C48F8F762FE71
:1012C00030190021FFF7D7FE0948FFF743FF01352A
:1012D00040F6CC3314349C42E7D11DB9BDE8F0414F
:1012E000044837E7BDE8F08188850108DD960108EC
:1012F0006CA30108639601082DE9F74F824604F0BC
:10130000C2FA054628B1012819D19AF800302A2BD3
:1013100015D15948FFF71EFF0024584E5848A159CF
:10132000F8F730FE30192946FFF7A5FE5548FFF7BC
:1013300011FF40F6CC3314349C42EED198E0504675
:101340003D2104F092FA002800F08D8003461D46EE
:1013500013F8012D202AFAD0441C204604F0E8FAA4
:1013600081462046F8F7FEFB0746CAEB05054FF01D
:10137000000B142404FB0BF4DFF8208108F5D07374
:10138000E6580193304604F07EFA844631466246C0
:101390005046CDF800C004F07FFADDF800C0019B94
:1013A000002856D1EAB2624553D11D194444D4F8FD
:1013B000AC0101F009F90146384601F00BFB0028A9
:1013C00045D0D4F8B00101F0FFF80146384601F0ED
:1013D000F7FA00283BD0B4F8A4319A0658BF4F461C
:1013E000142202FB0B881C0648BF2748D8F8A82106
:1013F00042BF90F8B0074FF4CC7404FB0022D8052C
:1014000042BF22480C24007803F03F0348BF04FB8E
:101410000022042B39460BD004D8013B012B0CD8F9
:1014200017700AE0102B05D0202B05D0082B04D113
:10143000118002E0176000E0176031461448F8F7A9
:10144000A1FD2846002103B0BDE8F04F13E6114886
:1014500005E00BF1010BBBF1970F8AD10E4803B0E9
:10146000BDE8F04F76E6504603B0BDE8F04F17E711
:1014700003B0BDE8F08F00BF5AA3010888850108BA
:10148000DD9601086CA30108FC2700203025002010
:101490006FA301087AA3010863960108E883010895
:1014A00010B50A48FFF756FE094B5C6A2046F9F76B
:1014B000BDFF18B90A20F9F7D4FEF7E7FAF7FCFBED
:1014C000F8F7B4FE034A044BDA6010BD9AA3010892
:1014D000302500200400FA0500ED00E008B50548BD
:1014E000FFF738FEFFF74EF8F8F7CAFEBDE80840F0
:1014F000D6E700BFA6A3010808B50448FFF72AFEF7
:10150000F8F7BEFEBDE80840CAE700BFBCA301086B
:101510002DE9F04F97498BB00B7813F0010F03F0D2
:10152000040200F07A81002A40F084819248066823
:1015300016F0806640F07E81980700F16E8143F0DE
:1015400004030B708D4B8E4F1A888E4B1A803B68AC
:101550001B0340F151818C4B80201E70F9F7BAFDBE
:1015600008B1FFF703FD894C2578012D40F0448137
:10157000874B93F8D61721B193F8D7270AB1914238
:1015800003D3012283F8D62711E096460846BEF120
:10159000000F06D090FBFEFC0EFB1C0C7046E646CE
:1015A000F5E791FBF0F192FBF0F283F8D61783F8A0
:1015B000D72793F8D827012A82BF754A002182F8DD
:1015C000D81793F8D897B9F1000F03D0B9F1010FEC
:1015D0002ED036E08020F8F745F9804688B3802188
:1015E000F8F71CF998F806206A4B022153F82230CC
:1015F0006070B3F5613F0CBF0222002298F9000031
:101600008DE806004A468021F8F702F8624B4FF455
:10161000FA721B68606003EB4303B3FBF2F31BB188
:10162000402BA8BF402300E00123237258B908E0F3
:101630005A4BDB682BB1FFF70FFA10B94023237226
:1016400001E00023D7E000211422554804F0D7F828
:10165000544B4F4803F17C022362F833A362524B90
:1016600090F8921162621B883A680029A4F8A031B0
:10167000C2F3C03318BF012390F884110593C2F35D
:10168000402C02F40063C2F34008484A04911168F8
:10169000C1F38002C1F3C0094179A1F119077C426D
:1016A0007C41012914BF2146012190F8D6470391BE
:1016B00090F8D7173E488C422CBF0021012106919B
:1016C0003C4900788A46D1F800B002906F1EFFB204
:1016D000791E132945D8DFE801F00C0C0C0C0C0C1A
:1016E0000C0C0AA7A931333D3F121212414703994E
:1016F0009DE00299B942B4BF0024012430E09BF878
:101700000010022913D1B91E5BF821000021CDF889
:1017100024C00893079201F03FF907AA4FF0010493
:1017200092E80C1008B14FF00004E4B218E00BEBA3
:1017300007014C79003418BF012411E0414676E0DE
:1017400023B10499481E4142414100E0194601F08D
:1017500001016CE061466AE0059968E0069966E07F
:1017600014B10121B9400E43142D25D80135EDB235
:10177000ACE700BF21300020900E0020F40E0020C6
:10178000901B00202A0E0020241600207025002027
:10179000FC270020B0910108101600201000002046
:1017A0007C2500209C250020FC1A00200816002023
:1017B0007C160020D40E0020DAF800001F4C853083
:1017C0001921C4F8A461F8F7D9F80023C4F8AC31A2
:1017D000A4F8B031A4F8B231C4F8BC31C4F8C031B7
:1017E000174BD4F8B8211B6884F8A801C4F8C43199
:1017F000C4F8B42102232370114B124A1B6892F8DB
:10180000E0214FF47A7101FB02330F4A0520136087
:101810000BB0BDE8F04FF9F75FBD5AB901200BB02E
:10182000BDE8F04FF9F788BD494600E011460029B0
:1018300097D19BE70BB0BDE8F08F00BF702500206B
:101840009C1B0020FC270020D80D002010B5154A55
:101850001378590725D523F004031370124B1B6826
:101860001B0319D5114C2378A3F10802012A0BD8C8
:10187000FF200021F5F79EFF0D4B1B68C4F8C43113
:10188000FFF71AF90A2306E0012B05D90A2B03D02A
:10189000FFF7F8F8012323700420BDE81040F9F7A2
:1018A0001BBD10BD21300020901B002070250020A2
:1018B0009C1B00200C4B0D49DA684378D243C2F3DD
:1018C0000222C2F10402934002781B01DBB20A44F7
:1018D00082F8003303780122580903F01F0302FA4B
:1018E00003F341F82030704700ED00E000E100E034
:1018F00070B5184B9B894FF47A7342B311B10C78D1
:10190000013107E0FF2405E04FF6FF75013B9BB274
:10191000AB420FD00F4D2E89B607F5D5A4B2AC81DE
:101920000C4C2589ED070BD44FF6FF74013B9BB29D
:10193000A342F5D1084A138801339BB2138006E015
:10194000A489A4B208B104700130013AD5E701209E
:1019500070BD00BF003800403C27002040F2E93352
:101960000F4A1189890704D4013B9BB2002BF7D1A0
:101970000BE040F2E93380B29081094A1189C9072E
:101980000AD4013B9BB2002BF7D1064AFF201388F3
:1019900001339BB2138070479089C0B2704700BF7B
:1019A000003800403C27002007B50B4A0B489369DC
:1019B00001A943F0100393614FF40053ADF80430D4
:1019C00002238DF8073010238DF80630F4F7A3FEBC
:1019D00003B05DF804FB00BF00100240001001409E
:1019E00010B504460F4B185CF5F797FA0E4800EB5C
:1019F0004400B0F90210B1F57A7F05DBB1F5FA6F5A
:101A0000A8BF4FF4FA6101E04FF47A71A1F57A7141
:101A10000A2391FBF3F1BDE810400920C9B2FEF79B
:101A2000A9BA00BF67AD01083C270020031EB8BF5C
:101A30002D2210B5B8BF58420C46B8BF01F8012B93
:101A40000A22F8F78BF900230370204610BD10B569
:101A50000446B0F90000FFF7E1F8B4F90200FFF71F
:101A6000DDF8B4F90400BDE81040FFF7D7B810B5B1
:101A700004460068FFF7D2F86068FFF7CFF8A06867
:101A8000BDE81040FFF7CAB82DE9F74F0120F7F77E
:101A9000E9FE002488B3012C2FD84FF04C0909FB34
:101AA00004FA174E06EB0A0808F17007BD7815B165
:101AB0000134E4B2EEE790F9003090F804E0184603
:101AC000104B03228DE8240001212A4653F82E30C2
:101AD000F7F79EFD834660B106F128005044294681
:101AE0004A4603F08CFE01231C44C8F828B0BB70A2
:101AF000E4B20120F7F79CFECCE703B0BDE8F08F1D
:101B00003C270020B091010808B52A221148002185
:101B100003F075FE104B002210490420515C013285
:101B200083F8F011052183F8F5018A424FF0000097
:101B300083F8F41183F8F70183F8F61103F1080331
:101B4000EAD1074B0122A3F8B222522283F8AE2237
:101B500008BD00BFEA290020FC27002062AD010873
:101B60003C27002070B50646441E14F8011F89B1B9
:101B7000094D284603F079FE0028F6D005F1080348
:101B800098423FBF054B401BC018A31B38BF80F8CD
:101B90004832EAE770BD00BF67AD01083C2700206E
:101BA00007B51C4B03F6A802C3F8A42893F85022EB
:101BB0005AB1012A14D1032183F8AA18072183F806
:101BC000AC2883F8AB180C2208E0022183F8AA188D
:101BD000032183F8AC2883F8AB18072283F8A828E0
:101BE0000D4A0E4B40201A60F7F73CFE70B10122FF
:101BF000002390F9000040218DE80C00084A4FF4C2
